:100000000C94BD090C94E5090C94E5090C94E509E0
:100010000C94E5090C94E5090C94E5090C94E509A8
:100020000C94E5090C94E5090C94E5090C94E50998
:100030000C94E5090C9481530C94E5090C94E509A2
:100040000C94E5090C94FD630C943E2C0C94E5098A
:100050000C94002E0C94E5090C94E5090C94E50928
:100060000C94E5090C94E5090C94E5090C94E50958
:100070000C94E5090C94E5090C94E509084AD73B72
:100080003BCE016E84BCBFFDC12F3D6C74319ABD67
:1000900056833DDA3D00C77F11BED9E4BB4C3E918B
:1000A0006BAAAABE000000803F05A84CCDB2D44E7A
:1000B000B93836A9020C50B9918688083CA6AAAA7C
:1000C0002ABE000000803F6563686F3A00656E716C
:1000D0007565696E67202200220073746172740076
:1000E000506F7765725570002045787465726E6147
:1000F0006C205265736574002042726F776E206FBA
:100100007574205265736574002057617463686468
:100110006F672052657365740020536F6674776152
:100120007265205265736574004D61726C696E2052
:1001300000312E302E302052433200204C61737437
:1001400020557064617465643A2000323031322D7C
:1001500030372D323900207C20417574686F723A37
:10016000200069776A002046726565204D656D6FD5
:1001700072793A20002020506C616E6E6572427573
:100180006666657242797465733A200053746F72C3
:1001900065642073657474696E6773207265747228
:1001A00065697665643A006F6B00446F6E65207315
:1001B0006176696E672066696C652E004572726FA4
:1001C000723A004C696E65204E756D6265722069E9
:1001D00073206E6F74204C617374204C696E6520BF
:1001E0004E756D6265722B312C204C617374204CFE
:1001F000696E653A00636865636B73756D206D6940
:10020000736D617463682C204C617374204C696E4B
:10021000653A004E6F20436865636B73756D207798
:10022000697468206C696E65206E756D6265722CEC
:10023000204C617374204C696E653A004E6F204CFF
:10024000696E65204E756D626572207769746820ED
:10025000636865636B73756D2C204C617374204CFF
:10026000696E653A006F6B005072696E746572203A
:1002700073746F707065642064657520746F206599
:1002800072726F72732E20466978207468652065DB
:1002900072726F7220616E6420757365204D3939FA
:1002A0003920746F2072657374617274212E202856
:1002B00054656D7065726174757265206973207222
:1002C000657365742E2053657420697420626566B9
:1002D0006F72652072657374617274696E6729004C
:1002E000446F6E65207072696E74696E672066690E
:1002F0006C6500426567696E2066696C65206C6993
:10030000737400456E642066696C65206C69737453
:10031000006F6B20543A00202F0020423A00202F1B
:100320000020403A00543A0020453A0020573A0055
:10033000543A0020453A0020423A004649524D576F
:100340004152455F4E414D453A4D61726C696E2098
:1003500056313B20537072696E7465722F677262FA
:100360006C206D617368757020666F722067656EB2
:1003700036204649524D574152455F55524C3A68D6
:100380007474703A2F2F7777772E6D656E64656C75
:100390002D70617274732E636F6D2050524F544FE5
:1003A000434F4C5F56455253494F4E3A312E302001
:1003B0004D414348494E455F545950453A4D656E4D
:1003C00064656C2045585452554445525F434F551F
:1003D0004E543A310A00583A00593A005A3A004508
:1003E0003A0020436F756E7420583A00593A005A0B
:1003F0003A00785F6D696E3A00795F6D696E3A0018
:100400007A5F6D696E3A00556E6B6E6F776E206322
:100410006F6D6D616E643A220022005365747469D9
:100420006E67732053746F726564005374657073E4
:100430002070657220756E69743A0020204D393243
:10044000205800205900205A002045004D6178694D
:100450006D756D2066656564726174657320286DC5
:100460006D2F73293A0020204D3230332058002060
:100470005900205A002045004D6178696D756D2046
:10048000416363656C65726174696F6E20286D6D80
:100490002F7332293A0020204D323031205800206D
:1004A0005900205A00204500416363656C65726104
:1004B00074696F6E3A20533D616363656C65726168
:1004C00074696F6E2C20543D726574726163742080
:1004D000616363656C65726174696F6E0020204DA5
:1004E000323034205300205400416476616E6365DD
:1004F00064207661726961626C65733A20533D4D88
:10050000696E20666565647261746520286D6D2F63
:1005100073292C20543D4D696E2074726176656C90
:1005200020666565647261746520286D6D2F73297E
:100530002C20423D6D696E696D756D207365676D28
:10054000656E742074696D6520286D73292C2058A0
:100550003D6D6178696D756D207859206A65726BA3
:1005600020286D6D2F73292C20205A3D6D617869EC
:100570006D756D205A206A65726B20286D6D2F7322
:10058000290020204D3230352053002054002042D5
:1005900000205800205A00204500486F6D65206FEC
:1005A000666673657420286D6D293A0020204D32EF
:1005B0003036205800205900205A005049442073FA
:1005C000657474696E67733A002020204D333031B2
:1005D000205000204900204400526573656E643A43
:1005E000006F6B005072696E7465722068616C7484
:1005F00065642E206B696C6C28292063616C6C65C6
:1006000064202121005072696E7465722073746FCA
:10061000707065642064657520746F206572726FF8
:1006200072732E2046697820746865206572726F37
:100630007220616E6420757365204D3939392074DC
:100640006F2072657374617274212E202854656D59
:100650007065726174757265206973207265736567
:10066000742E20536574206974206265666F72650C
:100670002072657374617274696E6729007C3C3EF8
:100680005E2B3D3F2F5B5D3B2C2A225C006563683F
:100690006F3A0020636F6C642065787472757369BB
:1006A0006F6E2070726576656E7465640020746F7D
:1006B0006F206C6F6E6720657874727573696F6EEA
:1006C0002070726576656E746564006563686F3A64
:1006D00000656E6473746F7073206869743A2000EB
:1006E00020583A0020593A00205A3A0024F404D9FC
:1006F000201BC40C5C0E9804C4095F0265077101DD
:10070000F405F900FB04B30048048700C103690045
:100710005803550003034500BE023A00840231002D
:1007200053022A002902250004022000E4011C00D3
:10073000C8011900AF0117009801140084011300CB
:10074000710110006101100051010E0043010D0004
:1007500036010B002B010B0020010B0015010900D5
:100760000C01090003010800FB000800F300080069
:10077000EB000700E4000600DE000600D8000600DB
:10078000D2000600CC000500C7000500C20005002D
:10079000BD000400B9000400B5000400B10004006D
:1007A000AD000400A9000400A5000300A20003009E
:1007B0009F0004009B0003009800030095000200C6
:1007C00093000300900003008D0002008B000300E3
:1007D00088000200860002008400030081000200FD
:1007E0007F0002007D0002007B0002007900020011
:1007F0007700010076000200740002007200010020
:10080000710002006F0002006D0001006C00020028
:100810006A00010069000200670001006600010033
:100820006500010064000200620001006100010037
:10083000600001005F0002005D0001005C0001003B
:100840005B0001005A00010059000100580001003E
:10085000570001005600010055000100540001003E
:10086000530000005300010052000100510001003C
:10087000500001004F0001004E0000004E0001003A
:100880004D0001004C0001004B0000004B00010036
:100890004A00010049000100480000004800010032
:1008A000470001004600000046000100450000002E
:1008B0004500010044000100430000004300010026
:1008C0004200000042000100410000004100010020
:1008D000400001003F0000003F0001003E0000001A
:1008E0003E0001003D0000003D0001003C00000012
:1008F0003C0000003C0001003B0000003B00010008
:100900003A0000003A0001003900000039000100FF
:1009100038000000380000003800010037000000F7
:1009200037000100360000003600000036000100EC
:1009300035000000350000003500010034000000E3
:1009400034000000340001003300000033000000D8
:1009500033000100320000003200000032000100CC
:1009600031000000310000003100010030000000C3
:1009700030000000300001002F0000002F000000B8
:100980002F0000002F0001002E0000002E000000AC
:100990002E0001002D0000002D0000002D000000A1
:1009A0002D0001002C0000002C0000002C00000095
:1009B0002C0001002B0000002B0000002B00000089
:1009C0002B0001002A0000002A0000002A0000007D
:1009D0002A00010029000000290000002900000071
:1009E0002900000029000100280000002800000064
:1009F0002800000028000000280001002700000057
:100A00002700000027000000270000002700010049
:100A1000260000002600000026000000260000003E
:100A20002600010025000000250000002500000030
:100A30002500000025000000250001002400000022
:100A40002400000024000000240000002400010015
:100A5000230000002300000023000000230000000A
:100A600023000000230000002300010022000000FA
:100A700022000000220000002200000022000000EE
:100A800022000100210000002100000021000000E0
:100A900021000000210000002100000021000100D1
:100AA00020000000200000002000000020000000C6
:100AB00020000000200000002000000020000100B5
:100AC0001F0000001F0000001F0000001F000000AA
:100AD0001F0000001F0000001F0001001E0000009A
:100AE0001E0000001E0000001E00000024F4D43090
:100AF00050C38E20C2A24017828B7011127A910DC2
:100B0000816CD90AA861E108C7586607615143069C
:100B10001E4B5D05C145A7041A411104093D980308
:100B2000713931034036DB0265339102D43054020F
:100B3000802E1D02632CEE01752AC501B028A0018C
:100B4000102781018F2564012B244B01E022340101
:100B5000AC211F018D200D01801FFC00841EED00C3
:100B6000971DDF00B81CD200E61BC600201BBC008E
:100B7000641AB200B219A8000A19A0006A189900F4
:100B8000D117910040178B00B516840031167E00F6
:100B9000B31579003A157300C7146F0058146A0032
:100BA000EE1366008813630025135E00C7125B0016
:100BB0006C12570015125400C111510070114F00F2
:100BC00021114B00D61049008D10470046104400FB
:100BD00002104200C00F4000800F3E00420F3C0058
:100BE000060F3B00CB0E3800930E37005C0E35002D
:100BF000270E3400F30D3200C10D3100900D30008E
:100C0000600D2E00320D2D00050D2C00D90C2B008F
:100C1000AE0C2900850C29005C0C2700350C270040
:100C20000E0C2600E80B2400C40B2400A00B2300AC
:100C30007D0B23005A0B2100390B2100180B2000DB
:100C4000F80A1F00D90A1E00BB0A1E009D0A1D00DB
:100C5000800A1D00630A1C00470A1B002C0A1B00A7
:100C6000110A1A00F7091A00DD091900C409190050
:100C7000AB091900920917007B09180063091700D6
:100C80004C09160036091600200916000A0915003D
:100C9000F5081500E0081400CC081400B80814008A
:100CA000A4081400900813007D0812006B081300BC
:100CB00058081200460812003408110023081100D9
:100CC0001208110001081100F0071000E0071000E1
:100CD000D0071000C0071000B0070F00A1071000D8
:100CE00091070E0083070F0074070F0065070E00C1
:100CF00057070E0049070E003B070D002E070E0098
:100D000020070D0013070D0006070D00F9060C0063
:100D1000ED060D00E0060C00D4060C00C8060C0021
:100D2000BC060C00B0060C00A4060B0099060C00D3
:100D30008D060B0082060B0077060B006C060B007D
:100D400061060A0057060B004C060A0042060A001C
:100D500038060A002E060A0024060A001A060A00AF
:100D60001006090007060A00FD050900F405090040
:100D7000EB050900E2050900D9050900D0050900C5
:100D8000C7050900BE050900B5050800AD05080046
:100D9000A50509009C050800940508008C050800BD
:100DA000840508007C050800740508006C05070030
:100DB000650508005D050700560508004E0507009B
:100DC0004705070040050800380507003105070002
:100DD0002A050700230507001C0506001605070065
:100DE0000F0507000805060002050700FB040600C2
:100DF000F5040700EE040600E8040600E20407001C
:100E0000DB040600D5040600CF040600C904060072
:100E1000C3040600BD040600B7040600B1040500C3
:100E2000AC040600A6040600A00405009B0406000E
:100E300095040500900406008A0405008504050059
:100E4000800406007A04050075040500700405009E
:100E50006B04050066040500610405005C040500E0
:100E600057040500520405004D0405004804050020
:100E7000430405003E0404003A040500350405005F
:100E8000300404002C04050027040400230405009A
:100E90001E0404001A0404001604050011040400D2
:100EA0000D04040009040500040404000004040007
:100EB000FC030400F8030400F4030400F00304003E
:100EC000EC030400E8030400E4030400E00304006E
:100ED000DC030400D8030400D4030400D00304009E
:100EE000CC030400C8030300C5030300206269614A
:100EF000733A200020643A2000206D696E3A200089
:100F0000206D61783A2000204B753A2000205475FE
:100F10003A200020436C61736963205049442000EB
:100F2000204B703A2000204B693A2000204B643A55
:100F30002000504944204175746F74756E652066B9
:100F400061696C6564212054656D706572617475AA
:100F5000726520746F2068696768006F6B20543A6F
:100F60000020403A00504944204175746F74756EFA
:100F700065206661696C6564212074696D656F75B3
:100F80007400504944204175746F74756E65206615
:100F9000696E6973686564202120506C6163652007
:100FA000746865204B702C204B6920616E64204B67
:100FB0006420636F6E7374616E747320696E207445
:100FC000686520636F6E66696775726174696F6EBC
:100FD0002E68004572726F723A00202D20496E769D
:100FE000616C6964206578747275646572206E75D1
:100FF0006D626572210070012C0190012701B00122
:101000002201C0011D01F00118011002130130027C
:101010000E016002090190020401C002FF000003FA
:10102000FA004003F5008003F000D003EB00200439
:10103000E6007004E100E004DC004005D700C005D4
:10104000D2004006CD00D006C8008007C30030089B
:10105000BE00F008B900C009B400B00AAF00B00B80
:10106000AA00D00CA500000EA000500F9B00C010DD
:1010700096005012910000148C00C0158700B01724
:101080008200B0197D00D01B7800001E7300402044
:101090006E0090226900F024640040275F009029D0
:1010A0005A00E02B5500102E500020304B0010321B
:1010B0004600E033410090353C001037370070386F
:1010C0003200A0392D00B03A2800A03B2300603C3C
:1010D0001E00103D1900903D1400103E0F00703EA0
:1010E0000A00C03E0500003F0000202D20496E761A
:1010F000616C6964206578747275646572206E75C0
:101100006D6265722021003A2045787472756465BD
:1011100072207377697463686564206F66662E2039
:101120004D415854454D502074726967676572652A
:10113000642021003A2045787472756465722073CA
:1011400077697463686564206F66662E204D494E2A
:1011500054454D502074726967676572656420213B
:101160000054656D706572617475726520686561A3
:10117000746564206265642073776974636865646C
:10118000206F66662E204D415854454D5020747294
:1011900069676765726564202121006563686F3A3D
:1011A00000534420696E6974206661696C00457261
:1011B000726F723A00766F6C756D652E696E697428
:1011C000206661696C6564006F70656E526F6F7444
:1011D000206661696C656400534420636172642019
:1011E0006F6B006F70656E206661696C65642C20A2
:1011F00046696C653A20002E0046696C65206F7068
:10120000656E65643A002053697A653A0046696CF8
:10121000652073656C6563746564006F70656E202E
:101220006661696C65642C2046696C653A20002E05
:10123000006F70656E206661696C65642C2046697C
:101240006C653A20002E0057726974696E672074CD
:101250006F2066696C653A20006F70656E2066616C
:10126000696C65642C2046696C653A20002E004646
:10127000696C652064656C657465643A0044656CEE
:101280006574696F6E206661696C65642C204669BF
:101290006C653A20002E005344207072696E7469A8
:1012A0006E67206279746520002F004E6F742053A2
:1012B00044207072696E74696E67006572726F7235
:1012C0002077726974696E6720746F2066696C6537
:1012D00000000000010200000000000000040307FD
:1012E00006000000000000000000000000000000F8
:1012F0000001020408102040800102040810204070
:101300008001020408102040808040201008040260
:1013100001020202020202020204040404040404A0
:10132000040303030303030303010101010101019A
:1013300001002225282B002124272A494E46494E08
:101340004954594E414E000020410000C84200401F
:101350001C4620BCBE4CCA1B0E5AAEC59D74CDCCDB
:10136000CC3D0AD7233C17B7D13877CC2B32959593
:10137000E6241FB14F0A362C3A2C11241FBECFEFA2
:10138000D0E1DEBFCDBF12E0A0E0B1E0E0EDF5EFCF
:1013900002C005900D92A63EB107D9F71EE0A6EE59
:1013A000B2E001C01D92A135B107E1F713E1C8E732
:1013B000D3E104C02297FE010E94E674C637D1072C
:1013C000C9F70E94082C0C94DB7A0C940000CF9291
:1013D000DF92EF92FF920F931F93CF93DF93EC0175
:1013E000CC0FDD1FCC0FDD1FFE01EB50FD4FC08089
:1013F000D180E280F3808E010F5F1C4FFE01EA591D
:10140000FD4FA701960160817181828193810E94C5
:10141000DB6FF80160837183828393838E010751B0
:101420001D4FCE58DD4FA7019601688179818A81D1
:101430009B810E94DB6FF8016083718382839383B9
:10144000DF91CF911F910F91FF90EF90DF90CF90A0
:10145000089507C03091C00035FFFCCF2093C6002F
:101460000196FC0124912111F5CF22E030E08DECB2
:1014700095E00C944430CF93DF93C7ECD0E0FE01AD
:1014800007C09091C00095FFFCCF8093C6003196B5
:1014900084918111F6CFEBE2F4E007C09091C00097
:1014A00095FFFCCF8093C600319684918111F6CFD1
:1014B0008091C00085FFFCCF8AE08093C600FE01CA
:1014C0008491E7ECF0E008C09091C00095FFFCCF5C
:1014D0008093C600319684918111F6CF40917F0DA3
:1014E0005091800D6091810D7091820D8BE394E09D
:1014F0000E94290A4091830D5091840D6091850DC1
:101500007091860D83E494E00E94290A4091870D32
:101510005091880D6091890D70918A0D86E494E058
:101520000E94290A40918B0D50918C0D60918D0D78
:1015300070918E0D89E494E00E94290A8091C00088
:1015400085FFFCCF8AE08093C600FE018491E7EC22
:10155000F0E008C09091C00095FFFCCF8093C600DA
:10156000319684918111F6CFECE4F4E007C09091BC
:10157000C00095FFFCCF8093C60031968491811105
:10158000F6CF8091C00085FFFCCF8AE08093C60033
:10159000FE018491E7ECF0E008C09091C00095FF57
:1015A000FCCF8093C600319684918111F6CF409193
:1015B0008F0D5091900D6091910D7091920D86E676
:1015C00094E00E94290A4091930D5091940D6091EE
:1015D000950D7091960D8FE694E00E94290A409136
:1015E000970D5091980D6091990D70919A0D82E729
:1015F00094E00E94290A40919B0D50919C0D6091AE
:101600009D0D70919E0D85E794E00E94290A8091BE
:10161000C00085FFFCCF8AE08093C600FE01849164
:10162000E7ECF0E008C09091C00095FFFCCF8093FC
:10163000C600319684918111F6CFE8E7F4E007C047
:101640009091C00095FFFCCF8093C60031968491A5
:101650008111F6CF8091C00085FFFCCF8AE0809396
:10166000C600FE018491E7ECF0E008C09091C00054
:1016700095FFFCCF8093C600319684918111F6CFFF
:10168000E6E9F4E007C09091C00095FFFCCF80939D
:10169000C600319684918111F6CF40916F0D509123
:1016A000700D6091710D7091720D2AE030E08DEC3B
:1016B00095E00E94272FEFE9F4E007C09091C00069
:1016C00095FFFCCF8093C600319684918111F6CFAF
:1016D0004091730D5091740D6091750D7091760D60
:1016E0002AE030E08DEC95E00E94272FE2EAF4E05A
:1016F00007C09091C00095FFFCCF8093C600319643
:1017000084918111F6CF4091770D5091780D6091C1
:10171000790D70917A0D2AE030E08DEC95E00E9411
:10172000272FE5EAF4E007C09091C00095FFFCCFB9
:101730008093C600319684918111F6CF40917B0D44
:1017400050917C0D60917D0D70917E0D2AE030E00E
:101750008DEC95E00E94272F8091C00085FFFCCF83
:101760008AE08093C600FE018491E7ECF0E008C0B7
:101770009091C00095FFFCCF8093C6003196849174
:101780008111F6CFE8EAF4E007C09091C00095FF20
:10179000FCCF8093C600319684918111F6CF809161
:1017A000C00085FFFCCF8AE08093C600FE018491D3
:1017B000E7ECF0E008C09091C00095FFFCCF80936B
:1017C000C600319684918111F6CF4091670D5091FA
:1017D000680D6091690D70916A0D8DED94E00E9425
:1017E000290A4091630D5091640D6091650D7091CF
:1017F000660D86EE94E00E94290A8091C00085FF64
:10180000FCCF8AE08093C600FE018491E7ECF0E013
:1018100008C09091C00095FFFCCF8093C600319620
:1018200084918111F6CFE9EEF4E007C09091C000F9
:1018300095FFFCCF8093C600319684918111F6CF3D
:101840008091C00085FFFCCF8AE08093C600FE0136
:101850008491E7ECF0E008C09091C00095FFFCCFC8
:101860008093C600319684918111F6CF40916B0D23
:1018700050916C0D60916D0D70916E0D82E895E048
:101880000E94290A4091530D5091540D6091550DBD
:101890007091560D8BE895E00E94290AEEE8F5E07C
:1018A00007C09091C00095FFFCCF8093C600319691
:1018B00084918111F6CF40919F0D5091A00D6091C0
:1018C000A10D7091A20D2AE030E08DEC95E00E9410
:1018D000272F40915F0D5091600D6091610D7091C7
:1018E000620D81E995E00E94290A40915B0D5091BB
:1018F0005C0D60915D0D70915E0D84E995E00E9434
:10190000290A4091570D5091580D6091590D7091D1
:101910005A0D87E995E00E94290A8091C00085FF51
:10192000FCCF8AE08093C600FE018491E7ECF0E0F2
:1019300008C09091C00095FFFCCF8093C6003196FF
:1019400084918111F6CFEAE9F5E007C09091C000DB
:1019500095FFFCCF8093C600319684918111F6CF1C
:101960008091C00085FFFCCF8AE08093C600FE0115
:101970008491E7ECF0E008C09091C00095FFFCCFA7
:101980008093C600319684918111F6CF4091F50283
:101990005091F6026091F7027091F8028CEA95E09E
:1019A0000E94290A4091F9025091FA026091FB02CB
:1019B0007091FC0285EB95E00E94290A4091FD029E
:1019C0005091FE026091FF027091000388EB95E058
:1019D0000E94290A8091C00085FFFCCF8AE0809395
:1019E000C600FE018491E7ECF0E008C09091C000D1
:1019F00095FFFCCF8093C600319684918111F6CF7C
:101A0000EBEBF5E007C09091C00095FFFCCF809311
:101A1000C600319684918111F6CF8091C00085FF78
:101A2000FCCF8AE08093C600FE01C491E7ECF0E0B1
:101A300008C08091C00085FFFCCFC093C6003196DE
:101A4000C491C111F6CF40913A0150913B01609190
:101A50003C0170913D0189EC95E00E94290AE3ED7B
:101A6000F5E007C09091C00095FFFCCF8093C600C1
:101A7000319684918111F6CF2DEB37E346E05EE39A
:101A80006091360170913701809138019091390150
:101A90000E94BB70AB01BC0122E030E08DEC95E010
:101AA0000E944430E6EDF5E007C09091C00095FF3C
:101AB000FCCF8093C600319684918111F6CF2DEB37
:101AC00037E346E05EE3609132017091330180912B
:101AD0003401909135010E948973AB01BC0122E071
:101AE00030E08DEC95E00E9444308091C00085FF8D
:101AF000FCCF8AE08093C600DF91CF910895CF9309
:101B0000DF9300D0CDB7DEB780914B0E90914C0E95
:101B10009E012F5F3F4F009719F421553E4002C0B0
:101B2000281B390B3A83298389819A810F900F9062
:101B3000DF91CF9108952091F2033091F303243087
:101B400031050CF06AC04091F4035091F50360E652
:101B5000649F9001659F300D1124BC01C9018A501A
:101B60009C4F0E94AC77E7ECF0E007C09091C0007A
:101B700095FFFCCF8093C600319684918111F6CFFA
:101B8000EDECF0E007C09091C00095FFFCCF809392
:101B9000C600319684918111F6CF8091F403909123
:101BA000F50320E6289FF001299FF00D1124EA504B
:101BB000FC4F06C09091C00095FFFCCF8093C600FB
:101BC00081918111F7CFE8EDF0E007C09091C0005E
:101BD00095FFFCCF8093C600319684918111F6CF9A
:101BE0008091C00085FFFCCF8AE08093C600809181
:101BF000F4039091F503019664E070E00E94727422
:101C00009093F5038093F4038091F2039091F30392
:101C100001969093F3038093F203089580918005D9
:101C20009091810560E070E001960C94EA748091D7
:101C30008005909181054AE050E060E070E00196F7
:101C40000C94417640917A0550917B0590E6949FE3
:101C50009001959F300D1124682F70E0C9018A50C2
:101C60009C4F0E94A177909381058093800521E08D
:101C7000892B09F420E0822F08950E94882C60931C
:101C80009205709393058093940590939505E09148
:101C90007A05F0917B05EA58FA4F8081811114C0D2
:101CA000E1EEF5E007C09091C00095FFFCCF809376
:101CB000C600319684918111F6CF8091C00085FFD6
:101CC000FCCF8AE08093C60008958DEC95E00E94D9
:101CD000892EE9EDF5E007C09091C00095FFFCCF9B
:101CE0008093C600319684918111F6CF409186058C
:101CF0005091870560918805709189054F5F5F4F0E
:101D00006F4F7F4F2AE030E08DEC95E00E943A2F34
:101D10008091C00085FFFCCF8AE08093C6000C94C0
:101D20003D0E2F923F924F925F926F927F928F92D1
:101D30009F92AF92BF92CF92DF92EF92FF920F935A
:101D40001F93CF93DF93CDB7DEB76F970FB6F8949D
:101D5000DEBF0FBECDBF70E6772EE4E04E2E512CD5
:101D6000E8E6F2E08490FAE0BF2EE5E6F2E0A49027
:101D70009924939480914E0690914F06209150069D
:101D800030915106821B930B8F779927892B09F08D
:101D900004C234C38D3051F08A3321F490917D0513
:101DA000992321F02F3531050CF4DAC121153105C5
:101DB00009F49FC28091F4039091F503789E70011D
:101DC000799EF00C1124F701E20FF31FEA50FC4F4B
:101DD000108220917D052111BEC110927D05FC016C
:101DE000EA58FA4F108287010A501C4F6EE470E0E7
:101DF000C8010E94A177009709F404C1909381055E
:101E000080938005801B910B8E0D9F1D4AE050E052
:101E100060E070E089509C4F0E944176609382059B
:101E2000709383058093840590938505C090860503
:101E3000D0908705E0908805F0908905970186018C
:101E40000F5F1F4F2F4F3F4F601771078207930798
:101E5000C1F12091F4033091F503729EC001739E8D
:101E6000900D112463E771E08A509C4F0E94D07757
:101E7000892B39F5ECEBF1E007C09091C00095FF9C
:101E8000FCCF8093C600319684918111F6CFE3ECAC
:101E9000F1E007C09091C00095FFFCCF8093C60091
:101EA000319684918111F6CF2AE030E0B701A60186
:101EB0008DEC95E00E943A2F8091C00085FFFCCF09
:101EC0008AC08091F4039091F503789E1001799E69
:101ED000300C112481010A501C4F6AE270E0C801E5
:101EE0000E94A177009721F450C0F3262F5F02C013
:101EF00020E0F12CF101E20FF11DEA50FC4F30819E
:101F00003A3299F79093810580938005801B910B5D
:101F1000820D931D60E070E089509C4F0E94EA742E
:101F20000E9423712F2D30E02617370709F459C07E
:101F3000ECEBF1E007C09091C00095FFFCCF8093DF
:101F4000C600319684918111F6CFE5EFF1E007C02C
:101F50009091C00095FFFCCF8093C600319684918C
:101F60008111F6CF409186055091870560918805D3
:101F7000709189052AE030E08DEC95E00E943A2FBF
:101F80008091C00085FFFCCF26C0ECEBF1E007C0DC
:101F90009091C00095FFFCCF8093C600319684914C
:101FA0008111F6CFE3E1F2E007C09091C00095FF08
:101FB000FCCF8093C600319684918111F6CF2AE040
:101FC00030E0B701A6018DEC95E00E943A2F809198
:101FD000C00085FFFCCF8AE08093C6000E94650E9A
:101FE00047C08091820590918305A0918405B091AE
:101FF00085058093860590938705A0938805B09307
:1020000089053BC06AE270E0C8010E94A177892B74
:10201000A1F1ECEBF1E007C09091C00095FFFCCF7F
:102020008093C600319684918111F6CFECE3F2E003
:1020300007C09091C00095FFFCCF8093C6003196F9
:1020400084918111F6CF409186055091870560916A
:102050008805709189052AE030E08DEC95E00E94BA
:102060003A2F8091C00085FFFCCF8AE08093C600A4
:1020700010927F0510927E05EFC18091F40390913C
:10208000F503789E8001799E100D112466EFE62EEF
:1020900063E0F62EE00EF11E67E470E0C7010E94D7
:1020A000A177009709F442C0909381058093800541
:1020B0008E199F09800F911F60E070E089509C4F3E
:1020C0000E94EA740E9423716430710578F5809152
:1020D000E602811117C080911803811127C08A2D53
:1020E000E5E6F2E008C09091C00095FFFCCF809338
:1020F000C600319684918111F6CF8091C00085FF92
:10210000FCCF12C0882DE8E6F2E008C09091C00034
:1021100095FFFCCF8093C600319684918111F6CF54
:102120008091C00085FFFCCFB092C6008091F4037F
:102130009091F5030196B2010E9472749093F50399
:102140008093F4038091F2039091F30301969093AE
:10215000F3038093F20310927F0510927E050ACE5E
:102160008B3311F490927D0590917D05911102CEF3
:102170004091F4035091F503749ED001759EB00D0B
:102180001124A20FB31FAA50BC4F8C932F5F3F4F57
:1021900030937F0520937E05EDCD8091F2039091E1
:1021A000F30304970CF42FC129C180917E0590910F
:1021B0007F05892B09F4E8C04FC14D3081F04A33C7
:1021C00021F420917D05222351F020917E0530914C
:1021D0007F052F3531051CF4019609F0B8C04091F8
:1021E000E8035091E9036091EA037091EB03809159
:1021F000E0039091E103A091E203B091E30348175B
:1022000059076A077B0708F46DC08F8DE0EEF2E096
:1022100008C09091C00095FFFCCF8093C600319616
:1022200084918111F6CF8091C00085FFFCCF709220
:10223000C6000E94882C60938A0570938B0580935A
:102240008C0590938D0520918E0530918F054091DE
:10225000900550919105621B730B840B950BA701A0
:1022600096010E948674CA01B901A50194010E94D9
:1022700086747F936F933F932F9388E791E09F93AA
:102280008F933F922F920E94EA77862D0FB6F89493
:10229000DEBF0FBECDBFE7ECF0E008C09091C000FC
:1022A00095FFFCCF8093C600319684918111F6CFC3
:1022B000F10106C09091C00095FFFCCF8093C6004D
:1022C00081918111F7CF8091C00085FFFCCF709282
:1022D000C60088E193E00E94076D61E088E193E029
:1022E0000E94FE6B20917E0530917F0521153105FE
:1022F00019F410927D05B0C08091F4039091F5031C
:10230000189FF001199FF00D1124E20FF31FEA50FE
:10231000FC4F1082FC01EA58FA4F00832091F2032F
:102320003091F3032F5F3F4F3093F3032093F20379
:102330000196B2010E9472749093F5038093F403A6
:1023400010927D0510927F0510927E053BC04B33A5
:1023500011F400937D0580917D05811133C080913A
:10236000F4039091F503189FF001199FF00D1124CB
:10237000E20FF31FEA50FC4F40832F5F3F4F309333
:102380007F0520937E051EC010E601E094E0492EF3
:10239000512CE0EEF2E034913F8F2AE0722E38EEBD
:1023A000C32E33E0D32EE12CF12C4CE3842E912C60
:1023B000A12CB12C22242394312C2C0E3D1EE7ECB1
:1023C000F0E064904091E8035091E9036091EA03E2
:1023D0007091EB038091E0039091E103A091E203FF
:1023E000B091E303481759076A077B07A8F5809166
:1023F000F2039091F3030497A4F02EC08091190387
:102400008111D3CE29C08DEC95E00E946D2E809372
:102410007C0520917E0530917F058A3009F0BACC89
:10242000C5CC8091CD039091CE03A091CF03B09104
:10243000D0038093E8039093E903A093EA03B09359
:10244000EB0385EC93E00E94D132482F80937C050A
:102450008A3009F0B2CEC3CE6F960FB6F894DEBFC5
:102460000FBECDBFDF91CF911F910F91FF90EF90E5
:10247000DF90CF90BF90AF909F908F907F906F90A4
:102480005F904F903F902F9008958F929F92AF92C0
:10249000BF92CF92DF92EF92FF920F931F93CF9351
:1024A000DF93A8E2AA2EA2E0BA2E01E013E0CAE967
:1024B000D5E0B4E18B2EB3E09B2EF50181915F0155
:1024C0000E94220E882319F10E940E0E6B017C01DE
:1024D000F4018081811103C06091AA0501C061E00F
:1024E00070E080E090E00E945671F8012081318117
:1024F000428153810E9489739B01AC01C701B601DF
:102500000E94DB6F688379838A839B8309C0F8010B
:1025100080819181A281B38188839983AA83BB83BF
:102520000C5F1F4F2496FFEF8F1A9F0A8CE2A816AC
:1025300082E0B80611F686E40E94220E8823D9F0C4
:102540000E940E0E6B017C016093B4057093B5057B
:102550008093B6059093B70520E030E0A9010E9472
:10256000B772181644F4C0921401D0921501E0928B
:102570001601F0921701DF91CF911F910F91FF90FB
:10258000EF90DF90CF90BF90AF909F908F90089585
:102590000E94451289E40E94220E882359F00E946D
:1025A0000E0E6093B8057093B9058093BA059093A9
:1025B000BB0508C01092B8051092B9051092BA0573
:1025C0001092BB058AE40E94220E882359F00E94D3
:1025D0000E0E6093BC057093BD058093BE0590936D
:1025E000BF0508951092BC051092BD051092BE055E
:1025F0001092BF050895CF92DF92EF92FF920F9352
:102600001F93C090E902D090EA02E090EB02F090B4
:10261000EC02A701960160919A0570919B0580914B
:102620009C0590919D050E94B47087FF08C0C092E0
:102630009A05D0929B05E0929C05F0929D05C09072
:10264000ED02D090EE02E090EF02F090F002A701D0
:10265000960160919E0570919F058091A0059091D3
:10266000A1050E94B47087FF08C0C0929E05D09259
:102670009F05E092A005F092A105C090F102D090D4
:10268000F202E090F302F090F402A701960160914B
:10269000A2057091A3058091A4059091A5050E94C3
:1026A000B47087FF08C0C092A205D092A305E09243
:1026B000A405F092A50520E030E04BE153E46091E1
:1026C0009A0570919B0580919C0590919D050E94B3
:1026D000B772181664F480E090E0ABE1B3E4809345
:1026E0009A0590939B05A0939C05B0939D0520E0CF
:1026F00030E046E153E460919E0570919F05809122
:10270000A0059091A1050E94B772181664F480E0AC
:1027100090E0A6E1B3E480939E0590939F05A0937B
:10272000A005B093A10520E030E044EB52E46091B5
:10273000A2057091A3058091A4059091A5050E9422
:10274000B772181664F480E090E0A4EBB2E48093D2
:10275000A2059093A305A093A405B093A5050E949C
:10276000882C6093920570939305809394059093C1
:1027700095056091020170910301882777FD80958E
:10278000982F0E94567120911401309115014091AB
:102790001601509117010E94897320E030E040E754
:1027A00052E40E94BB7020E030E048EC52E40E940A
:1027B000BB7018EEC12E12E0D12E7B018C0126EAEF
:1027C00035E042EA55E06EE975E08AE995E00E945D
:1027D0006D4780919A0590919B05A0919C05B091C1
:1027E0009D058093010390930203A0930303B0938C
:1027F000040380919E0590919F05A091A005B09142
:10280000A1058093050390930603A0930703B0935B
:1028100008038091A2059091A305A091A405B09111
:10282000A5058093090390930A03A0930B03B0932B
:102830000C038091A6059091A705A091A805B091E1
:10284000A90580930D0390930E03A0930F03B093FB
:1028500010031F910F91FF90EF90DF90CF9008959C
:10286000AF92BF92CF92DF92EF92FF920F931F939E
:10287000CF93DF93182F2091BC053091BD05409177
:10288000BE055091BF056091B8057091B905809162
:10289000BA059091BB050E94C472EB01082FF92E76
:1028A0006091020170910301882777FD8095982F30
:1028B0000E9456712091140130911501409116012A
:1028C000509117010E94897320E030E040E752E404
:1028D0000E94BB7020E030E048EC52E40E94BB70E4
:1028E0002091E8022F931F93FF920F93DF93CF93D2
:1028F0005B016C0102E0E02E01E020E048EB55E0D6
:102900006AE975E081E093E00E94B13D80919A050B
:1029100090919B05A0919C05B0919D05809301032A
:1029200090930203A0930303B093040380919E0548
:1029300090919F05A091A005B091A10580930503FA
:1029400090930603A0930703B09308038091A20518
:102950009091A305A091A405B091A50580930903CA
:1029600090930A03A0930B03B0930C038091A605E8
:102970009091A705A091A805B091A90580930D039A
:1029800090930E03A0930F03B09310030E94882C22
:1029900060939205709393058093940590939505A9
:1029A0000F900F900F900F900F900F90DF91CF919D
:1029B0001F910F91FF90EF90DF90CF90BF90AF905D
:1029C0000895F8940E94115F5E9A5E9A159A5E9A35
:1029D000ECEBF1E007C09091C00095FFFCCF809335
:1029E000C600319684918111F6CFE4EEF5E007C080
:1029F0009091C00095FFFCCF8093C60031968491E2
:102A00008111F6CF8091C00085FFFCCF8AE08093D2
:102A1000C600FFCFCF92DF92EF92FF920F931F93EA
:102A20000E94882C0091AC051091AD052091AE0557
:102A30003091AF05C0909205D0909305E090940539
:102A4000F09095056C197D098E099F0906171707E7
:102A50002807390730F4012B022B032B11F00E94B9
:102A6000E1148091190190911A01A0911B01B0917C
:102A70001C01892B8A2B8B2B09F10E94882C009139
:102A80009205109193052091940530919505601B56
:102A9000710B820B930B0091190110911A01209177
:102AA0001B0130911C01061717072807390730F45E
:102AB0009091610880916008981741F01F910F91E3
:102AC000FF90EF90DF90CF900C9449475E9A5E9A0A
:102AD000159A5E9AF3CF0E94115F8091E6028111F0
:102AE00034C081E08093E60280918605909187054D
:102AF000A0918805B09189058093B0059093B105A8
:102B0000A093B205B093B305ECEBF1E007C0909150
:102B1000C00095FFFCCF8093C6003196849181114F
:102B2000F6CFE5E0F6E007C09091C00095FFFCCF3E
:102B30008093C600319684918111F6CF8091C000B8
:102B400085FFFCCF8AE08093C60008958091E6025D
:102B50000895EF92FF920F931F93CF93DF938C0111
:102B60007B0184E0E80EF11CEB016991F8018081A2
:102B700091819C012F5F3F4F318320830E94F37925
:102B8000CE15DF0591F784E090E0DF91CF911F91A2
:102B90000F91FF90EF900895EF92FF920F931F9384
:102BA000CF93DF938C017B0180E1E80EF11CEB01F8
:102BB0006991F801808191819C012F5F3F4F3183A2
:102BC00020830E94F379CE15DF0591F780E190E034
:102BD000DF91CF911F910F91FF90EF900895EF92A9
:102BE000FF920F931F93CF93DF938C017B0184E0BF
:102BF000E80EF11CEB016991F801808191819C0143
:102C00002F5F3F4F318320830E94F379CE15DF057C
:102C100091F784E090E0DF91CF911F910F91FF90A9
:102C2000EF9008950F931F93CF93DF93CDB7DEB747
:102C30002A970FB6F894DEBF0FBECDBF80E390E3B6
:102C4000A0E3B0E08D839E83AF83B88784E690E0F5
:102C50009A878987BE016B5F7F4FCE0109960E94DC
:102C6000A9156FE77DE0CE0109960E94CC156FE8AB
:102C70007DE0CE0109960E94CC150FE61DE0F8011B
:102C800061918F0189859A859C012F5F3F4F3A871B
:102C900029870E94F379FDE00F371F0781F767E668
:102CA0007DE0CE0109960E94EF1563E67DE0CE013E
:102CB00009960E94EF156BE67DE0CE0109960E9411
:102CC000EF1563E57DE0CE0109960E94EF150FE94F
:102CD0001DE0F80161918F0189859A859C012F5F24
:102CE0003F4F3A8729870E94F379FDE0033A1F0797
:102CF00081F76FE57DE0CE0109960E94EF156BE547
:102D00007DE0CE0109960E94EF1567E57DE0CE01DA
:102D100009960E94EF1505EF12E0F80161918F010D
:102D200089859A859C012F5F3F4F3A8729870E94AA
:102D3000F379F3E001301F0781F76AE371E0CE0118
:102D400009960E94EF1566E371E0CE0109960E9494
:102D5000EF1562E371E0CE0109960E94EF1586E55A
:102D600090E3A6E3B0E089839A83AB83BC8384E6D7
:102D700090E09A878987BE016F5F7F4FCE010996E9
:102D80000E94A915E7ECF0E007C09091C00095FF04
:102D9000FCCF8093C600319684918111F6CFEBE190
:102DA000F4E007C09091C00095FFFCCF8093C6006F
:102DB000319684918111F6CF8091C00085FFFCCFC0
:102DC0008AE08093C6002A960FB6F894DEBF0FBE45
:102DD000CDBFDF91CF911F910F910895EF92FF9298
:102DE0000F931F93CF93DF938C017B0180E1E80E5B
:102DF000F11CEB01F801808191819C012F5F3F4F15
:102E0000318320830E94EB798993CE15DF0591F7FA
:102E100080E190E0DF91CF911F910F91FF90EF90B3
:102E20000895EF92FF920F931F93CF93DF938C013E
:102E30007B0184E0E80EF11CEB01F80180819181B7
:102E40009C012F5F3F4F318320830E94EB79899350
:102E5000CE15DF0591F784E090E0DF91CF911F91CF
:102E60000F91FF90EF900895AF92BF92CF92DF92B3
:102E7000EF92FF920F931F93CF93DF93CDB7DEB7FF
:102E8000EC970FB6F894DEBF0FBECDBFD82E24E668
:102E900030E03AAF29AF46E550E366E370E049AB76
:102EA0005AAB6BAB7CAB8E010B5C1F4FB8017E0144
:102EB00089E3E80EF11C89AD9AAD9C012F5F3F4F6D
:102EC0003AAF29AF6BAF7CAF0E94EB79F8018193E9
:102ED0008F016BAD7CADEE15FF0569F7D110A4C075
:102EE00043E050E0CE01C1960E94B377009709F00D
:102EF0009BC06FE77DE0C8010E94EE166FE87DE0A1
:102F0000C8010E94EE160FE61DE089AD9AAD9C0146
:102F10002F5F3F4F3AAF29AF0E94EB79F8018193C1
:102F20008F01FDE00F371F0781F767E67DE0CE01D7
:102F3000C9960E94111763E67DE0CE01C9960E94F2
:102F400011176BE67DE0CE01C9960E94111763E56B
:102F50007DE0CE01C9960E9411170FE91DE089ADF1
:102F60009AAD9C012F5F3F4F3AAF29AF0E94EB799A
:102F7000F80181938F01FDE0033A1F0781F76FE5A8
:102F80007DE0CE01C9960E9411176BE57DE0CE0170
:102F9000C9960E94111767E57DE0CE01C9960E948F
:102FA000111705EF12E089AD9AAD9C012F5F3F4FDD
:102FB0003AAF29AF0E94EB79F80181938F01F3E0DA
:102FC00001301F0781F76AE371E0CE01C9960E94C4
:102FD000111766E371E0CE01C9960E94111762E3F2
:102FE00071E0CE01C9960E941117E7ECF0E007C02E
:102FF0009091C00095FFFCCF8093C60031968491DC
:103000008111F6CFECE8F1E007C09091C00095FF88
:10301000FCCF8093C600319684918111F6CF8091C8
:10302000C00085FFFCCFDDC080E1E3E4F1E0DE011C
:10303000919601900D928A95E1F780E1E3E5F1E048
:10304000DE01519601900D928A95E1F780E1E3E669
:10305000F1E0DE01119601900D928A95E1F76E0183
:1030600081E2C80ED11C8FE7E82E8DE0F82E8E018C
:103070000F5E1F4F6FE87DE0AE014F5F5F4F9FE631
:10308000A92E9DE0B92E24E030E0F60181919191C6
:10309000A191B1916F01F70181939193A193B193A4
:1030A0007F01F80181919191A191B1918F01FB0173
:1030B00081939193A193B193BF01FA018191919171
:1030C000A191B191AF01F50181939193A193B19336
:1030D0005F0121503109C9F680E090E0AAE7B4E42D
:1030E0008093670D9093680DA093690DB0936A0D5E
:1030F0008093630D9093640DA093650DB093660D5E
:1031000010926B0D10926C0D10926D0D10926E0D51
:1031100080E29EE4A0E0B0E080939F0D9093A00D2C
:10312000A093A10DB093A20D1092530D1092540DC7
:103130001092550D1092560D80E090E0A0E7B1E49A
:1031400080935F0D9093600DA093610DB093620D1D
:103150004DEC5CEC6CEC7EE340935B0D50935C0DAE
:1031600060935D0D70935E0D8093570D9093580D95
:10317000A093590DB0935A0D1092FD021092FE02C9
:103180001092FF02109200031092F9021092FA02BC
:103190001092FB021092FC021092F5021092F602BD
:1031A0001092F7021092F802E7ECF0E007C090915D
:1031B000C00095FFFCCF8093C600319684918111A9
:1031C000F6CFE7E8F1E006C09091C00095FFFCCF94
:1031D0008093C60081918111F7CF8091C00085FF57
:1031E000FCCF8AE08093C600EC960FB6F894DEBF61
:1031F0000FBECDBFDF91CF911F910F91FF90EF9048
:10320000DF90CF90BF90AF9008952F923F924F9252
:103210005F926F927F928F929F92AF92BF92CF9266
:10322000DF92EF92FF920F931F93CF93DF93CDB76F
:10323000DEB7A6970FB6F894DEBF0FBECDBF87E40A
:103240000E94220E882309F40EC20E940E0E0E94D4
:10325000237164307105D9F144F46230710521F1B4
:103260005CF577FF17C00C94BC266A35710509F42C
:10327000A6C134F46C31710511F00C94BC266AC0FF
:103280006B35710509F49FC16C35710511F00C9413
:10329000BC269EC18091E602811106C00E944512A3
:1032A0000E94FB120C94D2298091E602811104C085
:1032B0000E94C81281E007C08091E602811107C018
:1032C0000E94C81280E00E9430140C94D22980E53C
:1032D0000E94220E882339F00E940E0E0E9428714F
:1032E0006B017C0103C0C12CD12C760183E50E94C7
:1032F000220E882361F00E940E0E20E030E04AE7A3
:1033000054E40E9489730E9428716B017C010E9421
:10331000DE590E94882C4B015C018C0C9D1CAE1C5C
:10332000BF1C0E94882C6093920570939305809334
:1033300094059093950505C00E942F5C81E00E9442
:103340000A150E94882C681579058A059B05A0F34B
:103350000C94BC268091140190911501A091160146
:10336000B09117018093960590939705A0939805C7
:10337000B0939905809102019091030190931303FA
:103380008093120384E690E09093030180930201FE
:103390000E94882C60939205709393058093940506
:1033A0009093950581E00E9478538091010390915C
:1033B0000203A0910303B091040380939A059093B4
:1033C0009B05A0939C05B0939D058091050390916A
:1033D0000603A0910703B091080380939E05909384
:1033E0009F05A093A005B093A1058091090390913A
:1033F0000A03A0910B03B0910C038093A205909354
:10340000A305A093A405B093A50580910D03909109
:103410000E03A0910F03B09110038093A605909323
:10342000A705A093A805B093A905109214011092C6
:103430001501109216011092170188E50E94220EC4
:10344000882311F090E00AC089E50E94220E8111C4
:10345000F9CF8AE50E94220E91E0982790931801F7
:1034600091110C94BF2688E50E94220E81110C94C4
:10347000BF268091180181110C949B2789E50E9439
:10348000220E81110C949B278091180181110C94BC
:1034900077288AE50E94220E81110C94772888E50E
:1034A0000E94220E8823D1F00E94170E672B682BF2
:1034B000692BA1F00E940E0E2091F5023091F602C8
:1034C0004091F7025091F8020E94DB6F6093010374
:1034D00070930203809303039093040389E50E9491
:1034E000220E8823D1F00E94170E672B682B692BC0
:1034F000A1F00E940E0E2091F9023091FA02409143
:10350000FB025091FC020E94DB6F609305037093F5
:10351000060380930703909308038AE50E94220E16
:103520008823D1F00E94170E672B682B692BA1F01E
:103530000E940E0E2091FD023091FE024091FF028A
:10354000509100030E94DB6F6093090370930A039C
:1035500080930B0390930C032DE033E049E053E09C
:1035600065E073E081E093E00E94FC5180E00E94FE
:1035700078538091960590919705A0919805B09108
:1035800099058093140190931501A0931601B093AF
:10359000170180911203909113039093030180937C
:1035A00002010E94882C609392057093930580938A
:1035B0009405909395050E9471530C94BC2610922B
:1035C000AA050C94BC2681E08093AA050C94BC2625
:1035D00085E40E94220E811102C00E94DE5958E249
:1035E000C52E52E0D52E65EFE62E62E0F62E01E004
:1035F00013E0B12CF60181916F010E94220E882305
:1036000039F1F3E0BF120CC00E940E0EF801608386
:103610007183828393838DE093E00E94985218C057
:103620000E940E0EF70120813181428153810E9458
:10363000DB6FF80160837183828393832DE033E035
:1036400049E053E065E073E081E093E00E94FC51C3
:10365000B394F4E0EF0EF11C0C5F1F4F24E0B212A4
:10366000C9CF0C94BC268DE40E94220E882311F44D
:103670000C940F260E940E0E0E9423716237710572
:1036800009F469C70CF06FC06C31710509F46DC1A4
:103690009CF56631710509F425C1ACF46231710500
:1036A00009F468C634F46131710511F00C94BC263C
:1036B000E2C06431710509F4E4C06531710511F0AF
:1036C0000C94BC2609C16931710509F434C154F464
:1036D0006731710509F40CC16831710511F00C9462
:1036E000BC2619C16A31710509F42BC16B31710512
:1036F00011F00C94BC2633C16435710509F43AC647
:10370000CCF46A32710509F43BC254F46E31710590
:1037100009F460C16F31710511F00C94BC2698C199
:103720006235710509F41FC66335710511F00C94FB
:10373000BC261CC66836710509F45FC254F46535B1
:10374000710509F452C66C35710511F00C94BC2654
:1037500062C66936710509F4C6C26D36710511F08D
:103760000C94BC2692C36E3C710511F40C94C024D9
:10377000D4F56C38710509F4A2C2C4F46737710539
:1037800011F40C948D2334F46337710511F00C940B
:10379000BC26D3C66837710511F40C9487236937AA
:1037A000710511F00C94BC260C9489236B3C7105B7
:1037B00011F40C9426245CF46E3B710509F437C5B2
:1037C000693C710511F00C94BC260C94EC236C3C04
:1037D000710511F40C9442246D3C710511F00C94A8
:1037E000BC260C946224603931E0730711F40C9408
:1037F000EB2504F56D3291E0790711F40C94FD246A
:1038000064F46C3D710511F40C94DC246D3D71057C
:1038100011F00C94BC260C94EE246E32F1E07F077C
:1038200011F40C94D8256F32714011F00C94BC2621
:103830000C94DC25663F31E0730711F40C94F325FA
:103840006CF4643F91E0790711F40C94EE25653F28
:10385000714011F00C94BC260C94F125673FF1E007
:103860007F0711F40C94F725673E734011F00C9418
:10387000BC260C94FA255E985E9815985E980C9478
:10388000BC26E3EFF2E007C09091C00095FFFCCFAB
:103890008093C600319684918111F6CF8091C0004B
:1038A00085FFFCCF8AE08093C60088E193E00E9408
:1038B000F866E3E0F3E007C09091C00095FFFCCF0D
:1038C0008093C600319684918111F6CF8091C0001B
:1038D00085FFFCCF0C94B92688E193E00E943A67FB
:1038E0000C94BC2688E193E00E9400680C94BC26EE
:1038F00000918005109181050C5F1F4F6AE270E016
:10390000C8010E94A177009719F0FC01319710823D
:1039100041E0B80159C088E193E00E9404680E9428
:10392000882C60938E0570938F05809390059093FB
:1039300091050C94BC2688E193E00E940B680C94DE
:10394000BC2680911A03882311F40C94BC2683E5CD
:103950000E94220E81110C9453290C94BC2688E1FC
:1039600093E00E943B6B0C94BC2680918005909163
:1039700081056AE270E004960E94A1778C010097AD
:10398000E1F020917A0530917B0540E6429FC0012D
:10399000439F900D11246EE470E08A509C4F0E946A
:1039A000A17760E270E00E94A17701969093810573
:1039B00080938005F80131971082609180057091A5
:1039C00081056C5F7F4F40E088E193E00E941068C2
:1039D0000C94BC2680911A03882311F40C94BC2605
:1039E00088E193E00E94F26C8091800590918105BE
:1039F0006AE270E004960E94A1778C010097E1F0E2
:103A000020917A0530917B0540E6429FC001439F9B
:103A1000900D11246EE470E08A509C4F0E94A177B3
:103A200060E270E00E94A1770196909381058093F7
:103A30008005F801319710826091800570918105B1
:103A40006C5F7F4F88E193E00E94FF690C94BC2675
:103A50000E94882C60938A0570938B0580938C0557
:103A600090938D0500918E0510918F052091900502
:103A700030919105601B710B820B930B28EE33E0A4
:103A800040E050E00E948674CA01B9012CE330E0A6
:103A900040E050E00E9486747F936F933F932F9392
:103AA00088E791E09F938F93CE0101969F938F9328
:103AB0000E94EA77E7ECF0E084910FB6F894DEBF5D
:103AC0000FBECDBFE7ECF0E008C09091C00095FFBD
:103AD000FCCF8093C600319684918111F6CFFE0110
:103AE000319606C09091C00095FFFCCF8093C60030
:103AF00081918111F7CF8091C00085FFFCCF8AE0D2
:103B00008093C6008091320D882311F40C94BC265A
:103B10001092320D6091E802E62FF0E0EE0FFF1FE9
:103B2000E45FF14F808191810E94635B20912101CC
:103B30003091220140912301509124010E94B772DB
:103B4000181614F00C94BC266091E802062F10E0C1
:103B500080E090E00E94935AF801EE0FFF1FE45FAF
:103B6000F14F91838083F801EE0FFF1FEE0FFF1FCF
:103B7000EE5FF14F10821182128213820C94BC26E8
:103B800083E50E94220E882311F40C94BC260E9427
:103B90000E0E0E9423717B0180E50E94220E882375
:103BA00011F40C94BC26F7FE02C00C94BC26FFEF67
:103BB000EF16F10409F014F40C9464290C94BC265B
:103BC000819191918017910711F40C94BC2622E009
:103BD000E03AF207A9F717FF02C00C94BC2661E097
:103BE000802F0E94B02D6E2D802F0E94CC2DB7010A
:103BF000802F0E94252D0C94BC268091E802809392
:103C0000AB0584E50E94220E882379F10E940E0EF6
:103C10000E9428716093AB05662339F1E7ECF0E070
:103C200007C09091C00095FFFCCF8093C6003196ED
:103C300084918111F6CFE5EAF1E006C09091C000D1
:103C400095FFFCCF8093C60081918111F7CF40E0B2
:103C500050E06091AB058DEC95E00E94332F809190
:103C6000C00085FFFCCF0C94B92683E50E94220E8C
:103C7000882309F1B090AB050E940E0E6B017C0108
:103C80000B2D10E00E942371DC01CB016B2D0E94F3
:103C9000935AF801EE0FFF1FE45FF14F9183808389
:103CA000F801EE0FFF1FEE0FFF1FEE5FF14FC08216
:103CB000D182E282F3820E94105F0C94BC2683E5DD
:103CC0000E94220E882311F40C94BC260E940E0E32
:103CD0000E942371CB010E94175B90930B0E80937F
:103CE0000A0E0C94BC268091E8028093AB0584E513
:103CF0000E94220E882379F10E940E0E0E942871E4
:103D00006093AB05662339F1E7ECF0E007C09091D2
:103D1000C00095FFFCCF8093C6003196849181113D
:103D2000F6CFECEBF1E006C09091C00095FFFCCF20
:103D30008093C60081918111F7CF40E050E06091FF
:103D4000AB058DEC95E00E94332F8091C00085FF7C
:103D5000FCCF0C94B926E1E1F3E007C09091C000DC
:103D600095FFFCCF8093C600319684918111F6CFE8
:103D70006091AB05E62FF0E0EE0FFF1FE85FF14F1B
:103D8000808191810E94635BAB01BC0121E030E046
:103D90008DEC95E00E944430E7E1F3E007C090919C
:103DA000C00095FFFCCF8093C600319684918111AD
:103DB000F6CF6091AB05E62FF0E0EE0FFF1FE45F5A
:103DC000F14F808191810E94635BAB01BC0121E0D6
:103DD00030E08DEC95E00E944430EAE1F3E007C06A
:103DE0009091C00095FFFCCF8093C60031968491DE
:103DF0008111F6CF8091060E9091070E0E941D5EF4
:103E0000AB01BC0121E030E08DEC95E00E94443034
:103E1000EEE1F3E007C09091C00095FFFCCF8093E6
:103E2000C600319684918111F6CF80910A0E90914F
:103E30000B0E0E941D5EAB01BC0121E030E08DEC59
:103E400095E00E944430E1E2F3E007C09091C000A9
:103E500095FFFCCF8093C600319684918111F6CFF7
:103E60008091AB0590E00E948D5A4AE050E0BC0181
:103E70008DEC95E00E944B2F8091C00085FFFCCF18
:103E80008AE08093C6000C94D2298091E802809346
:103E9000AB0584E50E94220E882371F10E940E0E6C
:103EA0000E9428716093AB05662331F1E7ECF0E0E6
:103EB00007C09091C00095FFFCCF8093C60031965B
:103EC00084918111F6CFE3EDF1E006C09091C0003E
:103ED00095FFFCCF8093C60081918111F7CF40E020
:103EE00050E06091AB058DEC95E00E94332F8091FE
:103EF000C00085FFFCCF3DC71092320D83E50E94C4
:103F0000220E882309F1B090AB050E940E0E6B01C2
:103F10007C010B2D10E00E942371DC01CB016B2D85
:103F20000E94935AF801EE0FFF1FE45FF14F918357
:103F30008083F801EE0FFF1FEE0FFF1FEE5FF14FC2
:103F4000C082D182E282F38283E50E94220E88231E
:103F500051F00E940E0E6093210170932201809314
:103F600023019093240182E40E94220E882351F0C1
:103F70000E940E0E60932501709326018093270105
:103F80009093280186E40E94220E882369F00E9403
:103F90000E0E60931D0170931E0180931F0190937C
:103FA000200181E08093320D0E94105F0E94882CD6
:103FB0004B015C018091AB0590E0880F991FFC01DB
:103FC000E45FF14F2081318138A32F8FFC01E85F3E
:103FD000F14F808191819EA38DA3CC24CA94DC2CC7
:103FE0007601E5E2F3E02490E8E2F3E03490ECE2DD
:103FF000F3E0049148EE442E43E0542E612C712CE2
:104000001AE00C948829822DE5E2F3E008C0909133
:10401000C00095FFFCCF8093C6003196849181113A
:10402000F6CF6091AB05E62FF0E0EE0FFF1FE85FE3
:10403000F14F808191810E94635BAB01BC0121E063
:1040400030E08DEC95E00E944430832DE8E2F3E00F
:1040500008C09091C00095FFFCCF8093C6003196B8
:1040600084918111F6CF6091AB054AE050E070E099
:104070008DEC95E00E944B2F802FECE2F3E008C01E
:104080009091C00095FFFCCF8093C600319684913B
:104090008111F6CFF7FE03C0EAEEF1E027C00E94DF
:1040A000882C4B015C01C701B601605F784D8F4FD2
:1040B0009F4F681979098A099B09A30192010E94FF
:1040C000867449015A012AE030E0B501A4018DEC63
:1040D00095E00E94272F8091C00085FFFCCF0DC086
:1040E0009091C00095FFFCCF8093C6008191811113
:1040F000F7CF8091C00085FFFCCF1093C6000E94CF
:10410000882C4B015C010E942F5C81E00E940A1503
:104110009FEFC916D906E906F906C1F56091AB050E
:10412000EF8DF8A12DA13EA12E173F0714F00C949E
:10413000A529E62FF0E0EE0FFF1FE85FF14F808129
:1041400091810E94635B69A37AA38BA39CA3609176
:10415000AB05E62FF0E0EE0FFF1FE45FF14F80812B
:1041600091810E94635B20E030E040E85FE30E94C1
:10417000DA6F9B01AC0169A17AA18BA19CA10E947D
:10418000B77287FD02C00C946D293AC0F7FC38C0A5
:104190006091AB05E62FF0E0EE0FFF1FE85FF14FF7
:1041A000808191810E94635B69A37AA38BA39CA306
:1041B0006091AB05E62FF0E0EE0FFF1FE45FF14FDB
:1041C000808191810E94635B9B01AC0169A17AA10E
:1041D0008BA19CA10E94DA6F0E942371AB01BC01EC
:1041E00077FF07C070956095509541955F4F6F4F71
:1041F0007F4F443051056105710514F00C946D2911
:104200003FEFC316D306E306F30611F40C94882996
:10421000F7FE02C00C9473290E94882C6C197D094A
:104220006031774210F40C9488290C94732983E54B
:104230000E94220E882359F00E940E0E0E942371C4
:10424000CB010E94175B90930B0E80930A0E0E9485
:10425000882C6B017C01E0E3F3E0A490E3E3F3E05E
:10426000B490E7E3F3E014910AE070C00E94882C58
:104270006C197D098E099F09693E7340810591057E
:1042800008F45FC06091E802A62FB0E0AA0FBB1F40
:10429000A85FB14F8D919C910E94635BAB01BC0103
:1042A0008A2DE0E3F3E008C09091C00095FFFCCFB9
:1042B0008093C600319684918111F6CF22E030E0E0
:1042C0008DEC95E00E9444308B2DE3E3F3E008C0D1
:1042D0009091C00095FFFCCF8093C60031968491E9
:1042E0008111F6CF6091E8024AE050E070E08DEC79
:1042F00095E00E944B2F812FE7E3F3E008C09091F7
:10430000C00095FFFCCF8093C60031968491811147
:10431000F6CF8091060E9091070E0E941D5EAB01B4
:10432000BC0121E030E08DEC95E00E9444308091AA
:10433000C00085FFFCCF0093C6000E94882C6B0153
:104340007C010E942F5C81E00E940A1520910A0ED8
:1043500030910B0E8091060E9091070E82179307F5
:104360000CF484CFCAC71092170306C581E080936E
:10437000170302C583E50E94220E882399F00E944C
:104380000E0E20E030E04AE754E40E9489730E9458
:1043900028716093190170931A0180931B01909307
:1043A0001C01EAC488E50E94220E8111C6C789E576
:1043B0000E94220E8111C1C78AE50E94220E81113E
:1043C000BCC785E40E94220E8111B7C7B0C75E9AB0
:1043D00089E50E94220E81115E9A8AE50E94220ED2
:1043E000882309F4C9C4159AC7C483E50E94220E24
:1043F0000E940E0E20E030E04AE754E40E948973E8
:104400000E9428716093AC057093AD058093AE0552
:104410009093AF05B1C428E232E03EA32DA34FE74D
:10442000242E4DE0342E8FE89DE098A38F8F53E427
:10443000852E5DE0952E10E0EDA1FEA18191FEA3F9
:10444000EDA30E94220E882309F466C0133009F000
:104450005CC00E940E0E6B017C0120E030E040EA5F
:1044600051E40E94B47087FF4AC0A7019601F10190
:1044700060817181828193810E94BB70762EA72E0C
:10448000B82E092F762F272F3A2D4B2D502F6091C4
:10449000570D7091580D8091590D90915A0D0E94B1
:1044A00089736093570D7093580D8093590D9093B5
:1044B0005A0D272D3A2D4B2D502FEF8DF8A16081ED
:1044C0007181828193810E948973EF8DF8A160834D
:1044D000718382839383F4016081718182819381EE
:1044E0000E945471272D3A2D4B2D502F0E94897315
:1044F0000E942871F4016083718382839383F101A8
:10450000C082D182E282F38207C00E940E0EF101C6
:1045100060837183828393831F5FF4E02F0E311CCD
:104520002F8D38A12C5F3F4F38A32F8F34E0830E9F
:10453000911C143009F080CF1FC4EBE3F3E007C0F7
:104540009091C00095FFFCCF8093C6003196849176
:104550008111F6CF11C4E6EDF3E007C09091C000E1
:1045600095FFFCCF8093C600319684918111F6CFE0
:104570004091010350910203609103037091040381
:1045800022E030E08DEC95E00E944430E9EDF3E06C
:1045900007C09091C00095FFFCCF8093C600319674
:1045A00084918111F6CF40910503509106036091EB
:1045B00007037091080322E030E08DEC95E00E9443
:1045C0004430ECEDF3E007C09091C00095FFFCCFC4
:1045D0008093C600319684918111F6CF40910903F2
:1045E00050910A0360910B0370910C0322E030E0BC
:1045F0008DEC95E00E944430EFEDF3E007C0909120
:10460000C00095FFFCCF8093C60031968491811144
:10461000F6CF40910D0350910E0360910F037091FE
:10462000100322E030E08DEC95E00E944430E2EE91
:10463000F3E007C09091C00095FFFCCF8093C600C7
:10464000319684918111F6CF0E94385A0E9456719A
:1046500020917F0D3091800D4091810D5091820D00
:104660000E94BB70AB01BC0122E030E08DEC95E014
:104670000E944430ECEEF3E007C09091C00095FF3B
:10468000FCCF8093C600319684918111F6CF81E0F2
:104690000E94385A0E9456712091830D3091840DEA
:1046A0004091850D5091860D0E94BB70AB01BC01FD
:1046B00022E030E08DEC95E00E944430EFEEF3E034
:1046C00007C09091C00095FFFCCF8093C600319643
:1046D00084918111F6CF82E00E94385A0E9456716F
:1046E0002091870D3091880D4091890D50918A0D50
:1046F0000E94BB70AB01BC0122E030E08DEC95E084
:104700000E9444308091C00085FFFCCF32C380E01E
:1047100001C081E00E9478532FC3E2EFF3E007C0AD
:104720009091C00095FFFCCF8093C6003196849194
:104730008111F6CF329B03C0EFE9F1E009C0E2EA54
:10474000F1E006C09091C00095FFFCCF8093C600B9
:1047500081918111F7CFE9EFF3E007C09091C0009C
:1047600095FFFCCF8093C600319684918111F6CFDE
:10477000339B03C0EFE9F1E009C0E2EAF1E006C0D3
:104780009091C00095FFFCCF8093C600819181116C
:10479000F7CFE0E0F4E007C09091C00095FFFCCFB8
:1047A0008093C600319684918111F6CF349B03C06B
:1047B000EFE9F1E009C0E2EAF1E006C09091C00043
:1047C00095FFFCCF8093C60081918111F7CF809136
:1047D000C00085FFFCCFCDC238E2E32E32E0F32EDD
:1047E00000E010E0F70181917F010E94220E8823F2
:1047F00039F10E940E0EBFE6CB2EBDE0DB2EC00EBF
:10480000D11E0E942871F601608371838283938395
:104810000E940E0E23E4C22E2DE0D22EC00ED11E19
:10482000F801E158F24F20813181428153810E9489
:1048300089730E942871F601608371838283938358
:104840000C5F1F4F0031110569F696C208E212E0B5
:10485000AFE8EA2EADE0FA2EF80181918F010E94B7
:10486000220E882339F00E940E0EF70160837183B7
:1048700082839383F4E0EF0EF11C22E00C321207E6
:1048800059F77AC283E50E94220E882351F00E94D4
:104890000E0E6093670D7093680D8093690D909371
:1048A0006A0D84E50E94220E882309F465C20E94E5
:1048B0000E0E6093630D7093640D8093650D90935D
:1048C000660D5AC283E50E94220E882351F00E9491
:1048D0000E0E60936B0D70936C0D80936D0D909325
:1048E0006E0D84E50E94220E882351F00E940E0E68
:1048F0006093530D7093540D8093550D9093560D06
:1049000082E40E94220E882361F00E940E0E0E9413
:10491000287160939F0D7093A00D8093A10D9093CB
:10492000A20D88E50E94220E882351F00E940E0EEF
:1049300060935F0D7093600D8093610D9093620D95
:104940008AE50E94220E882351F00E940E0E609389
:104950005B0D70935C0D80935D0D90935E0D85E40F
:104960000E94220E882309F407C20E940E0E609353
:10497000570D7093580D8093590D90935A0DFCC1AB
:1049800008E212E0F5EFEF2EF2E0FF2EF801819140
:104990008F010E94220E882339F00E940E0EF7012B
:1049A0006083718382839383F4E0EF0EF11C22E035
:1049B0000B32120759F7E0C183E50E94220E8823CB
:1049C00009F4DAC10E940E0E0E9423717093030154
:1049D0006093020181E080931103CEC183E50E94C0
:1049E000220E882309F4C8C10E940E0E0E94237172
:1049F0007093010160930001BFC180E50E94220E07
:104A0000882351F00E940E0E60933A0170933B018F
:104A100080933C0190933D0189E40E94220E8823FB
:104A200081F00E940E0E2DEB37E346E05EE30E941C
:104A300089736093360170933701809338019093A6
:104A4000390184E40E94220E882381F00E940E0E18
:104A50002DEB37E346E05EE30E94BB7060933201CA
:104A600070933301809334019093350183E40E9465
:104A7000220E882351F00E940E0E60932E01709337
:104A80002F0180933001909331010E94765AECEE11
:104A9000F1E006C09091C00095FFFCCF8093C60066
:104AA00081918111F7CFEFEEF1E006C09091C00047
:104AB00095FFFCCF8093C60081918111F7CF409183
:104AC0003A0150913B0160913C0170913D0122E01F
:104AD00030E08DEC95E00E944430E3EFF1E006C059
:104AE0009091C00095FFFCCF8093C6008191811109
:104AF000F7CF2DEB37E346E05EE36091360170912E
:104B0000370180913801909139010E94BB70AB014F
:104B1000BC0122E030E08DEC95E00E944430E7EFEC
:104B2000F1E006C09091C00095FFFCCF8093C600D5
:104B300081918111F7CF2DEB37E346E05EE3609181
:104B400032017091330180913401909135010E94BE
:104B50008973AB01BC0122E030E08DEC95E00E944E
:104B60004430EBEFF1E006C09091C00095FFFCCF20
:104B70008093C60081918111F7CF2DEB37E346E09A
:104B80005EE360912E0170912F0180913001909130
:104B900031010E948973AB01BC0122E030E08DEC51
:104BA00095E00E9444308091C00085FFFCCFE1C0B9
:104BB00081E00E94B252E0C083E50E94220E882369
:104BC00019F00E940E0E04C060E070E086E193E4EC
:104BD0000E94335FD1C00E94DE59CEC00E941216DF
:104BE000CBC080E001C081E00E943417C5C00E94A4
:104BF0003B0AC2C01092E6028091B0059091B105C7
:104C0000A091B205B091B305809386059093870576
:104C1000A0938805B09389050E94650EADC084E518
:104C20000E94220E882309F463C00E940E0E0E9487
:104C300028716093AB05662391F1E7ECF0E007C0C3
:104C40009091C00095FFFCCF8093C600319684916F
:104C50008111F6CFEFEFF1E006C09091C00095FF13
:104C6000FCCF8093C60081918111F7CF40E050E0E6
:104C70006091AB058DEC95E00E94332FE1E0F2E00E
:104C800006C09091C00095FFFCCF8093C600819133
:104C90008111F7CF8091C00085FFFCCF6AC01092D0
:104CA000E802E7ECF0E007C09091C00095FFFCCF70
:104CB0008093C600319684918111F6CFE2E1F2E053
:104CC00006C09091C00095FFFCCF8093C6008191F3
:104CD0008111F7CF6091E8024AE050E070E08DEC7E
:104CE00095E00E944B2F8091C00085FFFCCF41C012
:104CF000E7ECF0E007C09091C00095FFFCCF8093F7
:104D0000C600319684918111F6CFE7E0F4E007C048
:104D10009091C00095FFFCCF8093C600319684919E
:104D20008111F6CF80917A0590917B0520E6289F2E
:104D3000F001299FF00D1124EA50FC4F06C090911C
:104D4000C00095FFFCCF8093C60081918111F7CF01
:104D5000E9E1F4E007C09091C00095FFFCCF80939B
:104D6000C600319684918111F6CF8091C00085FFF5
:104D7000FCCF8AE08093C6000E943D0E13C31092C0
:104D800001031092020310920303109204032DE01A
:104D900033E049E053E065E073E081E093E00E9496
:104DA000FC5180E090E8A8E6B3EC80939A059093DC
:104DB0009B05A0939C05B0939D05609104017091A3
:104DC0000501809106019091070160931401709391
:104DD0001501809316019093170120E030E040E721
:104DE00052E40E94BB70E8EECE2EE2E0DE2E7B01A4
:104DF0008C0126EA35E042EA55E06EE975E08AE981
:104E000095E00E946D470E94DE59109201031092B6
:104E1000020310920303109204032DE033E049E0F3
:104E200053E065E073E081E093E00E94FC5180E094
:104E300090E0A0EAB0E480939A0590939B05A0933C
:104E40009C05B0939D0520E030E040E752E460917E
:104E500014017091150180911601909117010E9423
:104E6000BB707B018C0126EA35E042EA55E06EE931
:104E700075E08AE995E00E946D470E94DE5980E066
:104E800090E0A0E2B1EC80939A0590939B05A093EB
:104E90009C05B0939D0520E030E040E05FE3609129
:104EA00004017091050180910601909107010E9413
:104EB0008973FB01462F5F2F682F792F40931401D0
:104EC00050931501609316017093170120E030E0B4
:104ED00040E752E4BF010E94BB707B018C0126EACF
:104EE00035E042EA55E06EE975E08AE995E00E9416
:104EF0006D470E94DE5980E090E00E94E7098091B2
:104F0000010390910203A0910303B09104038093E5
:104F10009A0590939B05A0939C05B0939D051092D4
:104F200014011092150110921601109217010E949F
:104F300071530C94391A10920503109206031092C3
:104F40000703109208032DE033E049E053E065E0E9
:104F500073E081E093E00E94FC5180E090E0A1E6E4
:104F6000B3EC80939E0590939F05A093A005B0930A
:104F7000A105609108017091090180910A01909149
:104F80000B016093140170931501809316019093A7
:104F9000170120E030E040E752E40E94BB7058EE79
:104FA000C52E52E0D52E7B018C0126EA35E042EA7F
:104FB00055E06EE975E08AE995E00E946D470E9430
:104FC000DE59109205031092060310920703109207
:104FD00008032DE033E049E053E065E073E081E051
:104FE00093E00E94FC5180E090E0A0EAB0E480935E
:104FF0009E0590939F05A093A005B093A10520E086
:1050000030E040E752E46091140170911501809105
:105010001601909117010E94BB707B018C0126EA5A
:1050200035E042EA55E06EE975E08AE995E00E94D4
:105030006D470E94DE5980E090E0A0E2B1EC8093E1
:105040009E0590939F05A093A005B093A10520E035
:1050500030E040E05FE360910801709109018091C8
:105060000A0190910B010E948973FB01462F5F2F6B
:10507000682F792F40931401509315016093160106
:105080007093170120E030E040E752E4BF010E9436
:10509000BB707B018C0126EA35E042EA55E06EE9FF
:1050A00075E08AE995E00E946D470E94DE5981E033
:1050B00090E00E94E7098091050390910603A0917A
:1050C0000703B091080380939E0590939F05A093DA
:1050D000A005B093A1051092140110921501109231
:1050E0001601109217010E9471530C94441A1092E9
:1050F000090310920A0310920B0310920C032DE087
:1051000033E049E053E065E073E081E093E00E9422
:10511000FC5180E090E0A7E0B3EC8093A20590936F
:10512000A305A093A405B093A50560910C0170910F
:105130000D0180910E0190910F0160931401709305
:105140001501809316019093170120E030E040E7AD
:1051500052E40E94BB7048EEC42E42E0D42E7B0184
:105160008C0126EA35E042EA55E06EE975E08AE90D
:1051700095E00E946D470E94DE591092090310923B
:105180000A0310920B0310920C032DE033E049E068
:1051900053E065E073E081E093E00E94FC5180E021
:1051A00090E0A0E8BFE38093A2059093A305A093AD
:1051B000A405B093A50520E030E040E752E46091FB
:1051C00014017091150180911601909117010E94B0
:1051D000BB707B018C0126EA35E042EA55E06EE9BE
:1051E00075E08AE995E00E946D470E94DE5980E0F3
:1051F00090E0A0E0B0EC8093A2059093A305A0936B
:10520000A405B093A50520E030E040E05FE36091A5
:105210000C0170910D0180910E0190910F010E947F
:105220008973FB01462F5F2F682F792F409314015C
:1052300050931501609316017093170120E030E040
:1052400040E752E4BF010E94BB707B018C0126EA5B
:1052500035E042EA55E06EE975E08AE995E00E94A2
:105260006D470E94DE5982E090E00E94E70980913C
:10527000090390910A03A0910B03B0910C03809352
:10528000A2059093A305A093A405B093A505109241
:1052900014011092150110921601109217010E942C
:1052A00071530C944F1A0E94170EAB016093E803E0
:1052B0005093E9038093EA039093EB03BC0185ECE0
:1052C00093E00E945C3358CD0E940E0E0E94237121
:1052D0008B01ECE2F2E00C94E01D0E94882C6B0143
:1052E0007C010C9400210E94882C60938E057093A1
:1052F0008F0580939005909391050E94882C609370
:10530000920570939305809394059093950534CD01
:105310000E94882C681979098A099B09693E7340A3
:105320008105910510F00C9403200C9483200E94B9
:10533000DE595E9A0E944C5A1FCD0E94DE5988E5C4
:105340000E94220E811143C843C8E62FF0E0EE0F01
:10535000FF1FE85FF14F808191810E94635B69A329
:105360007AA38BA39CA36091AB05E62FF0E0EE0F30
:10537000FF1FE45FF14F808191810E94635B20E019
:1053800030E040E85FE30E94DB6F9B01AC0169A164
:105390007AA18BA19CA10E94B47018160CF09DCF2D
:1053A0000C940021A6960FB6F894DEBF0FBECDBFB9
:1053B000DF91CF911F910F91FF90EF90DF90CF90F1
:1053C000BF90AF909F908F907F906F905F904F9025
:1053D0003F902F900895CF93DF938091F2039091A7
:1053E000F303039714F40E94910E60E088E193E0C8
:1053F0000E94FE6B8091F2039091F303892B09F4D4
:1054000060C080911803882309F443C080917A0515
:1054100090917B0520E6289FE001299FD00D112463
:10542000CA50DC4F64E272E0CE010E94D077892B33
:10543000B9F4BE0188E193E00E94906BE7EAF1E0E5
:1054400007C09091C00095FFFCCF8093C6003196B5
:1054500084918111F6CF8091C00085FFFCCF15C0EB
:1054600088E193E00E94F26CEAEAF1E007C09091D3
:10547000C00095FFFCCF8093C600319684918111C6
:10548000F6CF8091C00085FFFCCF8AE08093C600F4
:1054900002C00E9405198091F2039091F3030197D5
:1054A0009093F3038093F20380917A0590917B05AA
:1054B000019664E070E00E94727490937B05809383
:1054C0007A050E942F5C81E00E940A15DF91CF913E
:1054D0000C94B552CF92DF92EF92FF920F931F93ED
:1054E000CF93DF9300D000D0CDB7DEB740E052ECD1
:1054F00061E070E08DEC95E00E94352EEAEDF0E081
:1055000007C09091C00095FFFCCF8093C6003196F4
:1055100084918111F6CF8091C00085FFFCCF8AE095
:105520008093C60087EC90E0FC0107C03091C0007A
:1055300035FFFCCF2093C600319624912111F6CF80
:1055400024B720FF14C0E0EEF0E007C04091C00097
:1055500045FFFCCF3093C600319634913111F6CF20
:105560003091C00035FFFCCF3AE03093C60021FFF8
:1055700014C0E8EEF0E007C04091C00045FFFCCF4A
:105580003093C600319634913111F6CF3091C0007E
:1055900035FFFCCF3AE03093C60022FF14C0E8EF9D
:1055A000F0E007C04091C00045FFFCCF3093C6003B
:1055B000319634913111F6CF3091C00035FFFCCFD8
:1055C0003AE03093C60023FF14C0E9E0F1E007C0E1
:1055D0004091C00045FFFCCF3093C6003196349116
:1055E0003111F6CF3091C00035FFFCCF3AE0309357
:1055F000C60025FF14C0E9E1F1E007C03091C0000A
:1056000035FFFCCF2093C600319624912111F6CFAF
:105610002091C00025FFFCCF2AE02093C60014BED5
:10562000E9E2F1E007C03091C00035FFFCCF2093E4
:10563000C600319624912111F6CFE1E3F1E007C0D5
:105640003091C00035FFFCCF2093C60031962491E5
:105650002111F6CF2091C00025FFFCCF2AE0209336
:10566000C600FC012491E7ECF0E008C03091C000D6
:1056700035FFFCCF2093C600319624912111F6CF3F
:10568000EBE3F1E007C03091C00035FFFCCF209381
:10569000C600319624912111F6CFEBE4F1E007C06A
:1056A0003091C00035FFFCCF2093C6003196249185
:1056B0002111F6CFE6E5F1E007C03091C00035FFDB
:1056C000FCCF2093C600319624912111F6CFE2E65B
:1056D000F1E007C03091C00035FFFCCF2093C60039
:1056E000319624912111F6CF2091C00025FFFCCFE7
:1056F0002AE02093C600FC018491E7ECF0E008C0AA
:105700009091C00095FFFCCF8093C60031968491A4
:105710008111F6CFE6E6F1E007C09091C00095FF59
:10572000FCCF8093C600319684918111F6CF0E9400
:105730007F0D4AE050E0BC018DEC95E00E944B2FBC
:10574000E5E7F1E007C09091C00095FFFCCF8093A2
:10575000C600319684918111F6CF4AE050E060EDA9
:1057600074E08DEC95E00E944B2F8091C00085FF86
:10577000FCCF8AE08093C6001092760510927705E0
:10578000109278051092790580E00E9434177FE628
:10579000C72E7DE0D72EEFE7EE2EEDE0FE2E03E4E0
:1057A0001DE0F60161917191819191916F01F70175
:1057B00021913191419151917F0129833A834B830A
:1057C0005C830E94547129813A814B815C810E94E3
:1057D00089730E942871F801619371938193919369
:1057E0008F01FFE7CF16FDE0DF06D9F60E94B45E19
:1057F0000E94D0450F900F900F900F90DF91CF91A6
:105800001F910F91FF90EF90DF90CF900C949259E1
:105810000E94EA2C0E946A2A0E94EB29FDCF24E80C
:1058200032E0FC01318320832581222319F0029686
:105830000C9443340895CF93DF93EC0185559F4F2B
:105840000E940F2CCE0185599F4F0E940F2CCE0134
:10585000825B9F4F0E940F2CCE01C1960E940F2C9D
:10586000CE014296DF91CF910C940F2C88E193E00A
:105870000C941C6588E193E00C941B2C1F920F92F2
:105880000FB60F9211242F933F938F939F93AF9353
:10589000BF938091C4059091C505A091C605B091B4
:1058A000C7053091CC05232F2D5F2D3720F40196AD
:1058B000A11DB11D05C0232F2A570296A11DB11DA0
:1058C0002093CC058093C4059093C505A093C6058D
:1058D000B093C7058091C8059091C905A091CA05EC
:1058E000B091CB050196A11DB11D8093C805909381
:1058F000C905A093CA05B093CB05BF91AF919F9105
:105900008F913F912F910F900FBE0F901F90189580
:105910000F931F938FB7F8940091C4051091C5059C
:105920002091C6053091C7058FBFB801C9011F91ED
:105930000F9108950F931F939FB7F8940091C80596
:105940001091C9052091CA053091CB0586B5A89B59
:1059500006C08F3F21F00F5F1F4F2F4F3F4F9FBF5C
:10596000322F212F102F0027080F111D211D311D4F
:1059700042E0000F111F221F331F4A95D1F7B801D3
:10598000C9011F910F910895CF92DF92EF92FF927C
:10599000CF93DF936B017C010E949A2CEB010EC028
:1059A0000E949A2C6C1B7D0B683E734038F081E09E
:1059B000C81AD108E108F108C851DC4FC114D1045C
:1059C000E104F10469F7DF91CF91FF90EF90DF9050
:1059D000CF900895789484B5826084BD84B5816049
:1059E00084BD85B5826085BD85B5816085BDEEE6E7
:1059F000F0E0808181608083E1E8F0E010828081C6
:105A000082608083808181608083E0E8F0E0808133
:105A100081608083E1EBF0E0808184608083E0EB53
:105A2000F0E0808181608083EAE7F0E0808184603B
:105A30008083808182608083808181608083808197
:105A4000806880831092C10008951F93CF93DF93E5
:105A5000182FEB0161E00E94B02D209711F460E057
:105A600004C0CF3FD10539F461E0812FDF91CF91A0
:105A70001F910C94CC2DE12FF0E0EF52FD4EE491FC
:105A8000E330B9F028F4E13051F0E230B1F50CC068
:105A9000E63019F1E73049F1E43079F514C084B506
:105AA000806884BDC7BD2EC084B5806284BDC8BD7A
:105AB00029C080918000806880938000D093890005
:105AC000C09388001FC08091800080628093800016
:105AD000D0938B00C0938A0015C08091B00080687D
:105AE0008093B000C093B3000DC08091B00080627D
:105AF0008093B000C093B40005C0C038D1050CF04D
:105B0000B3CFADCFDF91CF911F910895833069F06E
:105B100028F48130A1F0823011F514C08630B1F044
:105B20008730C1F08430D9F404C0809180008F7731
:105B300003C0809180008F7D80938000089584B59C
:105B40008F7702C084B58F7D84BD08958091B000A9
:105B50008F7703C08091B0008F7D8093B00008954F
:105B600090E0FC01EF50FD4E2491FC01EF5EFC4EF5
:105B7000E491EE2381F0F0E0EA5CFC4EA491B0E009
:105B80009FB7F8948C91611103C02095822301C0C6
:105B9000822B8C939FBF08950F931F93CF93DF9316
:105BA0001F92CDB7DEB7A82FB0E0FD01EF52FD4E3A
:105BB0008491FD01EF50FD4E1491FD01EF5EFC4E0E
:105BC00004910023B9F0882321F069830E94862D77
:105BD0006981E02FF0E0EF5CFC4EA491B0E09FB74C
:105BE000F8948C91611103C01095812301C0812B21
:105BF0008C939FBF0F90DF91CF911F910F910895CC
:105C00001F920F920FB60F9211242F933F934F9331
:105C10005F936F938F939F93EF93FF936091C60071
:105C200020914E0630914F06C90101968F77992732
:105C300040915006509151068417950741F0F901A3
:105C4000E253FA4F608390934F0680934E06FF9184
:105C5000EF919F918F916F915F914F913F912F9114
:105C60000F900FBE0F901F9018959A01AB01211550
:105C700081EE380741055105A9F42AC03093C500CB
:105C80002093C4008091C10080618093C100809105
:105C9000C10088608093C1008091C10080688093BA
:105CA000C100089582E08093C00060E079E08DE358
:105CB00090E00E94A8742150310941095109CA019C
:105CC000B90122E030E040E050E00E94A874D6CF55
:105CD0001092C00020E130E0D1CF80915006909129
:105CE000510620914E0630914F062817390769F06A
:105CF000FC01E253FA4F208101968F779927909308
:105D000051068093500630E002C02FEF3FEFC901EB
:105D10000895809150069091510690934F0680937C
:105D20004E0608956F927F928F929F92AF92BF928C
:105D3000CF92DF92EF92FF920F931F93CF93DF9357
:105D4000CDB7DEB7A0970FB6F894DEBF0FBECDBFBC
:105D50008C014115510561057105E1F420E030E049
:105D600040E350E060E070E0A0960FB6F894DEBF2C
:105D70000FBECDBFDF91CF911F910F91FF90EF909C
:105D8000DF90CF90BF90AF909F908F907F906F905B
:105D90000C943A2F66246394712C6C0E7D1EC12CDA
:105DA000D12C7601822E912CA12CB12CCB01BA01E1
:105DB000A50194010E948674FA01D3016D933D01FF
:105DC000BFEFCB1ADB0AEB0AFB0AA901BF014115A1
:105DD00051056105710551F781E0C81AD108E10844
:105DE000F1081AC0E1E0F0E0EC0FFD1FEC0DFD1D25
:105DF0008081482F8A3010F4405D01C0495C50E03A
:105E000060E070E020E030E0C8010E943A2FA1E09D
:105E1000CA1AD108E108F108BFEFCB16DB06EB0682
:105E2000FB0601F7A0960FB6F894DEBF0FBECDBFFC
:105E3000DF91CF911F910F91FF90EF90DF90CF9066
:105E4000BF90AF909F908F907F906F900895211595
:105E5000310539F48091C00085FFFCCF4093C60026
:105E600008950C94922E9A01462F50E060E070E065
:105E70000C94272F2115310539F48091C00085FF3E
:105E8000FCCF4093C60008952A30310511F40C94DC
:105E9000772F0C94922E9A01AB01662757FD6095DF
:105EA000762F0C943A2FCF93DF93EC0120E030E073
:105EB0004DE050E060E070E00E943A2F20E030E0DA
:105EC0004AE050E060E070E0CE01DF91CF910C94A9
:105ED0003A2FCF93DF93EC019A01AB0160E070E0C1
:105EE0000E94272FCE01DF91CF910C94532FCF9298
:105EF000DF92EF92FF92CF93DF93EC016A017B0177
:105F000077FF10C020E030E04DE250E060E070E04C
:105F10000E943A2FF094E094D094C094C11CD11CFC
:105F2000E11CF11C2AE0B701A601CE01DF91CF915F
:105F3000FF90EF90DF90CF900C94922E8F929F92D3
:105F4000AF92BF92CF92DF92EF92FF920F931F9387
:105F5000CF93DF938C014A015B01C22F20E030E038
:105F6000A901C501B4010E94B47087FF0DC020E0F3
:105F700030E04DE250E060E070E0C8010E943A2F4E
:105F8000B7FAB094B7F8B094D0E060E070E080E089
:105F90009FE307C020E030E040E251E40E94BB7084
:105FA000DF5FDC13F7CF262F372F482F592FC5017E
:105FB000B4010E94DB6FD62EE72EF82ED92F0E9457
:105FC0002871962EA72EB82EC92E0E9454719B01BF
:105FD000AC016D2D7E2D8F2D9D2F0E94DA6FD62F57
:105FE000F72EE82ED92E2AE0492D5A2D6B2D7C2D27
:105FF000C8010E94922ECC23C1F1EEE7F2E006C068
:106000009091C00095FFFCCF8093C60081918111D3
:10601000F7CF2BC020E030E040E251E46D2F7F2D20
:106020008E2D9D2D0E9489734B015C01792D9B2D36
:106030000E9423716B01EE24D7FCE094FE2CB70183
:10604000A601C8010E94772FC701B6010E945671B0
:106050009B01AC01682D792D8A2D9B2D0E94DA6F52
:10606000D62FF72EE82ED92EC150C111D3CFDF91F4
:10607000CF911F910F91FF90EF90DF90CF90BF9045
:10608000AF909F908F9008950C949E2FCF93DF93A5
:10609000EC019C012C5F3F4F41E050E060E070E07C
:1060A000898D9A8D0E940F3B8823A1F04D895E89CE
:1060B0006F89788D452B462B472B71F44C815D8180
:1060C0006E817F814D8B5E8B6F8B788F898180682D
:1060D000898302C080E001C081E0DF91CF91089503
:1060E000CF92DF92EF92FF921F93CF93DF93EC0159
:1060F00049895A896B897C89403E5F4F6F417105A0
:1061000008F06DC00E944630882309F468C00E94E0
:106110001A39882309F463C0E98DFA8DCC80DD80BB
:10612000EE80FF8032E0C31AD108E108F10805844F
:1061300004C0CC0CDD1CEE1CFF1C0A94D2F7468573
:10614000578560897189C40ED51EE61EF71E81E051
:1061500080935806C0925B08D0925C08E0925D087C
:10616000F0925E0880E092E0EBE5F6E0DF019C0152
:106170001D9221503040E1F711E011C0B701A60196
:10618000410F511D611D711D2BE536E080915906AF
:1061900090915A060E94906F882309F11F5FE98D44
:1061A000FA8D8481181750F3C12C82E0D82EE12C8F
:1061B000F12C058404C0CC0CDD1CEE1CFF1C0A94E1
:1061C000D2F749895A896B897C894C0D5D1D6E1DFA
:1061D0007F1D498B5A8B6B8B7C8B81E001C080E0EB
:1061E000DF91CF911F91FF90EF90DF90CF900895B6
:1061F000CF93DF93EC0141E0611101C040E06C8579
:106200007D858E859F850E945539882341F0288998
:1062100080E2289F90011124255A394F02C020E0C6
:1062200030E0C901DF91CF910895CF93FB0120E0C9
:1062300030E231932F5F2B30E1F7DC0130E0C7E033
:106240001CC0CA3051F138E0CAE017C0E21729F18A
:10625000FC010196E491E111F9CFC317F0F021326E
:10626000E0F02F37D0F4FB01E30FF11D822F8156B0
:106270008A3108F4205220833F5FCD012D912111F6
:1062800009C0FA018083918381E0FB019081903203
:1062900059F403C02F3219F4F4CF80E005C02E3238
:1062A00081F28DE796E0D4CFCF9108950F931F939D
:1062B000CF93DF93EC018B018B81882311F080E079
:1062C00044C0FB018789803131F528C083E08B838E
:1062D000F801428D538D648D758D4D8B5E8B6F8B68
:1062E000788F9E012F5E3F4FC8010E940F3A88238E
:1062F00031F31A8F098F81E089831C821D821E82EF
:106300001F82188619861A861B861C861D861E8685
:106310001F86188A1AC0803291F6D8CF82E08B830C
:106320001D8A1E8A1F8A188EFB01408D518D60E0E8
:1063300070E095E0440F551F661F771F9A95D1F7BF
:10634000498B5A8B6B8B7C8BD4CFDF91CF911F9174
:106350000F9108952F923F924F925F926F927F928A
:106360008F929F92AF92BF92CF92DF92EF92FF9265
:106370000F931F93CF93DF9300D000D0CDB7DEB73C
:106380009C838B831A01DC0113968C91811103C0CD
:106390002FEF3FEFEEC0EB81FC81818180FFF8CFD2
:1063A000BCC01601201A310A21015B018B819C813E
:1063B00004969A838983ABC0AB81BC8118960D91FA
:1063C0001D912D913C911B97D901C8019170AA276D
:1063D000BB273C01EB81FC8143816801790159E0D5
:1063E000F694E794D794C7945A95D1F7818D928DFE
:1063F000423061F4DC015A966D917D918D919C91B2
:106400005D976C0D7D1D8E1D9F1D4BC0FC01948002
:106410009A949C206114710401F591101EC0012B07
:10642000022B032B59F4EB81FC8185899689A7897E
:10643000B08D84839583A683B7830FC0AB81BC8165
:1064400014964D915D916D917C91179729813A81B8
:106450000E948E39882309F49BCFAB81BC81599669
:10646000ED91FC915A9714966D917D918D919C912F
:1064700017976250710981099109058404C0660F5C
:10648000771F881F991F0A94D2F7068517852089E0
:106490003189600F711F821F931F690D711D811D4E
:1064A000911D20E032E026193709720124153505C7
:1064B00008F47901E114B2E0FB0609F054C0009140
:1064C0005B0810915C0820915D0830915E086017B0
:1064D000710782079307D9F546C0C301855A994FC2
:1064E000A701BC01C5010E948D77AE0CBF1CEB81DA
:1064F000FC8100851185228533850E0D1F1D211D10
:10650000311D00871187228733874E185F08411499
:10651000510409F051CF91012CC0EB81FC81C1885D
:10652000D288E388F48800851185228533852A0185
:10653000612C712C46015701801A910AA20AB30AF4
:10654000481459046A047B0408F02BCF2DCF950121
:10655000AB01BC018091590690915A060E946D6E64
:106560008111C3CF15CF40E00E9455398111B5CFBD
:106570000FCFC9010F900F900F900F90DF91CF9127
:106580001F910F91FF90EF90DF90CF90BF90AF9051
:106590009F908F907F906F905F904F903F902F9043
:1065A0000895CF93DF931F92CDB7DEB741E050E05F
:1065B000BE016F5F7F4F0E94AA31019719F42981B4
:1065C00030E002C02FEF3FEFC9010F90DF91CF9174
:1065D00008950F931F93CF93DF938C01EB01FC0180
:1065E0008381823028F140855185628573854F71A2
:1065F000552766277727452B462B472BC9F440E2C2
:1066000050E0BE01C8010E94AA318032910521F0FC
:10661000892B71F480E00DC088818823D9F3853EF1
:1066200071F38E3261F38B8583FDE9CF80E201C087
:106630008FEFDF91CF911F910F910895CF92DF924D
:10664000EF92FF92CF93DF93EC018B81823018F4AD
:1066500020E030E029C0C884D984EA84FB8475E056
:10666000F694E794D794C7947A95D1F78FE0C8222F
:10667000DD24EE24FF24CE010E94D13297FDE8CF25
:10668000488559856A857B85415E5F4F6F4F7F4F97
:10669000488759876A877B87960165E0220F331FF9
:1066A0006A95E1F7255A394FC901DF91CF91FF90E3
:1066B000EF90DF90CF9008958F929F92AF92BF920C
:1066C000CF92DF92EF92FF920F931F93CF93DF93BE
:1066D000EC014A015B012B81222309F475C08989F1
:1066E0009A89AB89BC8984179507A607B70708F470
:1066F0006BC06CC081149104A104B10449F41C82E4
:106700001D821E821F82188619861A861B865AC011
:10671000088519852A853B85E98DFA8D858590E068
:106720000996B901A8014150510961097109082E62
:1067300004C076956795579547950A94D2F7CC246F
:10674000CA94DC2C7601C80CD91CEA1CFB1C04C0C2
:10675000F694E794D794C7948A95D2F7C416D506D1
:10676000E606F70620F0012B022B032B49F44D8996
:106770005E896F89788D4C835D836E837F8316C0BD
:10678000C41AD50AE60AF70A11C04C815D816E81F0
:106790007F819801898D9A8D0E948E3991E0C91A66
:1067A000D108E108F108811104C014C08E010C5F0A
:1067B0001F4FC114D104E104F10439F7888699868A
:1067C000AA86BB8681E006C080E004C0223009F0C2
:1067D00091CFF4CFDF91CF911F910F91FF90EF9068
:1067E000DF90CF90BF90AF909F908F9008950F93C0
:1067F0001F93CF93DF93EC018B818823E1F1898193
:1068000087FF33C061E0CE010E94F8308C01009711
:1068100091F1FC018081853E71F18B81823040F4E1
:1068200049895A896B897C89448F558F668F778F08
:106830004D895E896F89788DF801538F428F758BF2
:10684000648BE0915206F0915306309759F0B801ED
:106850006A5E7F4FC80148960995F801808D918D39
:10686000938B828B89818F778983DF91CF911F9161
:106870000F910C941A3981E0888380E0DF91CF91E9
:106880001F910F910895CF93DF93EC010E94F7338E
:106890001B82DF91CF910895FC01238121110C947B
:1068A000433408956F927F928F929F92AF92BF92DE
:1068B000CF92DF92EF92FF920F931F93CF93DF93CC
:1068C00000D000D0CDB7DEB73C016A017B01FC01EE
:1068D0008381813009F083C0818181FF80C081C0C4
:1068E000452B462B472B09F478C0F3018084918413
:1068F000A284B384B701A601C3010E945C33811155
:1069000001C06DC0F301818D928DC114D104E104E9
:10691000F10479F4458956896789708D0E94203C7D
:10692000882309F45CC0F301158A168A178A108E31
:106930003AC0F30144815581668177819E012F5FC2
:106940003F4F0E948E39882309F449C049815A81FA
:106950006B817C81F301818D928DFC01278920312F
:1069600039F4483FFFEF5F0761057105E0F407C0A8
:10697000483F2FEF520762072FE07207A0F40E94F2
:10698000203C882361F1F301448155816681778140
:106990000FEF1FEF2FEF3FE0818D928D0E94773A2E
:1069A000811101C01CC0F301C18AD28AE38AF48A32
:1069B000818180688183C3010E94F733882379F045
:1069C000B701A6018C149D04AE04BF0410F4B501F8
:1069D000A401C3010E945C3310C081E00EC080E0BE
:1069E0000CC0F30141895289638974894C155D0596
:1069F0006E057F0508F074CFF2CF0F900F900F90C7
:106A00000F90DF91CF911F910F91FF90EF90DF904A
:106A1000CF90BF90AF909F908F907F906F90089590
:106A2000CF93DF93EC0140E050E0BA010E94523472
:106A3000882371F061E0CE010E94F830009741F0A8
:106A400025EEFC0120831B82DF91CF910C941A3933
:106A500080E0DF91CF910895FF920F931F93CF9322
:106A6000DF93EC01F42E80E2689FF0011124E55AD7
:106A7000F94F8385817121F0842F827109F05CC008
:106A800000915B0810915C0820915D0830915E08D0
:106A90000C871D872E873F87688B4489558960E066
:106AA00070E0BA0155274427028D138D20E030E0B5
:106AB000402B512B622B732B4D8B5E8B6F8B788F02
:106AC0008385887151F4048D158D268D378D098B42
:106AD0001A8B2B8B3C8B81E00CC0803169F59E01B9
:106AE0002F5E3F4F898D9A8D0E940F3A882321F1A6
:106AF00084E08B838F2D8F7089831C821D821E8280
:106B00001F82188619861A861B86F4FE18C040E07C
:106B100050E0BA01CE010E945234811110C012C05F
:106B200049895A896B897C89CE01DF91CF911F9168
:106B30000F91FF900C945C331B8280E003C0F5FC46
:106B4000EFCF81E0DF91CF911F910F91FF900895DA
:106B50006F927F928F929F92AF92BF92CF92DF926D
:106B6000EF92FF920F931F93CF93DF935C01EB01A2
:106B70004A01722E898D9A8DF501928F818F40E0A6
:106B800050E0BA01CE010E945C33612C33C045E075
:106B900036952795179507954A95D1F70F70CE0131
:106BA0000E941E33DC01009709F495C08C91882364
:106BB00011F0853EB1F4611010C0C0905B08D09018
:106BC0005C08E0905D08F0905E08F501C486D5860B
:106BD000E686F786008B662463948C9181110AC047
:106BE00075C04BE050E0BD01C4010E948077009762
:106BF00009F46FC0088519852A853B85C988DA881C
:106C0000EB88FC880C151D052E053F0508F4BFCF49
:106C10005DC071FE60C0662051F0F501008961E041
:106C2000C5010E94F830EC01009771F454C08B81CB
:106C3000823009F450C0CE010E947030882309F4DC
:106C40004AC0CBE5D6E000E080E2FE0111928A95D1
:106C5000E9F78BE0F401DE0101900D928A95E1F7EE
:106C6000E0915206F0915306309739F0BE01625F11
:106C70007F4FCE014096099508C081E298E2998B3A
:106C8000888B80E098E09F878E87888999899B8B85
:106C90008A8B998F888F8E859F859F8B8E8B0E9484
:106CA0001A398823C1F0472D602FC501DF91CF919C
:106CB0001F910F91FF90EF90DF90CF90BF90AF901A
:106CC0009F908F907F906F900C942C3576FCA1CF85
:106CD00002C077FEE8CF80E0DF91CF911F910F9146
:106CE000FF90EF90DF90CF90BF90AF909F908F90EC
:106CF0007F906F9008955F926F927F928F929F9294
:106D0000AF92BF92CF92DF92EF92FF920F931F93B9
:106D1000CF93DF93CDB7DEB7C354D1090FB6F89444
:106D2000DEBF0FBECDBF5C016B0124965FAF4EAFDF
:106D30002497522E1C8E1F8E19821C82611571059C
:106D400011F410E075C0FC0183818111FACF249603
:106D5000EEADFFAD249780818F3239F0760117C0F8
:106D600031962496FFAFEEAF24972496EEADFFAD9B
:106D7000249780818F32A1F3F60183818250823083
:106D800060F4ECCFEE24E394F12CEC0EFD1E8E01AA
:106D9000045E1F4F480138010CC0F601618D728DF1
:106DA000CE0101960E9456318111ECCFCACF7801F5
:106DB0008301AE014E5B5F4FBE01695C7F4F24963D
:106DC0008EAD9FAD24970E941531811106C0B9CFB9
:106DD00031962496FFAFEEAF24972496EEADFFAD2B
:106DE000249780818F32A1F38823C9F021E0AE017E
:106DF000495C5F4FB701C8010E94A835882309F498
:106E0000A0CFEC14FD0419F0C7010E94433408150B
:106E1000190569F68E010F5F1F4F7301CACF252D2B
:106E2000AE01495C5F4FB701C5010E94A835182F1C
:106E3000CE0101960E944C34CE014C960E944C34F7
:106E4000812FCD5BDF4F0FB6F894DEBF0FBECDBFF5
:106E5000DF91CF911F910F91FF90EF90DF90CF9036
:106E6000BF90AF909F908F907F906F905F900895AC
:106E70001F93CF93DF93CDB7DEB76B970FB6F89420
:106E8000DEBF0FBECDBFAB0119821C8222E0BC0168
:106E9000CE0101960E947B36882331F0CE01019607
:106EA0000E941035182F01C010E0CE0101960E94FB
:106EB0004C34812F6B960FB6F894DEBF0FBECDBF5A
:106EC000DF91CF911F9108952F923F924F925F9241
:106ED0007F928F929F92AF92BF92CF92DF92EF926A
:106EE000FF920F931F93CF93DF9300D000D000D079
:106EF000CDB7DEB71C01162F072F5E834D83DC0153
:106F000013968C911397813009F054C111968C918E
:106F100081FF50C155C1F10141895289638974894A
:106F200080859185A285B38584179507A607B70745
:106F300029F4AD80BE80812E902E07C1C1010E9430
:106F40005C338111F6CF36C1D10159968D919C9158
:106F50005A97FC0174807A94B701A601E9E076950E
:106F6000679557954795EA95D1F77422F1E0DF22AE
:106F7000EE24FF24260171104AC0C114D10409F087
:106F800046C014964D915D916D917C911797411576
:106F900051056105710561F455960D911D912D9175
:106FA0003C915897011511052105310549F522C07D
:106FB0009E012F5F3F4F0E948E39882309F4FAC04B
:106FC00009811A812B813C81D1015996ED91FC9167
:106FD0005A978789803139F4083FBFEF1B07210595
:106FE000310540F40DC0083FEFEF1E072E07EFE01C
:106FF0003E0730F0C1010E944630811108C0DAC05E
:10700000D10114960D931D932D933C93179780E017
:1070100092E08419950985018A159B0508F48C0175
:10702000D1015996ED91FC915A971496CD90DD902F
:10703000ED90FC901797B2E0CB1AD108E108F10867
:10704000058404C0CC0CDD1CEE1CFF1C0A94D2F796
:1070500086859785A089B189C80ED91EEA1EFB1EB8
:10706000C70CD11CE11CF11C0115E2E01E0731F533
:1070700080915B0890915C08A0915D08B0915E08DA
:107080008C159D05AE05BF0569F4109258068FEF6B
:107090009FEFDC0180935B0890935C08A0935D08F0
:1070A000B0935E089401B701A601809159069091B2
:1070B0005A060E94906F811137C07CC04114510460
:1070C00019F5D10118964D915D916D917C911B97A9
:1070D00051968D919D910D90BC91A02D4817590707
:1070E0006A077B0788F00E941A39882309F462C076
:1070F00081E080935806C0925B08D0925C08E092D1
:107100005D08F0925E0808C041E0C701B6010E9428
:107110005539882309F44EC09201255A394FA801E8
:10712000B401C9010E948D77F101C084D184E28449
:10713000F384C00ED11EE11CF11CC086D186E2860C
:10714000F386800E911EA01AB10AF101C084D18489
:10715000E284F384A114B10409F0F6CE0189128906
:10716000238934890C151D052E053F0530F4D10106
:10717000C18AD28AE38AF48A0BC080915206909128
:107180005306892B59F0ED81FE81EF2B39F0D101A7
:1071900011968C911197806811968C93F1018181E1
:1071A00083FD03C02D813E810EC0C1010E94F733D3
:1071B0008111F8CF81E0D1018C932FEF3FEF03C015
:1071C00082FDA9CEB6CEC90126960FB6F894DEBFD1
:1071D0000FBECDBFDF91CF911F910F91FF90EF9028
:1071E000DF90CF90BF90AF909F908F907F905F90F7
:1071F0004F903F902F900895DB010D900020E9F70C
:10720000AD0141505109461B570B02960C9464374F
:10721000CF93DF931F92CDB7DEB7698341E050E093
:10722000BE016F5F7F4F02960E9464370F90DF911F
:10723000CF910895809158068823A9F140915B0869
:1072400050915C0860915D0870915E082BE536E016
:107250008091590690915A060E94906F811102C048
:1072600080E008954091540650915506609156066D
:1072700070915706411551056105710591F02BE597
:1072800036E08091590690915A060E94906F8823AB
:1072900039F3109254061092550610925606109229
:1072A00057061092580681E00895CF92DF92EF9230
:1072B000FF92CF936B017C01C42F80915B0890916A
:1072C0005C08A0915D08B0915E088C159D05AE0527
:1072D000BF05D1F00E941A39811102C080E018C0A8
:1072E0002BE536E0B701A6018091590690915A0628
:1072F0000E946D6E882391F3C0925B08D0925C0867
:10730000E0925D08F0925E0881E0C111809358061A
:10731000CF91FF90EF90DF90CF900895AF92BF9202
:10732000CF92DF92EF92FF920F931F93CF93DF9351
:107330005C016A017B01E901FC014185528563859D
:1073400074854F5F5F4F6F4F7F4F4C155D056E0526
:107350007F0510F480E058C0FC018789803129F452
:1073600099278F2D7E2D6D2D0CC0803299F7C70186
:10737000B60127E096958795779567952A95D1F779
:10738000F5010389148925893689600F711F821FD1
:10739000931F00915B0810915C0820915D0830916B
:1073A0005E08601771078207930729F4F501878942
:1073B0008031A1F406C040E00E9455398111F6CF1A
:1073C000C9CFDD24EE24FF24F601EE0FFF1FE55A9E
:1073D000F94F80819181A0E0B0E011C0E894C7F836
:1073E000DD24EE24FF24F601EE0FFF1FEE0FFF1F3A
:1073F000E55AF94F80819181A281B381BF70888362
:107400009983AA83BB8381E0DF91CF911F910F9174
:10741000FF90EF90DF90CF90BF90AF9008956F9264
:107420007F928F929F92AF92BF92CF92DF92EF9214
:10743000FF920F931F93CF93DF9300D000D0CDB76F
:10744000DEB78C0149835A836B837C833901C12C5D
:10745000D12C7601812C42E0942EA12CB12C4981B3
:107460005A816B817C819E012F5F3F4FC8010E9432
:107470008E39882341F1D501C401F801058404C087
:10748000880F991FAA1FBB1F0A94D2F7C80ED91ED6
:10749000EA1EFB1E49815A816B817C81878980317C
:1074A00031F4483F5F4F6105710530F4D8CF483F54
:1074B0005F4F6F4F7F4098F2F301C082D182E2822A
:1074C000F38281E001C080E00F900F900F900F9049
:1074D000DF91CF911F910F91FF90EF90DF90CF90B0
:1074E000BF90AF909F908F907F906F9008956F9214
:1074F0007F928F929F92AF92BF92CF92DF92EF9244
:10750000FF920F931F93CF93DF9300D0CDB7DEB7D9
:107510003C014A015B01423051056105710508F4E7
:107520006CC0F30141855285638574854F5F5F4F61
:107530006F4F7F4F481559056A057B0508F45DC0FC
:107540008789803129F4FF24EB2CDA2CC92C0DC05B
:10755000803209F052C07501640177E0F694E79437
:10756000D794C7947A95D1F7F30183899489A58933
:10757000B689C80ED91EEA1EFB1E41E0C701B6013E
:1075800029833A830E94553929813A818823A9F1B8
:10759000F3018789803159F49924AA24BB24F4018A
:1075A000EE0FFF1FE55AF94F1183008310C0E894D6
:1075B00087F89924AA24BB24F401EE0FFF1FEE0FD5
:1075C000FF1FE55AF94F0083118322833383F301B0
:1075D0008289823080F085819681A781B0858C0D6B
:1075E0009D1DAE1DBF1D8093540690935506A0931C
:1075F0005606B093570681E001C080E00F900F90CF
:10760000DF91CF911F910F91FF90EF90DF90CF907E
:10761000BF90AF909F908F907F906F9008952F9222
:107620003F924F925F926F927F928F929F92AF9212
:10763000BF92CF92DF92EF92FF920F931F93CF935F
:10764000DF93CDB7DEB72F970FB6F894DEBF0FBE2E
:10765000CDBF1C014C875D876E877F873B872A875C
:10766000DC0119964D905D906D907C901C97BFEF5A
:107670004B1A5B0A6B0A7B0AF90180809180A28019
:10768000B38081149104A104B10431F0FFEF8F1A8B
:107690009F0AAF0ABF0A10C0DC018D909D90AD908B
:1076A000BC90B1E0BD832C853D854E855F85213042
:1076B00031054105510509F01D82750164011E82E5
:1076C0001F8218861986F10181859285A385B4856C
:1076D0002E813F8148855985281739074A075B075E
:1076E00008F052C04C145D046E047F0450F4B2E004
:1076F000CB2ED12CE12CF12C12E0812E912CA12C3F
:10770000B12C9E012F5F3F4FB701A601C1010E941E
:107710008E398823C9F149815A816B817C81D701D7
:10772000C6010196A11DB11D452B462B472B19F013
:107730004C015D010DC088199909AA09BB092C8566
:107740003D854E855F8582179307A407B50789F0AD
:107750008E819F81A885B9850196A11DB11D8E835B
:107760009F83A887B9879FEFC91AD90AE90AF90A3E
:10777000AACF0FEF1FEF2FEF3FE0A601B701C10126
:107780000E94773A811115C080E041C044244A9498
:10779000542C32014C0C5D1C6E1C7F1C9701860121
:1077A000B301A201C1010E94773A882369F37301F2
:1077B00062018C149D04AE04BF0440F3AA85BB850E
:1077C0004D915D916D917C9141155105610571055A
:1077D00051F4EA85FB8580829182A282B382FD8189
:1077E000F11109C013C095018401C1010E94773ACB
:1077F0008111EFCFC9CF2FEF821A920AA20AB20AE3
:10780000D1018D929D92AD92BC92139781E02F96FB
:107810000FB6F894DEBF0FBECDBFDF91CF911F91A1
:107820000F91FF90EF90DF90CF90BF90AF909F901F
:107830008F907F906F905F904F903F902F90089522
:10784000AF92BF92CF92DF92EF92FF920F931F936E
:10785000CF93DF9300D000D0CDB7DEB75C016A01D3
:107860007B0142E050E060E070E0FC014083518326
:10787000628373839E012F5F3F4FB701A601C5014D
:107880000E948E39811102C080E023C000E010E028
:107890009801B701A601C5010E94773A8823A1F398
:1078A000C980DA80EB80FC80F5018789803141F462
:1078B000F8EFCF16FFEFDF06E104F10448F4DACF6A
:1078C00088EFC8168FEFD806E8068FE0F80690F22A
:1078D00081E00F900F900F900F90DF91CF911F914B
:1078E0000F91FF90EF90DF90CF90BF90AF900895F1
:1078F0008F929F92AF92BF92CF92DF92EF92FF92C0
:107900000F931F93CF93DF93EC01142F70935A06BC
:10791000609359061F8A52E0C52ED12CE12CF12C20
:10792000C882D982EA82FB821092580610925406CD
:10793000109255061092560610925706CC24CA94FF
:10794000DC2C7601C0925B08D0925C08E0925D0866
:10795000F0925E08442359F1453008F0DDC040E064
:1079600060E070E0CB010E945539882309F4D4C04F
:1079700020E1129FF0011124E75FF74F80818F779C
:1079800009F0CAC0C484D584E684F78434E6C316FB
:10799000D104E104F10408F4BFC0C084D184E284BE
:1079A000F384C114D104E104F10421F4B5C0C12C65
:1079B000D12C760140E0C701B6010E9455398823D9
:1079C00009F4AAC0809166069091670681159240DD
:1079D00009F0A2C020916B06222309F49DC080917A
:1079E000690690916A06009709F496C0409168066E
:1079F000442309F491C02A8B4C831D8650E061E03A
:107A000070E006C02E2F2F5F2D87E83008F084C06D
:107A1000ED859B010E2E02C0220F331F0A94E2F760
:107A20004217530779F7209171063091720621159C
:107A3000310519F040E050E008C020917F063091F8
:107A4000800640918106509182062D833E834F83AC
:107A5000588746015701880E991EA11CB11C8B8ABC
:107A60009C8AAD8ABE8A00916C0610916D06198FB2
:107A7000088FA0916B06B0E00E944F74680D791DCD
:107A80008A1D9B1D6A8F7B8F8C8F9D8F980105E0CF
:107A9000220F331F0A95E1F721503E4F232F332742
:107AA0002695DC01CB01820F931FA11DB11D8E878E
:107AB0009F87A88BB98B80906E0690906F0681147B
:107AC000910419F0A12CB12C08C080907B069090F5
:107AD0007C06A0907D06B0907E06A7019601281B2B
:107AE000390B4A0B5B0BDA01C901880D991DAA1DE0
:107AF000BB1D04C0B695A79597958795EA95D2F7D3
:107B000089879A87AB87BC87853F3FE09307A105AC
:107B1000B10520F48CE08F8B80E016C0853F9F4F2D
:107B2000A105B10510F480E10DC040918706509188
:107B300088066091890670918A064A8F5B8F6C8FE8
:107B40007D8F80E28F8B81E0DF91CF911F910F912C
:107B5000FF90EF90DF90CF90BF90AF909F908F906D
:107B600008952F923F924F925F926F927F928F92E1
:107B70009F92AF92BF92CF92DF92EF92FF920F93BC
:107B80001F93CF93DF93CDB7DEB7CA54D1090FB699
:107B9000F894DEBF0FBECDBF1C017E8B6D8B3A010A
:107BA0002BA30EA3E8A6AEAABFAAC8AED9AE34E0F6
:107BB000239F80011124400F511F5BAB4AABDA01B8
:107BC0008D909D90AD90BC90FC01E00FF11F208145
:107BD000318142815381C501B4010E94DB6F6AAFDC
:107BE0007BAF8CAF9DAFEEA1B4E0EB9F7001112491
:107BF00093012E0D3F1D3DAB2CABD9014D905D90F7
:107C00006D907C90F101EE0DFF1D2081318142814C
:107C10005381C301B2010E94DB6F6EAF7FAF21962B
:107C20008FAF219722969FAF2297E8A5B4E0EB9FF4
:107C3000C0011124F101E80FF91F20813181428137
:107C400053812B8F3C8F4D8F5E8FED89FE89E80F1E
:107C5000F91F60817181828193810E94DA6F462FC2
:107C6000572F682F792F498B5A8B6B8B7C8BAD8963
:107C7000BE891C968D919D910D90BC91A02D8AA7D7
:107C80009BA7ACA7BDA7D1011C962D913D914D910D
:107C90005C911F972F8F38A349A35AA3B7FAB094CA
:107CA000B7F8B09477FA709477F87094ED89FE89FC
:107CB000E00FF11F7AAD6BAD9CAD8DAD272F362F48
:107CC000492F582F60817181828193810E94DA6FE0
:107CD0006F8B788F898F9DA3ED89FE89EE0DFF1D37
:107CE0007EAD6FAD21969FAD219722968FAD2297E5
:107CF000272F362F492F582F6081718182819381E0
:107D00000E94DA6F162F072F382E292E7F89688D53
:107D1000998D8DA1272F362F492F582FC501B401DA
:107D20000E9489736B017C01B801C101272F362F96
:107D3000492F582FC301B2010E9489739B01AC01E6
:107D4000C701B6010E94DB6F6B017C01B801C10164
:107D5000272F362F492F582FC501B4010E94897350
:107D60006EA77FA788AB99AB7F89688D998D8DA110
:107D7000272F362F492F582FC301B2010E94897334
:107D80009B01AC016EA57FA588A999A90E94DA6F15
:107D9000A70196010E944E70362E272E182F092F0C
:107DA00020E030E0A901D101F8016B2F7A2F8F2F4D
:107DB0009E2F0E94B47087FF10C02BED3FE049EC6E
:107DC00050E4D101F8016B2F7A2F8F2F9E2F0E9444
:107DD000DB6F362E272E182F092FA4968FADA49770
:107DE000882381F02BED3FE049EC50E4D101F8010C
:107DF0006B2F722D8F2F902F0E94DA6F362E272E29
:107E0000182F092FC988DA88EB88FC88E894F7F8DE
:107E1000A3962CAD3DAD4EAD5FADA397D101F8015A
:107E20006B2F722D8F2F902F0E948973A7019601BF
:107E30000E94C4726B017C012FE632E143E85AE3F1
:107E40000E94B47087FD90C2C701B6010E94917173
:107E50000E9428717A8F698FFB01EF2B21F421E0BA
:107E600030E03A8F298F498D5A8DBA0180E090E039
:107E70000E9454716B017C019B01AC01D101F8019E
:107E80006B2F722D8F2F902F0E94BB706F8B788F6E
:107E90001C01A701960169897A898B899C890E94B6
:107EA000BB7024966FAF249725967FAF25972696B3
:107EB0008FAF269727969FAF27972F8D38A149A17F
:107EC0005AA16AA57BA58CA59DA50E94DA6FA70182
:107ED00096010E94BB7028966FAF289729967FAFB6
:107EE00029972A968FAF2A972B969FAF2B9720E042
:107EF00030E040E05FE3BF89A88D6B2F7A2F822DA1
:107F0000932D0E948973BF89A88D2B2F3A2F422D64
:107F1000532D0E9489739B01AC0160E070E080E802
:107F20009FE30E94DA6F6DA37AA78EA723969FAF77
:107F30002397CE010196FC01A8A554E0A59FE00D72
:107F4000F11D11242B8D3C8D4D8D5E8D2083318351
:107F5000428353832F8D38A149A15AA12D873E8793
:107F60004F87588B198A41E050E05C8F4B8F81E03E
:107F700090E08C0F9D1FBBA1A4E0BA9F800D911DC6
:107F8000112499A788A721E030E02C0F3D1F5EA1A6
:107F900044E0549F200D311D11243FA32EA3FCA3C8
:107FA000EBA3C1C1898989310CF050C07F89688DEC
:107FB000272F362F422D532DC501B4010E948973FE
:107FC0006B017C017DA16AA59EA523968FAD2397A9
:107FD000272F362F492F582FC301B2010E948973D2
:107FE0009B01AC01C701B6010E94DB6F7B018C01D4
:107FF0007DA16AA59EA523968FAD2397272F362FA7
:10800000492F582FC501B4010E9489735B016C018F
:108010007F89688D272F362F422D532DC301B20142
:108020000E9489739B01AC016A2D7B2D8C2D9D2DA7
:108030000E94DA6F862E972EA82EB92E99899F5FFF
:10804000998B4E2C5F2C602E712E72C0AB8DBC8D27
:10805000BD0180E090E00E945471BF89A88D2B2F54
:108060003A2F422D532D0E9489737B018C017F2D65
:10807000802F912F0E94B8702B013C016E2D7F2D17
:10808000802F912F0E94EC73698B7A8B8B8B9C8B4A
:10809000EAA9FBA980819181A281B3819C01AD01F4
:1080A00050582F8F38A349A35AA3ACA9BDA9CD908E
:1080B000DD90ED90FC90A30192016F8D78A189A1D4
:1080C0009AA10E9489734B015C0129893A894B89E5
:1080D0005C89C701B6010E9489739B01AC01C5018F
:1080E000B4010E94DB6F862E972EA82EB92E298907
:1080F0003A894B895C896F8D78A189A19AA10E94E8
:108100008973698B7A8B8B8B9C8BA3019201C7013E
:10811000B6010E9489739B01AC0169897A898B89B8
:108120009C890E94DA6F462E572E682E792E198A66
:10813000A5019401BAADABADFCADEDAD6B2F7A2FBF
:108140008F2F9E2F0E94DB6FE8A5F9A560837183B6
:1081500082839383A3019201BEADAFAD2196FFADA3
:1081600021972296EFAD22976B2F7A2F8F2F9E2F7C
:108170000E94DB6FAEA1BFA16D937D938D939C9305
:10818000139724967FAD249725966FAD2597269655
:108190009FAD269727968FAD2797272F362F492FEC
:1081A000582FEBA1FCA160817181828193810E9493
:1081B000DB6FABA1BCA16D937D938D939C931397C3
:1081C00028967FAD289729966FAD29972A969FAD5F
:1081D0002A972B968FAD2B97272F362F492F582F65
:1081E0006D857E858F8598890E94DB6F6D877E8780
:1081F0008F87988BC090E902D090EA02E090EB0262
:10820000F090EC02A701960169817A818B819C81B3
:108210000E94B47087FF04C0C982DA82EB82FC82BC
:10822000C090ED02D090EE02E090EF02F090F002EC
:10823000A70196016D817E818F8198850E94B4701F
:1082400087FF04C0CD82DE82EF82F886C090F10203
:10825000D090F202E090F302F090F402A7019601B0
:1082600069857A858B859C850E94B47087FF04C0E0
:10827000C986DA86EB86FC8620E030E04BE153E4E9
:1082800069817A818B819C810E94B772181644F4AF
:1082900080E090E0ABE1B3E489839A83AB83BC8355
:1082A00020E030E046E153E46D817E818F81988546
:1082B0000E94B772181644F480E090E0A6E1B3E49F
:1082C0008D839E83AF83B88720E030E044EB52E497
:1082D00069857A858B859C850E94B772181644F44F
:1082E00080E090E0A4EBB2E489879A87AB87BC87F3
:1082F00094E6C92ED12CCC0EDD1EEEA8FFA808AD49
:1083000019AD9E01235F3F4FAE01475F5F4FBE0136
:108310006B5F7F4FCE0101960E946D47EB8DFC8D08
:108320003196FC8FEB8F2B8D3C8D498D5A8D241708
:10833000350708F437CE2D893E89245F3F4F4D899C
:108340005E89485F5F4F6D897E896C5F7F4F84E6F1
:10835000C82ED12CCC0EDD1EEEA8FFA808AD19AD9D
:108360008D899E890E946D47C65BDF4F0FB6F894DA
:10837000DEBF0FBECDBFDF91CF911F910F91FF9058
:10838000EF90DF90CF90BF90AF909F908F907F90B5
:108390006F905F904F903F902F9008952F923F9253
:1083A0004F925F926F927F928F929F92AF92BF9205
:1083B000CF92DF92EF92FF920F931F93CF93DF93B1
:1083C000CDB7DEB768970FB6F894DEBF0FBECDBF4E
:1083D0001C014A015B0168017901DC01D8966D91AD
:1083E0007D918D919C91DB970E94547169837A8372
:1083F0008B839C83A50194010E9489730E94A170C4
:108400000E9428716D837E838F839887A7019601D0
:1084100069817A818B819C810E9489730E94A170FD
:108420000E94287169877A878B879C872D813E817E
:108430004F815885283731054105510540F488E7BB
:1084400090E0A0E0B0E08D839E83AF83B88729855C
:108450003A854B855C85283731054105510540F447
:1084600088E790E0A0E0B0E089879A87AB87BC8777
:10847000F101EC5BFF4F4080518062807380C3014B
:10848000B2010E9456716B017C01D101DC966D91A5
:108490007D918D919C91DF970E9454716D877E87AD
:1084A0008F87988B20E030E0A901C701B6010E94B8
:1084B000B470882339F129813A814B815C81CA01EA
:1084C000B9010E9489734B015C012D853E854F8562
:1084D0005889CA01B9010E9489739B01AC01C50189
:1084E000B4010E94DA6F4B015C01A7019601C7013C
:1084F000B6010E94DB6F9B01AC01C501B4010E9473
:10850000BB7004C060E070E080E090E00E94A17069
:108510000E9423714B015C0166277727CB01641908
:108520007509860997090E9456712B013C01F101DA
:10853000E05CFF4F60817181828193810E94547160
:10854000698B7A8B8B8B9C8B20E030E0A901C30177
:10855000B2010E94B470882379F129893A894B8944
:108560005C89CA01B9010E9489736D8B7E8B8F8BE8
:10857000988F29813A814B815C81CA01B9010E949F
:1085800089739B01AC016D897E898F89988D0E94CA
:10859000DA6F69837A838B839C83A3019201C30181
:1085A000B2010E94DB6F9B01AC0169817A818B81F2
:1085B0009C810E94BB7004C060E070E080E090E0AD
:1085C0000E949171D10150962D913D914D915C91F8
:1085D000539729833A834B835C8329013A014818D6
:1085E00059086A087B080E942371461A570A680ACC
:1085F000790A77FE6CC020E030E0A901C701B6011E
:108600000E94B470882309F445C0A7019601C701F0
:10861000B6010E94DB6F2B013C0169817A818B815D
:108620009C810E9454719B01AC01C301B2010E9464
:1086300089732B013C012D853E854F855889CA01E0
:10864000B9010E9489739B01AC01C301B2010E9470
:10865000DA6F2B013C0129893A894B895C89CA016F
:10866000B9010E9489739B01AC01C301B2010E9450
:10867000DB6F4B015C0120E030E040E850E4C701D3
:10868000B6010E9489739B01AC01C501B4010E942F
:10869000BB7004C060E070E080E090E00E94A170D8
:1086A0000E9423714B015C01B7FE03C0812C912C09
:1086B000540129813A814B815C8182169306A4067C
:1086C000B50610F049015A01412C512C32018FB7E7
:1086D000F894F101E45BFF4F9081911125C0D10125
:1086E00054968D929D92AD92BC925797480C591C0E
:1086F0006A1C7B1CF101408E518E628E738E2D811F
:108700003E814F815885DC962D933D934D935C932C
:10871000DF97A05CBF4F29853A854B855C852D93FB
:108720003D934D935C9313978FBF68960FB6F89463
:10873000DEBF0FBECDBFDF91CF911F910F91FF9094
:10874000EF90DF90CF90BF90AF909F908F907F90F1
:108750006F905F904F903F902F900895AF92BF928F
:10876000CF92DF92EF92FF920F931F93CF93DF93FD
:108770005B017A016115710509F475C04115510558
:1087800009F471C0FB0102A513A5D4A5C5A5CE01AE
:10879000202F312F492F582F66A177A180A591A5B1
:1087A0000E94B470882309F45EC0F50187A9811185
:1087B0004BC0F701C6A0D7A0E0A4F1A4A701960181
:1087C000DE01602F712F8B2F9A2F0E94B77218161F
:1087D000DCF5A7019601C701B6010E9489736B0100
:1087E0007C01F50182A993A9A4A9B5A9BC01CD0179
:1087F00090589B01AC010E94DB6FF50126A537A5BF
:1088000040A951A90E9489739B01AC01C701B6011F
:108810000E94DA6F0E94F6736B017C01762F272F7E
:108820003D2D4E2D5F2DFE01602F712F8F2F9E2F1E
:108830000E94B47087FF03C06801ED2EFC2E5C2DF2
:108840004D2D3E2D2F2D03C0502F412F9E01852FE2
:10885000942FA32FB22FF50186A397A3A0A7B1A7AA
:1088600081E0F50186ABDF91CF911F910F91FF90D1
:10887000EF90DF90CF90BF90AF900895CF92DF92AE
:10888000EF92FF920F931F93CF93DF931F92CDB779
:10889000DEB7809161088FB7F894F09060088FBFC1
:1088A0008091610890E08F1991098F709927049742
:1088B00004F12091610823502F7040E050E000E067
:1088C00010E08DE4E82E13C0211101C020E12150F9
:1088D000E29E6001112482E698E0C80ED91EB8011C
:1088E000C60129830E94AE43A801860129812F1168
:1088F000EBCF0F90DF91CF911F910F91FF90EF90F1
:10890000DF90CF9008952F923F924F925F926F9297
:108910007F928F929F92AF92BF92CF92DF92EF920F
:10892000FF920F931F93CF93DF93EC011B010097EE
:1089300009F464C08FA9811161C08EA09FA0A8A472
:10894000B9A4FB01C6A0D7A0E0A4F1A42C2D3D2D15
:108950004E2D5F2DC501B4010E94B47087FF4EC03B
:10896000A5019401C501B4010E9489732B013C014A
:108970008AA89BA8ACA8BDA8C501B40190589B01CA
:10898000AC010E94DB6F2EA53FA548A959A90E9402
:1089900089739B01AC01C301B2010E94DA6F0E948E
:1089A000F6738B01D82FC92F762FCE01272F312FA9
:1089B000492F582F6C2D7D2D8E2D9F2D0E94B47028
:1089C00087FF03C08601DE2DCF2DCE01202F312F52
:1089D000492F5C2F6C2D7D2D8E2D9F2D0E94B47004
:1089E000882361F09E01802F912FA32FBC2FF101CE
:1089F00086A397A3A0A7B1A781E086ABDF91CF9113
:108A00001F910F91FF90EF90DF90CF90BF90AF90AC
:108A10009F908F907F906F905F904F903F902F909E
:108A20000895EF92FF920F931F93CF93DF93F090EF
:108A30006008C0E0D0E080E090E02DE4E22E11C0BC
:108A4000EF9C800111240E59174FA801BE010E940E
:108A500083448F2D8F5F803109F480E0F82ECE01A2
:108A6000E80120916108F212EBCF40E050E0BE0136
:108A7000DF91CF911F910F91FF90EF900C94834461
:108A80004F925F926F927F928F929F92AF92BF921E
:108A9000CF92DF92EF92FF920F931F93CF93DF93CA
:108AA00050906008C0E0D0E03DE4432E37C0489EBF
:108AB0003001499E700C112482E698E0680E791E00
:108AC000209731F18EA9811104C0F30186A9882372
:108AD000F9F0CAA0DBA0ECA0FDA0A7019601F3016C
:108AE00066A177A180A591A50E94BB704B015C0196
:108AF000A70196016EA17FA188A599A50E94BB70D0
:108B0000AB01BC0195018401CE010E94CE411EAA99
:108B10005394F0E15F1201C0512CE301852D992798
:108B200087FD90952091610830E08217930709F046
:108B3000BECF2097F1F0CAA0DBA0ECA0FDA0A7015A
:108B400096016DEC7CEC8CE49DE30E94BB704B01C4
:108B50005C01A70196016EA17FA188A599A50E943D
:108B6000BB70AB01BC0195018401CE010E94CE41D6
:108B70001EAADF91CF911F910F91FF90EF90DF9090
:108B8000CF90BF90AF909F908F907F906F905F90AD
:108B90004F9008950E943E440E9411450C94404518
:108BA000109261081092600880E1E3E3FDE0DF01CC
:108BB0001D928A95E9F71092A30D1092A40D1092C0
:108BC000A50D1092A60D1092A70D1092A80D10924F
:108BD000A90D1092AA0D1092AB0D1092AC0D10922F
:108BE000AD0D1092AE0D1092AF0D1092B00D10920F
:108BF000B10D1092B20D1092B30D1092B40D1092EF
:108C0000B50D1092B60D08954F925F926F927F92BC
:108C10008F929F92AF92BF92CF92DF92EF92FF928C
:108C20000F931F93CF93DF938091320D882309F424
:108C30001FC160E080910C0E90910D0E0E94635B4D
:108C40000091210110912201D0912301C0912401B2
:108C500020E030E040E050E40E94DB6FFE01202F76
:108C6000312F4F2F5E2F0E94B47087FD01C1F0900D
:108C70006008B12CC12CD12CE12C4DE4A42E5CC099
:108C80002F2D30E0A29EF001A39EF00D1124EE598D
:108C9000F74F80819181A281B381892B8A2B8B2B05
:108CA00081F484819581A681B781892B8A2B8B2BB6
:108CB00041F480859185A285B385892B8A2B8B2BE6
:108CC000C1F1A29E4001A39E900C112482E698E07F
:108CD000880E991EF40164857585868597850E94A6
:108CE00056712B013C01F401608971898289938955
:108CF0000E9454719B01AC01C301B2010E94BB7080
:108D0000F40122A133A144A155A10E9489733B0122
:108D10004C012B2D3C2D4D2D5E2D662D772D882D54
:108D2000992D0E94B772181624F4B62CC72CD82C93
:108D3000E92CF394FFE0FF2280916108F812A0CFA4
:108D400020911D0130911E0140911F015091200181
:108D50006B2D7C2D8D2D9E2D0E9489739B01AC0166
:108D6000FE01602F712F8F2F9C2F0E94DB6F6B01F4
:108D70007C01CE01202F312F492F5C2F6C2D7D2DB2
:108D80008E2D9F2D0E94B47087FD03C08601DE2DBD
:108D9000CF2DC0902501D0902601E0902701F090C2
:108DA00028012C2D3D2D4E2D5F2DFE01602F712FA2
:108DB0008F2F9C2F0E94B77218161CF06801ED2EA1
:108DC000FC2E8090B70D9090B80DA090B90DB0908A
:108DD000BA0D2C2D3D2D4E2D5F2DC501B4010E94E5
:108DE000B7721816F4F420E037ED43EA5CE36C2D1B
:108DF0007D2D8E2D9F2D0E9489738B01D82FC92F19
:108E000028E431EE4AE75FE3C501B4010E948973AB
:108E1000FE01202F312F4F2F5E2F0E94DB6F6B0141
:108E20007C018C2D9D2DAE2DBF2D8093B70D909381
:108E3000B80DA093B90DB093BA0D6C2D7D2D8E2D6C
:108E40009F2D0E942371DC01CB0160E00E94935AA8
:108E500090930D0E80930C0E8C2D9D2DAE2DBF2D5D
:108E60008093020E9093030EA093040EB093050E10
:108E7000DF91CF911F910F91FF90EF90DF90CF90F6
:108E8000BF90AF909F908F907F906F905F904F902A
:108E9000089590916008809161089817D9F0209109
:108EA000600830E04DE410C0429FF0011124EE59FB
:108EB000F74F80859185A285B385892B8A2B8B2BD3
:108EC00009F03F5F2F5F2F70809161082813ECCF6E
:108ED000311101C0159A0C9404462F923F924F9283
:108EE0005F926F927F928F929F92AF92BF92CF923A
:108EF000DF92EF92FF920F931F93CF93DF93CDB743
:108F0000DEB7C357D1090FB6F894DEBF0FBECDBF91
:108F10002C013B014A0159013E2CF9AA0AAB212E32
:108F2000DDAACCAA209161082F5F63962FAF6397CB
:108F3000203119F463961FAE639763963FAD639734
:108F4000032F112707FD109505C00E942F5C81E0BB
:108F50000E940A158091600890E080179107A9F39C
:108F600020917F0D3091800D4091810D5091820DA7
:108F7000D2016D917D918D919C910E9489730E9487
:108F8000597323966FAF239724967FAF2497259626
:108F90008FAF259726969FAF26972091830D30910E
:108FA000840D4091850D5091860DF3016081718192
:108FB000828193810E9489730E94597327966FAFB3
:108FC000279728967FAF289729968FAF29972A96BB
:108FD0009FAF2A972091870D3091880D4091890D80
:108FE00050918A0DD4016D917D918D919C910E943B
:108FF00089730E9459732B966FAF2B972C967FAF76
:109000002C972D968FAF2D972E969FAF2E97209150
:109010008B0D30918C0D40918D0D50918E0DF50181
:1090200060817181828193810E9489730E9459734A
:109030006AAF7BAF8CAF9DAF80913F0D9091400D9B
:10904000A091410DB091420D2AAD3BAD4CAD5DAD4F
:10905000281739074A075B07C1F16091E802E62F3C
:10906000F0E0EE0FFF1FE85FF14F808191810E94D9
:10907000635B20E030E04AE253E40E94B47087FF73
:1090800024C080915F08811120C00C94D25190912E
:10909000C00095FFFCCF8093C6003196849181116A
:1090A000F6CFE3E9F6E007C09091C00095FFFCCF52
:1090B0008093C600319684918111F6CF8091C000D3
:1090C00085FFFCCF8AE08093C60080913F0D909190
:1090D000400DA091410DB091420D2AAD3BAD4CAD7C
:1090E0005DAD281B390B4A0B5B0BCA01B90157FF59
:1090F00007C090958095709561957F4F8F4F9F4FDA
:109100000E9456714B015C0120E030E848E953E4CD
:1091100060918B0D70918C0D80918D0D90918E0DC5
:109120000E9489739B01AC01C501B4010E94B77212
:1091300018166CF58AAD9BADACADBDAD80933F0DFF
:109140009093400DA093410DB093420DEDE8F6E0F1
:1091500007C09091C00095FFFCCF8093C600319668
:1091600084918111F6CFEDEAF6E007C09091C0003E
:1091700095FFFCCF8093C600319684918111F6CF84
:109180008091C00085FFFCCF8AE08093C60080916B
:109190006108EDE48E9FD0011124AE59B74FBCA3F6
:1091A000ABA3FD01E45BFF4F10822091330D3091A2
:1091B000340D4091350D5091360D2DA33EA34FA394
:1091C00058A726964CAC5DAC6EAC7FAC2697421A85
:1091D000530A640A750A77FE08C07094609450942C
:1091E0004094411C511C611C711CABA1BCA14D924F
:1091F0005D926D927C9213972091370D3091380DCE
:109200004091390D50913A0D29A73AA74BA75CA779
:109210002A968CAC9DACAEACBFAC2A97821A930A4E
:10922000A40AB50AB7FE08C0B094A09490948094A4
:10923000811C911CA11CB11CABA1BCA114968D92E8
:109240009D92AD92BC92179720913B0D30913C0DB1
:1092500040913D0D50913E0D2DA73EA74FA758AB15
:109260002E964CAD5DAD6EAD7FAD2E978DA59EA5B6
:10927000AFA5B8A9481B590B6A0B7B0B77FF07C03A
:1092800070956095509541955F4F6F4F7F4F142FAC
:10929000052F6EAB78AFABA1BCA118964C93189775
:1092A00019965C9319971A966C931A971B967C9350
:1092B000C0903F0DD090400DE090410DF090420DD8
:1092C000A0910001B09101012AAD3BAD4CAD5DAD67
:1092D0002C193D094E095F0957FF07C0509540956D
:1092E000309521953F4F4F4F5F4F0E945A7424E6AF
:1092F00030E040E050E00E94A874EBA1FCA124877C
:10930000358746875787812F902FAEA9B8AD88152E
:109310009905AA05BB0514F4D501C401821793076A
:10932000A407B50714F4DA01C901930182014816B4
:1093300059066A067B0614F48C019D01ABA1BCA101
:1093400050960D931D932D933C9353970630110522
:109350002105310510F40C94E251FD01E85BFF4F4B
:109360008091E70290E0A0E0B0E080839183A28347
:10937000B38326962CAD3DAD4EAD5FAD26978DA146
:109380009EA1AFA1B8A5281739074A075B072CF0A3
:10939000ABA1BCA190961C9204C081E0EBA1FCA102
:1093A00080A32A962CAD3DAD4EAD5FAD2A9789A521
:1093B0009AA5ABA5BCA5281739074A075B0744F453
:1093C000ABA1BCA190968C919097826090968C9363
:1093D0002E962CAD3DAD4EAD5FAD2E978DA59EA5C5
:1093E000AFA5B8A9281739074A075B0744F4ABA112
:1093F000BCA190968C919097846090968C932AADA6
:109400003BAD4CAD5DAD2C153D054E055F0544F4FF
:10941000ABA1BCA190968C919097886090968C930C
:10942000ECA9FDA98081ABA1BCA191968C934528A4
:109430004628472809F05E98EBA1FCA1848195811C
:10944000A681B781892B8A2B8B2B09F05E98EBA123
:10945000FCA180859185A285B385892B8A2B8B2BD6
:1094600009F01598EBA1FCA184859585A685B785A3
:10947000892B8A2B8B2B09F05E98ABA1BCA11C9683
:109480002D913D914D915C911F9722962CAF3DAF50
:109490004EAF5FAF2297232B242B252BD9F440907E
:1094A000530D5090540D6090550D7090560D242D15
:1094B000352D462D572DA9A9FAA9632D7A2F8F2F67
:1094C000922D0E94B47087FD0EC0432C59A86AA843
:1094D000722C09C040906B0D50906C0D60906D0D1A
:1094E00070906E0DE4CF26966CAD7DAD8EAD9FADC8
:1094F00026972DA13EA14FA158A5621B730B840B8B
:10950000950B0E94567120917F0D3091800D4091F6
:10951000810D5091820D0E94BB706DA379AB8AAB17
:109520009CAB362F272F982F8CA9432F522F692FB2
:10953000782F498B5A8B6B8B7C8B2A966CAD7DADCB
:109540008EAD9FAD2A9729A53AA54BA55CA5621BB8
:10955000730B840B950B0E9456712091830D3091F3
:10956000840D4091850D5091860D0E94BB70162F81
:10957000072F89A79EAB9801982F8EA9432F522FB2
:10958000692F782F4D8B5E8B6F8B788F2E966CADFD
:109590007DAD8EAD9FAD2E972DA53EA54FA558A9AB
:1095A000621B730B840B950B0E9456712091870DE3
:1095B0003091880D4091890D50918A0D0E94BB70A9
:1095C0006DA778AF382E292E362F272FC101432FB4
:1095D000522F692F782F498F5A8F6B8F7C8FA090D5
:1095E0000001B09001016AAD7BAD8CAD9DAD6C19F1
:1095F0007D098E099F090E94567120918B0D309133
:109600008C0D40918D0D50918E0D0E94BB706B01A1
:109610007C01B501882777FD8095982F0E945671AF
:109620009B01AC01C701B6010E94897320E030E0C4
:1096300048EC52E40E94BB70462F572F682F792FB9
:10964000DB01CA014D8F5E8F6F8F78A3EBA1FCA168
:1096500080809180A280B380F6E08F169104A104EF
:10966000B104E4F4EBA1FCA14481558166817781CA
:1096700046305105610571058CF440855185628540
:109680007385463051056105710544F4AC01BD0197
:109690007F7746A757A760AB71AB3AC05DA149A9D8
:1096A0003AA92CA9652F742F832F922F0E9434740E
:1096B0006B017C01A80139A52EA9652F702F832F7E
:1096C000922F0E9434749B01AC01C701B6010E9425
:1096D000DB6F162F072FF82EE92E5DA548AD9101FF
:1096E000652F742F832F922D0E9434749B01AC013F
:1096F000D801F7016B2F7A2F8F2F9E2F0E94DB6FDF
:109700000E94F673EBA1FCA166A777A780AB91AB93
:10971000ABA1BCA19E962D913D914D915C91D197AD
:10972000AA962CAF3DAF4EAF5FAFAA9760E070E056
:1097300080E89FE30E94BB709B01AC01642D752DF6
:10974000862D972D0E94897369A77DA789AB9CAB55
:109750009091610880916008E92FF0E0E81BF10921
:10976000EF70FF27FBABEAAB762F6DA599A98CA90B
:10977000272F362F492F582F60E074E284E799E4B1
:109780000E94BB700E9459731B018C012AA93BA93E
:10979000223031050CF44AC06901EE24D7FCE09474
:1097A000FE2CC701B6010E94567120E030E040E077
:1097B00051E40E94B47087FF39C0210138018091C3
:1097C0009F0D9091A00DA091A10DB091A20D4816F2
:1097D00059066A067B0650F5BC01CD01641975096E
:1097E00086099709660F771F881F991FA7019601A1
:1097F0000E948674CA01B9010E9454710E94597373
:10980000AB01BC01CB01BA01640D751D861D971D0E
:109810000E9454719B01AC0160E074E284E799E41A
:109820000E94BB7069A77DA789AB9CAB79A56DA58C
:1098300099A98CA9272F362F492F582FAA966CAD9E
:109840007DAD8EAD9FADAA970E9489736E966FAF66
:109850006E97A2967FAFA2972F968FAF2F97A6965F
:109860009FAFA697362F272F982FA6968FADA69736
:10987000432F522F692F782FABA1BCA192964D9305
:109880005D936D937C93959750966D917D918D919D
:109890009C9153970E9454716B017C0179A56DA531
:1098A00099A98CA9272F362F492F582FC701B60108
:1098B0000E9489730E94A1700E94287167966CAF04
:1098C0007DAF8EAF9FAF6797EBA1FCA160AF71AF8B
:1098D00082AF93AF9E012F5E3F4F3FAB2EABAE01E9
:1098E0004F5F5F4F5EA34DA38FE89DE06D969FAFE6
:1098F0008EAF6D97DE019196BAA3A9A359AF48AF79
:10990000212C312C00E81FE3EEA9FFA96191719190
:1099100081919191FFABEEABB9A5ADA5F9A9ECA9E9
:109920002B2F3A2F4F2F5E2F0E948973AB01BC0162
:10993000A8ADB9AD4D935D936D937D93B9AFA8AFCD
:10994000DB01CA01BF776B968CAF9DAFAEAFBFAFE7
:109950006B976D96AEADBFAD6D974D905D906D9070
:109960007D906D96BFAFAEAF6D97A30192016B96E0
:109970006CAD7DAD8EAD9FAD6B970E94B772181622
:10998000F4F46B962CAD3DAD4EAD5FAD6B97C3015E
:10999000B2010E94BB702B01782E692E762FC30175
:1099A000272F352D492F582F622D732D802F912F62
:1099B0000E94B47087FD03C01201072D162DEEA979
:1099C000FFA929A13AA1E217F30709F09DCF20E0F2
:1099D00030E040E85FE3622D732D802F912F0E94CD
:1099E000B47087FF4FC03E0131E1630E711C222D20
:1099F000332D402F512FADA1BEA16D917D918D9141
:109A00009C910E948973EDA1FEA161937193819352
:109A10009193FEA3EDA3E615F70549F7222D332D0B
:109A2000402F512F6E96BFAD6E97A296AFADA29705
:109A30002F96FFAD2F97A696EFADA6976B2F7A2F97
:109A40008F2F9E2F0E948973ABA1BCA192966D931C
:109A50007D938D939C93959767966CAD7DAD8EAD00
:109A60009FAD67970E945471222D332D402F512FA7
:109A70000E9489730E942871EBA1FCA160AF71AFB5
:109A800082AF93AFAA962CAD3DAD4EAD5FADAA9718
:109A9000C701B6010E94BB70162F072F382E292E42
:109AA00081149104A104B10491F5EBA1FCA184817E
:109AB0009581A681B781892B8A2B8B2B41F58085D7
:109AC0009185A285B385892B8A2B8B2B01F520915B
:109AD000630D3091640D4091650D5091660DD80174
:109AE000F1016B2F7A2F8F2F9E2F0E9489730E9476
:109AF000A170EBA0FCA0F4E4EF0EF11C0E94287111
:109B0000D7016D937D938D939C93139700C1209102
:109B1000670D3091680D4091690D50916A0DD80123
:109B2000F1016B2F702F8F2F922D0E9489730E944D
:109B3000A1700E942871EBA1FCA1EC5BFF4FFEA37A
:109B4000EDA360837183828393834090430D509093
:109B5000440D6090450D7090460D0E94547169A7A8
:109B60007AA78BA79CA7C501B4010E9456719B01DF
:109B7000AC0169A57AA58BA59CA50E948973A70154
:109B800096010E94BB704B015C01C301B2010E94AF
:109B900054719B01AC01C501B4010E94B772181643
:109BA00034F4EDA1FEA14082518262827382409022
:109BB000470D5090480D6090490D70904A0DADA131
:109BC000BEA16D917D918D919C910E9454714B012C
:109BD0005C01EBA1FCA164817581868197810E9463
:109BE00056719B01AC01C501B4010E948973A701A4
:109BF00096010E94BB704B015C01C301B2010E943F
:109C000054719B01AC01C501B4010E94B7721816D2
:109C10003CF4ADA1BEA14D925D926D927C921397E2
:109C200040904F0D5090500D6090510D7090520D1E
:109C3000EBA1FCA1EC5BFF4FFEA3EDA36081718162
:109C4000828193810E9454714B015C0122966CAD1C
:109C50007DAD8EAD9FAD22970E9456719B01AC01E8
:109C6000C501B4010E948973A70196010E94BB70CF
:109C70004B015C01C301B2010E9454719B01AC0114
:109C8000C501B4010E94B77218163CF4ADA1BEA183
:109C90004D925D926D927C92139740904B0D509037
:109CA0004C0D60904D0D70904E0DEDA1FEA16081A8
:109CB0007181828193810E9454714B015C01ABA13F
:109CC000BCA118966D917D918D919C911B970E94DE
:109CD00056719B01AC01C501B4010E948973A701B3
:109CE00096010E94BB706B017C01C301B2010E940E
:109CF00054719B01AC01C701B6010E94B7721816DE
:109D000034F4EDA1FEA14082518262827382EBA104
:109D1000FCA1EC5BFF4F60817181828193810E9485
:109D200054716B017C01B801C101272F302F492FDD
:109D3000522DC701B6010E94BB70462F572F682FC6
:109D4000792FE0964CAF5DAF6EAF7FAFE097ABA1E0
:109D5000BCA1D2964D935D936D937C93D5972DEBDB
:109D600037E346E051E4C701B6010E9489730E94BF
:109D70002371EBA1FCA1648F758F868F978F409024
:109D80005F0D5090600D6090610D7090620D20E04D
:109D900030E040E05FE3C301B2010E9489736DA32C
:109DA00079A78DA799AB29853A854B855C85A196C6
:109DB0002CAF3DAF4EAF5FAFA19780905B0D909001
:109DC0005C0DA0905D0DB0905E0D20E030E040E0B5
:109DD0005FE3C501B4010E948973162F072FF82E87
:109DE000E92EA1966CAD7DAD8EAD9FADA1979F770D
:109DF000D801F7012B2F3A2F4F2F5E2F0E94B772F9
:109E00001816B4F4B801C701272F362F492F582F41
:109E1000BDA1A9A5FDA5E9A96B2F7A2F8F2F9E2F94
:109E20000E94B47087FD04C01DA309A7FDA6E9AA7E
:109E30008D859E85AF85B889A5968CAF9DAFAEAF59
:109E4000BFAFA597C090570DD090580DE090590D19
:109E5000F0905A0D20E030E040E05FE3C701B6012A
:109E60000E948973162F072F382E292EA5966CADC8
:109E70007DAD8EAD9FADA5979F77D801F1012B2FBA
:109E80003A2F4F2F5E2F0E94B7721816B4F4B80104
:109E9000C101272F362F492F582FBDA1A9A5FDA5F8
:109EA000E9A96B2F7A2F8F2F9E2F0E94B47087FD08
:109EB00004C01DA309A73DA629AAABA1BCA19296E7
:109EC000BC91BCABEBA1FCA1F3A1FEABABA1BCA1CF
:109ED0009496BC91B8AFEBA1FCA1F5A1FEAF7CA913
:109EE0006EA9272F362F4B2F5F2FBDA1A9A5FDA54A
:109EF000E9A96B2F7A2F8F2F9E2F0E94B47087FDB8
:109F000008C02CA92DA33EA939A748AD4DA75EAD29
:109F100059AB8AA99BA902970CF443C19091B30D48
:109F20009AABA091B40D6496AFAF6497B091B50DA4
:109F30006896BFAF6897E091B60D6C96EFAF6C97DF
:109F400027E137EB41ED58E36896FFAD6897692F3D
:109F50007A2F8F2F9E2F0E94B77218160CF021C1F6
:109F60002091A30D3091A40D4091A50D5091A60D07
:109F700069817A818B819C810E94DA6F162F072F6D
:109F8000382E292E2091A70D3091A80D4091A90DB2
:109F90005091AA0D6D817E818F8198850E94DA6F24
:109FA0002F966FAF2F97A6967FAFA697AB968FAFE2
:109FB000AB97AC969FAFAC97B801C101272F362F56
:109FC000492F582FD801F1016B2F7A2F8F2F9E2FF9
:109FD0000E948973E4966CAF7DAF8EAF9FAFE4971C
:109FE0002F967FAD2F97A6966FADA697AB969FAD98
:109FF000AB97AC968FADAC97272F362F492F582FA4
:10A00000DB01FC016B2F7A2F8F2F9E2F0E9489730B
:10A010009B01AC01E4966CAD7DAD8EAD9FADE49738
:10A020000E94DB6F0E94F67362966CAF7DAF8EAFBD
:10A030009FAF6297A30192010E94B77218166CF449
:10A0400062962CAD3DAD4EAD5FAD6297C301B201DE
:10A050000E94BB708B011C0106C000E010E050E8BC
:10A06000252E6FE3362E2091AB0D3091AC0D409133
:10A07000AD0D5091AE0DA1966CAD7DAD8EAD9FAD89
:10A08000A1970E94DA6F2B013C01E89477F8A501B3
:10A090009401C301B2010E94B7721816D4F4A3014F
:10A0A0009201C501B4010E94BB704B01B82EA92ECC
:10A0B000762FC501272F392D492F582F602F712F4B
:10A0C000822D932D0E94B47087FD03C084012B2C38
:10A0D0003A2C2091AF0D3091B00D4091B10D5091BF
:10A0E000B20DA5966CAD7DAD8EAD9FADA5970E94CE
:10A0F000DA6F4B015C01E894B7F8A7019601C5013E
:10A10000B4010E94B7721816D4F4A5019401C701D6
:10A11000B6010E94BB706B01F82EE92E762FC701A5
:10A12000272F3D2D492F582F602F712F822D932DD2
:10A130000E94B47087FD03C086012F2C3E2C202F77
:10A14000312F422D532DBCA9AEA9F8ADEEAD6B2F2A
:10A150007A2F8F2F9E2F0E9489734B015C01762FDF
:10A16000272F392D4A2D5B2DBAA96496AFAD649780
:10A170006896FFAD68976C96EFAD6C976B2F7A2F52
:10A180008F2F9E2F0E94B47087FF0FC08AA86496FD
:10A190009FAC64976896AFAC68976C96BFAC6C97B1
:10A1A00004C08DA099A4ADA4B9A8482D592D6A2D3D
:10A1B0007B2DABA1BCA19A964D935D936D937C933F
:10A1C0009D97E0966CAD7DAD8EAD9FADE0979058BC
:10A1D0009B01AC010E94DB6FAA962CAD3DAD4EAD4C
:10A1E0005FADAA970E9489739B01AC016BE077ED8C
:10A1F00083E29BE30E94DA6F0E94F6738B01F82ED4
:10A20000E92E762FC701272F312F492F582F682D80
:10A21000792D8A2D9B2D0E94B47087FD03C04801C3
:10A22000AF2CBE2C482D592D6A2D7B2DEBA1FCA106
:10A2300046A357A360A771A7C701202F312F492F2D
:10A240005E2DBCA9AEA9F8ADEEAD6B2F7A2F8F2F86
:10A250009E2F0E94B470181634F081E0ABA1BCA10F
:10A26000D7968C9303C0EBA1FCA117AA81E0ABA108
:10A27000BCA1D6968C9380E1FE013196A3EABDE0A5
:10A2800001900D928A95E1F73CA92EA998AD8EAD6B
:10A29000432F522F692F782F4093B30D5093B40D55
:10A2A0006093B50D7093B60D232F352F492F582F7E
:10A2B000BDA1A9A5FDA5E9A96B2F7A2F8F2F9E2FF0
:10A2C0000E94BB706B017C017CA96EA998AD8EAD1C
:10A2D000272F362F492F582F682D792D8A2D9B2D0A
:10A2E0000E94BB70AB01BC01970186018BA19CA1B0
:10A2F0000E94CE416396BFAD6397B09361082696E6
:10A300002CAD3DAD4EAD5FAD26972093330D309310
:10A31000340D4093350D5093360D2A968CAD9DAD7E
:10A32000AEADBFAD2A978093370D9093380DA093B3
:10A33000390DB0933A0D2E962CAD3DAD4EAD5FADBF
:10A340002E9720933B0D30933C0D40933D0D509341
:10A350003E0D8AAD9BADACADBDAD80933F0D9093EE
:10A36000400DA093410DB093420D0E94CA45CD58B7
:10A37000DF4F0FB6F894DEBF0FBECDBFDF91CF9198
:10A380001F910F91FF90EF90DF90CF90BF90AF9013
:10A390009F908F907F906F905F904F903F902F9005
:10A3A0000C947B532AAD3BAD4CAD5DAD20933F0D7E
:10A3B0003093400D4093410D5093420DEDE8F6E08F
:10A3C0000C944E48CD58DF4F0FB6F894DEBF0FBE49
:10A3D000CDBFDF91CF911F910F91FF90EF90DF9054
:10A3E000CF90BF90AF909F908F907F906F905F9035
:10A3F0004F903F902F900895EF92FF920F931F93ED
:10A40000CF93DF937B018A01E90120917F0D309189
:10A41000800D4091810D5091820DFC016081718110
:10A42000828193810E9489730E945973E3E3FDE066
:10A4300060837183828393832091830D3091840D97
:10A440004091850D5091860DF70160817181828167
:10A4500093810E9489730E945973E7E3FDE0608352
:10A460007183828393832091870D3091880D409171
:10A47000890D50918A0DF8016081718182819381EB
:10A480000E9489730E945973EBE3FDE0608371833E
:10A490008283938320918B0D30918C0D40918D0D93
:10A4A00050918E0D688179818A819B810E94897388
:10A4B0000E945973EFE3FDE060837183828393838D
:10A4C0009F014BE35DE067E37DE083E39DE00E9455
:10A4D000EB591092B30D1092B40D1092B50D10926D
:10A4E000B60D1092A30D1092A40D1092A50D10920E
:10A4F000A60D1092A70D1092A80D1092A90D109202
:10A50000AA0D1092AB0D1092AC0D1092AD0D1092E1
:10A51000AE0D1092AF0D1092B00D1092B10D1092C1
:10A52000B20DDF91CF911F910F91FF90EF900895A1
:10A5300020918B0D30918C0D40918D0D50918E0D91
:10A54000FC0160817181828193810E9489730E94E4
:10A550005973EFE3FDE06083718382839383CF01BE
:10A560000C94275A80935F0808958091CD0D811136
:10A57000B5C08091CC0D8111B1C08091CB0D8111FE
:10A58000ADC008959091C00095FFFCCF8093C600A8
:10A59000319684918111F6CFE1EDF6E007C09091FC
:10A5A000C00095FFFCCF8093C60031968491811145
:10A5B000F6CF8091CD0D882349F1E0EEF6E007C09B
:10A5C0009091C00095FFFCCF8093C6003196849196
:10A5D0008111F6CF6091CE0D7091CF0D8091D00D8D
:10A5E0009091D10D0E94567120917F0D3091800D78
:10A5F0004091810D5091820D0E94BB70AB01BC0156
:10A6000022E030E08DEC95E00E9444308091CC0D4A
:10A61000882349F1E4EEF6E007C09091C00095FF71
:10A62000FCCF8093C600319684918111F6CF609162
:10A63000D20D7091D30D8091D40D9091D50D0E94C3
:10A6400056712091830D3091840D4091850D50916C
:10A65000860D0E94BB70AB01BC0122E030E08DECA6
:10A6600095E00E9444308091CB0D882349F1E8EEBB
:10A67000F6E007C09091C00095FFFCCF8093C60024
:10A68000319684918111F6CF6091D60D7091D70DDE
:10A690008091D80D9091D90D0E9456712091870D0F
:10A6A0003091880D4091890D50918A0D0E94BB70A8
:10A6B000AB01BC0122E030E08DEC95E00E9444301B
:10A6C0008091C00085FFFCCF8AE08093C600109285
:10A6D000CD0D1092CC0D1092CB0D0895EBECF6E061
:10A6E00058CF1092CD0D1092CC0D1092CB0D089535
:10A6F00080932D010895EFE6F0E0808182608083F1
:10A7000008951F920F920FB60F9211240F931F936B
:10A710002F933F934F935F936F937F938F939F9369
:10A72000AF93BF93EF93FF938091DE0D9091DF0D78
:10A73000892B09F07DC1909161088091600898177C
:10A7400071F0E09160088DE4E89FF0011124EE596A
:10A75000F74FDF01A45BBF4F81E08C9302C0E0E0C4
:10A76000F0E0F093DF0DE093DE0D309709F45AC16D
:10A77000DF01A45BBF4F81E08C931092E00D10923B
:10A78000E10D1092E20D1092E30D60AD71AD6134F8
:10A790009CE9790728F461329EE4790748F002C009
:10A7A00060E47CE9769567957695679584E007C0C7
:10A7B000613197E2790730F07695679582E0809372
:10A7C000E40D07C08093E40D6032710510F460E27F
:10A7D00070E060527109611588E07807D0F0872F2A
:10A7E0009927880F991F880F991F8451994FFC0151
:10A7F000329645915491AA27659F9001649F210D3F
:10A800003A1F06942A1F3A1F1124FC018591949146
:10A810001DC09B01369527952C7F2451354FF9019A
:10A82000859194912E5F3F4FF90145915491FB0121
:10A83000E770FF274E9F90014F9F300D5E9F300DB8
:10A84000112413E0369527951A95E1F7821B930B97
:10A8500084369105A0F4EAE8F2E006C09091C000C9
:10A8600095FFFCCF8093C60081918111F7CF4AE01C
:10A8700050E08DEC95E00E94692F84E690E0909383
:10A88000E60D8093E50DE091DE0DF091DF0D64ADF6
:10A8900075AD7093E80D6093E70D61349CE979071D
:10A8A00028F461328EE4780748F002C060E47CE965
:10A8B000769567957695679584E007C0613197E254
:10A8C000790730F07695679582E08093E40D08C0B3
:10A8D00081E08093E40D6032710510F460E270E075
:10A8E00060527109611588E07807E0F0872F992799
:10A8F000880F991F880F991F8451994FFC01329638
:10A9000025913491AA27639FA001629F410D5A1F90
:10A9100006944A1F5A1F1124FC0125913491241BCF
:10A92000350B1EC0CB01969587958C7F8451954F32
:10A93000FC01259134910296FC0145915491FB0153
:10A94000E770FF274E9FC0014F9F900D5E9F900DB7
:10A95000112443E0969587954A95E1F7281B390B1A
:10A9600024363105A0F4EAE8F2E006C09091C00078
:10A9700095FFFCCF8093C60081918111F7CF4AE00B
:10A9800050E08DEC95E00E94692F24E630E0C9018B
:10A99000A0E0B0E08093E90D9093EA0DA093EB0D59
:10A9A000B093EC0D3093890020938800E091DE0D88
:10A9B000F091DF0D80899189A289B389B695A79519
:10A9C00097958795B095A095909581959F4FAF4F9E
:10A9D000BF4F8093ED0D9093EE0DA093EF0DB093CC
:10A9E000F00D8093F10D9093F20DA093F30DB093C1
:10A9F000F40D8093F50D9093F60DA093F70DB093A1
:10AA0000F80D8093F90D9093FA0DA093FB0DB09380
:10AA1000FC0D1092DA0D1092DB0D1092DC0D1092ED
:10AA2000DD0D06C080ED97E090938900809388004B
:10AA3000E091DE0DF091DF0D309709F460C480A144
:10AA40008093FD0D80FF38C0459A8FEF80932901D8
:10AA500080912D018823A1F1329942C480E029C060
:10AA600080819181A281B381181619061A061B06EE
:10AA7000FCF48091BB0D9091BC0DA091BD0DB091E7
:10AA8000BE0D8093CE0D9093CF0DA093D00DB093BB
:10AA9000D10D81E08093CD0D80899189A289B38900
:10AAA0008093DA0D9093DB0DA093DC0DB093DD0D58
:10AAB00081E08093FE0D04C0459881E080932901D8
:10AAC0008091FD0D81FF3CC047988FEF80932A0154
:10AAD00080912D018823C1F1339907C480E02DC0F6
:10AAE000E091DE0DF091DF0D84819581A681B78123
:10AAF000181619061A061B06FCF48091BF0D9091DA
:10AB0000C00DA091C10DB091C20D8093D20D909354
:10AB1000D30DA093D40DB093D50D81E08093CC0DCF
:10AB200080899189A289B3898093DA0D9093DB0D96
:10AB3000A093DC0DB093DD0D81E08093FF0D04C088
:10AB4000479A81E080932A018091FD0D82FF3CC0ED
:10AB50002A988FEF80932B0180912D018823C1F1DA
:10AB60003499C8C380E02DC0E091DE0DF091DF0D77
:10AB700080859185A285B385181619061A061B06CD
:10AB8000FCF48091C30D9091C40DA091C50DB091BE
:10AB9000C60D8093D60D9093D70DA093D80DB0938A
:10ABA000D90D81E08093CB0D80899189A289B389E9
:10ABB0008093DA0D9093DB0DA093DC0DB093DD0D47
:10ABC00081E08093000E04C02A9A81E080932B01DB
:10ABD0008091FD0D83FF03C0289A8FEF02C0289853
:10ABE00081E080932C0120E030E081C18091C000A1
:10ABF00087FF19C0E091C60040914E0650914F0664
:10AC0000CA0101968F77992760915006709151067D
:10AC10008617970741F0DA01A253BA4FEC9390934D
:10AC20004F0680934E06E091DE0DF091DF0D80918E
:10AC3000ED0D9091EE0DA091EF0DB091F00D4081D2
:10AC4000518162817381840F951FA61FB71F809366
:10AC5000ED0D9093EE0DA093EF0DB093F00D18163F
:10AC600019061A061B0644F55F9A408951896289C4
:10AC70007389841B950BA60BB70B8093ED0D9093F6
:10AC8000EE0DA093EF0DB093F00D4091290180914E
:10AC9000BB0D9091BC0DA091BD0DB091BE0D840F68
:10ACA000911DA11DB11D8093BB0D9093BC0DA09370
:10ACB000BD0DB093BE0D5F98E091DE0DF091DF0DFC
:10ACC0008091F10D9091F20DA091F30DB091F40DE2
:10ACD0004481558166817781840F951FA61FB71F18
:10ACE0008093F10D9093F20DA093F30DB093F40DBA
:10ACF000181619061A061B0644F5469A408951890A
:10AD000062897389841B950BA60BB70B8093F10D99
:10AD10009093F20DA093F30DB093F40D40912A019E
:10AD20008091BF0D9091C00DA091C10DB091C20D49
:10AD3000840F911DA11DB11D8093BF0D9093C00D77
:10AD4000A093C10DB093C20D4698E091DE0DF09135
:10AD5000DF0D8091F50D9091F60DA091F70DB0915A
:10AD6000F80D4085518562857385840F951FA61F58
:10AD7000B71F8093F50D9093F60DA093F70DB09348
:10AD8000F80D181619061A061B0644F52B9A408969
:10AD9000518962897389841B950BA60BB70B80932D
:10ADA000F50D9093F60DA093F70DB093F80D40912B
:10ADB0002B018091C30D9091C40DA091C50DB09150
:10ADC000C60D840F911DA11DB11D8093C30D9093DD
:10ADD000C40DA093C50DB093C60D2B98E091DE0D68
:10ADE000F091DF0D8091F90D9091FA0DA091FB0D7E
:10ADF000B091FC0D4485558566857785840F951F38
:10AE0000A61FB71F8093F90D9093FA0DA093FB0D29
:10AE1000B093FC0D181619061A061B0644F5299A5C
:10AE20004089518962897389841B950BA60BB70BE6
:10AE30008093F90D9093FA0DA093FB0DB093FC0D48
:10AE400040912C018091C70D9091C80DA091C90D22
:10AE5000B091CA0D840F911DA11DB11D8093C70D26
:10AE60009093C80DA093C90DB093CA0D29988091F5
:10AE7000DA0D9091DB0DA091DC0DB091DD0D019606
:10AE8000A11DB11D8093DA0D9093DB0DA093DC0D15
:10AE9000B093DD0D4091DA0D5091DB0D6091DC0D2A
:10AEA0007091DD0D2F5F3F4FE091DE0DF091DF0DD2
:10AEB00080899189A289B389481759076A077B0756
:10AEC000B0F04091DA0D5091DB0D6091DC0D709186
:10AED000DD0DE091DE0DF091DF0D84899589A68965
:10AEE000B78984179507A607B70748F4E0C0809193
:10AEF000E40D90E0281739070CF478CEE2CF4091AA
:10AF0000E90D5091EA0D6091EB0D7091EC0D048DFF
:10AF1000158D268D378DAA27419FB12D529FC001D7
:10AF2000629F900D619F800D911D429FB00D811D0C
:10AF30009A1F519FB00D811D9A1F609FB00D811DFA
:10AF40009A1F509FB10D8A1F9A1FB6958A1F9A1F8C
:10AF5000112444AD55AD480F591F5093E80D40934F
:10AF6000E70D80AD91ADA2ADB3AD60E070E08417A8
:10AF70009507A607B70720F49093E80D8093E70D97
:10AF80006091E70D7091E80D61349CE9790728F430
:10AF900061328EE4780748F002C060E47CE976957F
:10AFA00067957695679584E007C0613197E27907E8
:10AFB00030F07695679582E08093E40D08C081E0DB
:10AFC0008093E40D6032710510F460E270E060522D
:10AFD0007109611588E07807E0F0872F9927880FBD
:10AFE000991F880F991F8451994FFC013296259122
:10AFF0003491AA27639FA001629F410D5A1F0694B6
:10B000004A1F5A1F1124FC0125913491241B350B32
:10B010001EC0CB01969587958C7F8451954FFC017E
:10B02000259134910296FC0145915491FB01E77002
:10B03000FF274E9FC0014F9F900D5E9F900D1124E2
:10B04000F3E096958795FA95E1F7281B390B24369E
:10B050003105A0F4EAE8F2E006C09091C00095FF47
:10B06000FCCF8093C60081918111F7CF4AE050E078
:10B070008DEC95E00E94692F24E630E03093890042
:10B08000209388008091E90D9091EA0DA091EB0D3D
:10B09000B091EC0D820F931FA11DB11D8093E90D9E
:10B0A0009093EA0DA093EB0DB093EC0DF3C040919B
:10B0B000DA0D5091DB0D6091DC0D7091DD0D808D0E
:10B0C000918DA28DB38D84179507A607B70708F059
:10B0D000D9C04091E00D5091E10D6091E20D709169
:10B0E000E30D048D158D268D378DAA27419FB12D37
:10B0F000529FC001629F900D619F800D911D429FE4
:10B10000B00D811D9A1F519FB00D811D9A1F609F28
:10B11000B00D811D9A1F509FB10D8A1F9A1FB695C1
:10B120008A1F9A1F11242091E70D3091E80DE05CF1
:10B13000FF4F2817390718F42081318102C0281BDE
:10B14000390B80819181A281B381A90160E070E017
:10B15000481759076A077B0708F49C0121349CE9CA
:10B16000390728F421328EE4380748F002C020E481
:10B170003CE9369527953695279584E007C021311F
:10B1800097E2390730F03695279582E08093E40DF9
:10B1900008C081E08093E40D2032310510F420E2F4
:10B1A00030E0B90160527109611588E07807E0F07C
:10B1B000872F9927880F991F880F991F8451994FBE
:10B1C000FC01329645915491AA27659F9001649F96
:10B1D000210D3A1F06942A1F3A1F1124FC014591A4
:10B1E0005491421B530B1EC0CB01969587958C7FC3
:10B1F0008451954FFC01459154910296FC01259193
:10B200003491FB01E770FF272E9FC0012F9F900D07
:10B210003E9F900D112433E0969587953A95E1F77E
:10B22000481B590B44365105A0F4EAE8F2E006C089
:10B230009091C00095FFFCCF8093C6008191811151
:10B24000F7CF4AE050E08DEC95E00E94692F44E68C
:10B2500050E050938900409388008091E00D9091D8
:10B26000E10DA091E20DB091E30D840F951FA11D9A
:10B27000B11D8093E00D9093E10DA093E20DB0938A
:10B28000E30D08C08091E50D9091E60D9093890043
:10B29000809388004091DA0D5091DB0D6091DC0DB8
:10B2A0007091DD0DE091DE0DF091DF0D80899189C7
:10B2B000A289B389481759076A077B0700F11092E2
:10B2C000DF0D1092DE0D9091610880916008981753
:10B2D000B1F0809160088F5F8F70809360080FC01D
:10B2E0008091FE0D8111BCCBE3CB8091FF0D8111CC
:10B2F000F7CB22CC8091000E811136CC61CCFF912E
:10B30000EF91BF91AF919F918F917F916F915F91DD
:10B310004F913F912F911F910F910F900FBE0F9062
:10B320001F9018953D9A3F9A229A209A569A5E9AB3
:10B33000569A5E9A0D9A159A569A5E9A3A98429A39
:10B340003B98439A3C98449A579A5F985E9A3E9AE3
:10B3500046985E9A239A2B98159A219A29985E9A74
:10B36000A1E8B0E08C918F7E8C938C9188608C9357
:10B37000E0E8F0E080818D7F808380818E7F808314
:10B3800080818F73808380818F7C80838C91887F84
:10B3900082608C9380E090E4909389008093880091
:10B3A0001092850010928400EFE6F0E080818260C8
:10B3B000808381E080932D017894089590916108B5
:10B3C00080916008981731F00E942F5C81E00E9404
:10B3D0000A15F4CF0895CF93DF93EFB7F894EC01FB
:10B3E00088819981AA81BB818093BB0D9093BC0D0C
:10B3F000A093BD0DB093BE0DEB0188819981AA8108
:10B40000BB818093BF0D9093C00DA093C10DB093ED
:10B41000C20DEA0188819981AA81BB818093C30D05
:10B420009093C40DA093C50DB093C60DE90188811A
:10B430009981AA81BB818093C70D9093C80DA09379
:10B44000C90DB093CA0DEFBFDF91CF9108952FB70B
:10B45000F894FC0180819181A281B3818093C70D12
:10B460009093C80DA093C90DB093CA0D2FBF089536
:10B470000F931F939FB7F89424E0829FF00111244B
:10B48000E554F24F00811181228133819FBFB801C1
:10B49000C9011F910F9108950E94DE595E9A5E9A2C
:10B4A000159A5E9A089580916F008D7F80936F004A
:10B4B00006C0809160088F5F8F70809360089091C4
:10B4C00061088091600898130AC01092DF0D1092F5
:10B4D000DE0D80916F00826080936F0008959091DF
:10B4E000610880916008981751F3E3CF20913601ED
:10B4F00030913701409138015091390160E070E09E
:10B500008FE793E40E94BB7060930F0E7093100E50
:10B510008093110E9093120E0895825F914FFC015B
:10B52000808190E008950F931F93CF93DF93EC01F8
:10B53000662309F461C0E3EDFFE007C09091C0000D
:10B5400095FFFCCF8093C600319684918111F6CF90
:10B550004AE050E070E08DEC95E00E944B2FEAED60
:10B56000FFE007C09091C00095FFFCCF8093C6001C
:10B57000319684918111F6CF8091C00085FFFCCF78
:10B580008AE08093C6000E94E11436C0C901880F8A
:10B59000991F880F991FFC01E850F04F6591749135
:10B5A0006C177D073CF521503109220F331F220F04
:10B5B000331FF901EA50F04F059114912850304F94
:10B5C000F90145915491FC01EA50F04F25913491D5
:10B5D000C41BD50B201B310BC29FC001C39F900D14
:10B5E000D29F900D1124641B750B0E947274600F22
:10B5F000711F13C04F5F01C041E0242F30E04D3375
:10B6000009F0C4CF2D33310531F4E6EEF0E1859138
:10B610009491BC0102C060E070E020EF3FE3261B84
:10B62000370BC901DF91CF911F910F910895CF93EF
:10B63000DF9321E030E0D901AA0FBB1FAA0FBB1F87
:10B64000FD01E850F04F659174916817790744F552
:10B6500021503109220F331F220F331FF901EA5005
:10B66000F04FC591D4912850304FF9014591549134
:10B67000FD01EA50F04F25913491FC01E41BF50BDC
:10B680002C1B3D0BE29FC001E39F900DF29F900D9C
:10B690001124641B750B0E9472746C0F7D1F0BC00C
:10B6A0002F5F3F4F2D33310509F0C5CFE6EEF0E1B6
:10B6B00085919491BC0120EF3FE3261B370BC90114
:10B6C000DF91CF9108952F923F924F925F926F92A8
:10B6D0007F928F929F92AF92BF92CF92DF92EF9222
:10B6E000FF920F931F93CF93DF938C01662351F149
:10B6F000E3EDFFE007C09091C00095FFFCCF809381
:10B70000C600319684918111F6CF4AE050E070E096
:10B710008DEC95E00E944B2FEAEEF0E107C090918E
:10B72000C00095FFFCCF8093C600319684918111B3
:10B73000F6CF8091C00085FFFCCF8AE08093C600E1
:10B740000E94E114C0EFDFE3C01BD10B41E05EC0FB
:10B750009C01220F331F220F331FF901EA50F04FD3
:10B7600065907490C615D7050CF04FC00197880FEF
:10B77000991F880F991FFC01E850F04F25903490D5
:10B780008A50904FFC0105911491F901E850F04F57
:10B7900045905490B101882777FD8095982F0E949D
:10B7A00056716B017C01BE01601B710B882777FD10
:10B7B0008095982F0E9456714B015C01B20162196D
:10B7C0007309882777FD8095982F0E9456719B01F9
:10B7D000AC01C501B4010E9489734B015C01B30146
:10B7E000601B710B882777FD8095982F0E945671FA
:10B7F0009B01AC01C501B4010E94BB709B01AC016F
:10B80000C701B6010E94DB6F17C04F5F842F90E025
:10B810004D3309F09DCFCD9759F4E8EEF0E16591F5
:10B820007491882777FD8095982F0E94567104C0E7
:10B8300060E070E080E090E0DF91CF911F910F9188
:10B84000FF90EF90DF90CF90BF90AF909F908F9040
:10B850007F906F905F904F903F902F9008952F9220
:10B860003F924F925F926F927F928F929F92AF9290
:10B87000BF92CF92DF92EF92FF920F931F93CF93DD
:10B88000DF9300D0CDB7DEB78091010E882309F495
:10B89000BFC18FB7F8941092010E8FBF60E0809106
:10B8A000080E9091090E0E94635B6B017C019B0165
:10B8B000AC016091020E7091030E8091040E909184
:10B8C000050E0E94DA6FB62EA72E182F092FA5019C
:10B8D0009801852F942FA32FB22F8093130E90934E
:10B8E000140EA093150EB093160E20E030E040E247
:10B8F00051E4D501F8016B2F7A2F8F2F9E2F0E94D4
:10B90000B77218160CF41DC120E030E040E251EC93
:10B91000D501F8016B2F7A2F8F2F9E2F0E94B470C4
:10B9200087FD0BC18091170E8111FCC020913A0157
:10B9300030913B0140913C0150913D01D501F8010E
:10B940006B2F7A2D8F2F902F0E948973762E672E62
:10B9500089839A83A301382F292F852F942FA32F12
:10B96000B22F80931C0E90931D0EA0931E0EB093C9
:10B970001F0E2091180E3091190E40911A0E509101
:10B980001B0ED501F8016B2F7A2D8F2F902F0E945F
:10B99000DB6F8B012C018090200E9090210EA090E7
:10B9A000220EB090230E282D392D4A2D5B2D602FAD
:10B9B000712F842D952D0E94B47087FF9DC0840146
:10B9C0002501802F912FA42DB52D8093180E9093D3
:10B9D000190EA0931A0EB0931B0E209136013091D0
:10B9E00037014091380150913901602F712F842D1A
:10B9F000952D0E9489734B015C01862F992DAA2DEC
:10BA0000BB2D8093240E9093250EA093260EB09309
:10BA1000270E2091280E3091290E40912A0E509128
:10BA20002B0EC701B6010E94DA6F209132013091CE
:10BA3000330140913401509135010E94897320ED0A
:10BA40003CEC4CE45DE30E9489731B012C0123E371
:10BA500033E343E75FE360912C0E70912D0E8091EC
:10BA60002E0E90912F0E0E9489739B01AC01C20192
:10BA7000B1010E94DB6F8B012C01862F912FA42D29
:10BA8000B52D80932C0E90932D0EA0932E0EB09377
:10BA90002F0EC092280ED092290EE0922A0EF0921C
:10BAA0002B0E282D392D4A2D5B2DD301F980EA80EC
:10BAB0006B2F762D8F2D9E2D0E94DB6F202F312F27
:10BAC000442D552D0E94DA6F8B017C0120E030E07F
:10BAD000A901712F9F2D0E94B47087FD3CC020E00A
:10BAE00030E04FE753E4602F712F8E2D9F2D0E9481
:10BAF000B7721816A4F528C080900F0E9090100E03
:10BB0000A090110EB090120E282D392D4A2D5B2DCC
:10BB1000602F712F842D952D0E94B77218160CF08E
:10BB200050CF4DCF1092180E1092190E10921A0E7F
:10BB300010921B0E1092170EF9CE81E08093170E13
:10BB40000AC081E08093170E00E010E08FE7E82E36
:10BB500093E4F92E04C000E010E0E12CF12C2091D8
:10BB6000080E3091090E4091300E5091310E42175F
:10BB700053071CF010920E0E11C040913E015091DF
:10BB80003F0124173507B4F7602F712F8E2D9F2D9D
:10BB90000E9423717595679560930E0E0E94882C04
:10BBA0000091320E1091330E2091340E3091350EEB
:10BBB000601B710B820B930B6838734181059105F3
:10BBC00038F10E94882C6093320E7093330E80936C
:10BBD000340E9093350E8091060E9091070E2091B1
:10BBE000360E3091370E281739078CF4209140011A
:10BBF000309141018217930754F420910A0E30913D
:10BC00000B0E821793070CF002C05A9A01C05A9883
:10BC10000F900F90DF91CF911F910F91FF90EF90B8
:10BC2000DF90CF90BF90AF909F908F907F906F905C
:10BC30005F904F903F902F9008952F923F924F9298
:10BC40005F926F927F928F929F92AF92BF92CF92AC
:10BC5000DF92EF92FF920F931F93CF93DF93C0EF8A
:10BC6000DFE3C81BD90B81E090E09C01220F331F5A
:10BC7000220F331FF901EA50F04F65907490C615FA
:10BC8000D7050CF04FC00197880F991F880F991F97
:10BC9000FC01E850F04F259034908A50904FFC0101
:10BCA00005911491F901E850F04F45905490B1017D
:10BCB000882777FD8095982F0E9456716B017C0133
:10BCC000BE01601B710B882777FD8095982F0E941D
:10BCD00056714B015C01B20162197309882777FD27
:10BCE0008095982F0E9456719B01AC01C501B4014B
:10BCF0000E9489734B015C01B301601B710B8827A3
:10BD000077FD8095982F0E9456719B01AC01C5016B
:10BD1000B4010E94BB709B01AC01C701B6010E9437
:10BD2000DB6F0FC001968D33910509F09ECFE8EED1
:10BD3000F0E165917491882777FD8095982F0E9496
:10BD40005671DF91CF911F910F91FF90EF90DF908F
:10BD5000CF90BF90AF909F908F907F906F905F90AB
:10BD60004F903F902F9008951092200E1092210E28
:10BD70001092220E1092230E20913601309137013D
:10BD8000409138015091390160E070E08FE793E411
:10BD90000E94BB7060930F0E7093100E8093110E73
:10BDA0009093120E559A529A87ED80937A00EEE79F
:10BDB000F0E010828081806880838081806480834D
:10BDC00080E888BDEEE6F0E08081846080836AEFE1
:10BDD00070E080E090E00E94C42C60E085E090E09C
:10BDE0000E94935A9093310E8093300E60E083E16D
:10BDF00091E00E94935A90933F0180933E0185E029
:10BE000090E00E94175B9093370E8093360E86E980
:10BE100090E00E94175B9093410180934001089548
:10BE2000089560E080E090E00E94935A1092020E24
:10BE30001092030E1092040E1092050E80E090E016
:10BE40000E94175B90930B0E80930A0E10920D0EBA
:10BE500010920C0E10920E0E5D9810920B0E109216
:10BE60000A0E5A9808952F923F924F925F926F92C6
:10BE70007F928F929F92AF92BF92CF92DF92EF927A
:10BE8000FF920F931F93CF93DF93CDB7DEB7E19768
:10BE90000FB6F894DEBF0FBECDBF688B798B8A8B4F
:10BEA0009B8B0E94882C6C8B7D8B8E8B9F8BEEE9FD
:10BEB000F2E006C09091C00095FFFCCF8093C600D1
:10BEC00081918111F7CF8091C00085FFFCCF8AE07E
:10BED0008093C6000E94115F8FE780930E0E4C88FE
:10BEE0005D886E887F884C865D866E867F86AFE72C
:10BEF000CA2ED12CE12CF12CBFE78B2E912CA12C3A
:10BF0000B12C8EA69FA6A8AAB9AA11E01B861A86F4
:10BF1000ECEEFEE094909FA2E4EFFEE0A490A8A6D1
:10BF2000E9EFFEE0B490B9A6E0E0FFE084908AA6D5
:10BF3000E7E0FFE094909BA6EDE0FFE0A490ACA6C4
:10BF40008091010E882309F4BBC28FB7F894109238
:10BF5000010E8FBF60E08091080E9091090E0E9443
:10BF6000635B6E837F8388879987762F6F81982F95
:10BF70008985272F362F492F582FB88DA98DEA8D07
:10BF8000FB8D6B2F7A2FCF010E94B772181644F0E9
:10BF9000BE80B88E8F80898E98849A8EA984AB8E4D
:10BFA0007E816F8198858985272F362F492F582FBD
:10BFB000ECA1602F722D832D9E2F0E94B47087FDFF
:10BFC00005C00E812F803884B984BCA2112309F4E6
:10BFD0003FC3788969899A898B89272F362F492F02
:10BFE000582FBE81AF81E885F9856B2F7A2FCF015D
:10BFF0000E94B77218160CF063C20E94882C641954
:10C00000750986099709693873418105910508F416
:10C0100057C28EA59FA5A8A9B9A98C199D09AE09DB
:10C02000BF09B595A7959795879580930E0E0E94A9
:10C03000882C6C877D878E879F874B015C018418D5
:10C040009508A608B70888A299A2AAA2BBA29888B8
:10C05000988EA988A98EBA88BA8E8B888B8EF8C2E2
:10C060000E94882C8C849D84AE84BF8468197909D1
:10C070008A099B09693873418105910508F41FC23B
:10C080000E94882C2B013C018A849B84892809F416
:10C09000FCC1DC01CB018C849D84AE84BF848819F3
:10C0A0009909AA09BB0988A099A0AAA0BBA0880EDB
:10C0B000991EAA1EBB1E28A139A14AA15BA1281B5B
:10C0C000390B4A0B5B0BCA01B901A70196010E940B
:10C0D0006274A50194010E94A8748EA59FA5A8A9C9
:10C0E000B9A9280F391F4A1F5B1F243131054105AB
:10C0F000510524F12EA73FA748AB59AB2C3E310583
:10C100004105510544F02BEE30E040E050E02EA711
:10C110003FA748AB59AB8EA59FA5A8A9B9A9803860
:10C120009105A105B105C4F0EEEFCE2ED12CE12C86
:10C13000F12CC81AD90AEA0AFB0A12C024E130E03D
:10C1400040E050E02EA73FA748AB59AB74E1C72EA3
:10C15000D12CE12CF12C04C0CEA4DFA4E8A8F9A8CE
:10C160008FA1ECEEFEE008C09091C00095FFFCCFDF
:10C170008093C600319684918111F6CF2AE030E099
:10C180004EA55FA568A979A98DEC95E00E943A2F8C
:10C1900088A5E4EFFEE008C09091C00095FFFCCFB9
:10C1A0008093C600319684918111F6CF2AE030E069
:10C1B000B701A6018DEC95E00E943A2F89A5E9EF21
:10C1C000FEE008C09091C00095FFFCCF8093C600B0
:10C1D000319684918111F6CF22E030E08CA1402F7E
:10C1E000522D632D782F8DEC95E00E9444308AA566
:10C1F000E0E0FFE008C09091C00095FFFCCF809385
:10C20000C600319684918111F6CF22E030E0F88D9E
:10C21000E98D9A8D8B8D4F2F5E2F692F782F8DECA6
:10C2200095E00E9444308091C00085FFFCCF8AE0F9
:10C230008093C6004A855B85433051050CF425C1C7
:10C24000C701B6010E94567120E030E040E850E49A
:10C250000E9489736C8F7D8F8E8F9F8F8CA1202F72
:10C26000322D432D582FB88DA98DEA8D1B8D6B2F44
:10C270007A2F8E2F912F0E94DA6F20ED3FE049E454
:10C2800050E40E94897320E030E040E05FE30E94C8
:10C2900089739B01AC016C8D7D8D8E8D9F8D0E946D
:10C2A000BB70362E072F182F9C8FC501B4010E943A
:10C2B000567120E030E04AE754E40E94BB70A62E9D
:10C2C000972E282E892E8BA5E7E0FFE008C09091DD
:10C2D000C00095FFFCCF8093C600319684918111F8
:10C2E000F6CF22E030E08C8D432D502F612F782F38
:10C2F0008DEC95E00E9444308CA5EDE0FFE008C095
:10C300009091C00095FFFCCF8093C6003196849138
:10C310008111F6CF22E030E04A2D592D622D782D83
:10C320008DEC95E00E9444308091C00085FFFCCFE9
:10C330008AE08093C6002AE939E949E15FE3EC8DA0
:10C34000632D702F812F9E2F0E948973362E072F09
:10C35000182FB92E762F272F302F412F5B2D632DCD
:10C36000702F812F9B2D0E94DB6F2A2D392D422D9E
:10C37000582D0E94BB706C8F7CA38DA39EA32A2D89
:10C38000392D422D582D632D702F812F9B2D0E940A
:10C39000897320E030E040E05EE30E948973A62EBE
:10C3A000972E282E892EE3E1FFE007C09091C00070
:10C3B00095FFFCCF8093C600319684918111F6CF12
:10C3C0008091C00085FFFCCF8AE08093C600E0E248
:10C3D000FFE007C09091C00095FFFCCF8093C6009E
:10C3E000319684918111F6CF22E030E0432D502F19
:10C3F000612F7B2D8DEC95E00E9444308091C00030
:10C4000085FFFCCF8AE08093C600E6E2FFE007C02C
:10C410009091C00095FFFCCF8093C6003196849127
:10C420008111F6CF22E030E0FC8DECA19DA18EA120
:10C430004F2F5E2F692F782F8DEC95E00E944430AE
:10C440008091C00085FFFCCF8AE08093C600ECE2BB
:10C45000FFE007C09091C00095FFFCCF8093C6001D
:10C46000319684918111F6CF22E030E04A2D592D8A
:10C47000622D782D8DEC95E00E9444308091C000B3
:10C4800085FFFCCF8AE08093C6008EA59FA5A8A952
:10C49000B9A98C0D9D1DAE1DBF1DB595A79597958E
:10C4A000879580930E0E8A859B8501969B878A8748
:10C4B000088929883A888B888CA211E001C010E095
:10C4C00020E030E040EA51E4B889A989EA89FB8993
:10C4D0006B2F7A2FCF010E94DB6F9B01AC01BE81D5
:10C4E000AF81E885F9856B2F7A2FCF010E94B77253
:10C4F000181694F4E2E3FFE007C09091C00095FFA6
:10C50000FCCF8093C600319684918111F6CF809143
:10C51000C00085FFFCCF98C00E94882C8C889D8825
:10C52000AE88BF88681979098A099B09613D7740FF
:10C530008105910508F43FC00E94882C6C8B7D8B8F
:10C540008E8B9F8BEBE5FFE007C09091C00095FFBD
:10C55000FCCF8093C600319684918111F6CF60E0C4
:10C560008091080E9091090E0E94635BAB01BC01A3
:10C5700022E030E08DEC95E00E944430E1E6FFE0FF
:10C5800007C09091C00095FFFCCF8093C600319604
:10C5900084918111F6CF60910E0E4AE050E070E078
:10C5A0008DEC95E00E944B2F8091C00085FFFCCF61
:10C5B0008AE08093C6000E94882C6A837B838C83E8
:10C5C0009D830E94882C8C849D84AE84BF84840CBF
:10C5D000951CA61CB71C2A813B814C815D812819C2
:10C5E00039094A095B09260F371F481F591F21388F
:10C5F0003F444241510590F0E5E6FFE007C09091CD
:10C60000C00095FFFCCF8093C600319684918111C4
:10C61000F6CF8091C00085FFFCCF16C0AA85BB85F0
:10C6200016970CF48DCCE2E8FFE007C09091C000B3
:10C6300095FFFCCF8093C600319684918111F6CF8F
:10C640008091C00085FFFCCF8AE08093C60015C0B2
:10C65000788969899A898B89272F362F492F582FF6
:10C66000BE81AF811885F9856B2F7A2F812F9F2F7F
:10C670000E94B47087FDF4CC22CFE1960FB6F894F7
:10C68000DEBF0FBECDBFDF91CF911F910F91FF9005
:10C69000EF90DF90CF90BF90AF909F908F907F9062
:10C6A0006F905F904F903F902F900895CF93DF93BE
:10C6B0001F92CDB7DEB789830E94115F0E94A61535
:10C6C000698181112FC0E3EDFFE007C08091C000B8
:10C6D00085FFFCCF9093C600319694919111F6CFCF
:10C6E0004AE050E070E08DEC95E00E944B2F809185
:10C6F000C00085FFFCCF8AE08093C600E7E0F1E14F
:10C7000007C09091C00095FFFCCF8093C600319682
:10C7100084918111F6CF8091C00085FFFCCF8AE023
:10C720008093C6000F90DF91CF910895CF93DF9350
:10C730001F92CDB7DEB789830E94115F0E94A615B4
:10C74000698181112FC0E3EDFFE007C08091C00037
:10C7500085FFFCCF9093C600319694919111F6CF4E
:10C760004AE050E070E08DEC95E00E944B2F809104
:10C77000C00085FFFCCF8AE08093C600E4E3F1E1CE
:10C7800007C09091C00095FFFCCF8093C600319602
:10C7900084918111F6CF8091C00085FFFCCF8AE0A3
:10C7A0008093C6000F90DF91CF9108955A980E9410
:10C7B000A615811121C0E3EDFFE007C09091C000F4
:10C7C00095FFFCCF8093C600319684918111F6CFFE
:10C7D000E1E6F1E107C09091C00095FFFCCF8093A6
:10C7E000C600319684918111F6CF8091C00085FFFB
:10C7F000FCCF8AE08093C60008951F920F920FB677
:10C800000F9211242F933F934F935F936F937F93D6
:10C810008F939F93AF93BF93EF93FF9380914201C8
:10C82000811106C080910E0E8093380E81115D9AA1
:10C830009091380E80914201891708F05D988F5FC2
:10C840008F77809342018091390E833009F443C081
:10C8500020F48130D1F0A8F50CC0853009F457C020
:10C8600008F453C0863009F454C0873009F05AC028
:10C8700052C010927B0087E480937C0080917A0004
:10C88000806480937A0081E019C020917800309113
:10C89000790080913A0E90913B0EA0913C0EB091A0
:10C8A0003D0E820F931FA11DB11D80933A0E9093F0
:10C8B0003B0EA0933C0EB0933D0E82E08093390E68
:10C8C00031C086E480937C0080917A0080648093FC
:10C8D0007A0083E0F3CF2091780030917900809145
:10C8E0003E0E90913F0EA091400EB091410E820FEE
:10C8F000931FA11DB11D80933E0E90933F0EA093F8
:10C90000400EB093410E84E0D9CF85E0D7CF86E0CA
:10C91000D5CF87E0D3CF1092390E8091420E8F5F32
:10C920008093420E8091420E803108F474C02FEF44
:10C930003FE380913A0E90913B0EA901481B590BA1
:10C94000CA015093090E4093080E40913E0E50913B
:10C950003F0E241B350B3093070E2093060E21E06B
:10C960002093010E1092420E10923A0E10923B0E3E
:10C9700010923C0E10923D0E1092430E1092440EF7
:10C980001092450E1092460E1092470E1092480ECD
:10C990001092490E10924A0E10923E0E10923F0EC7
:10C9A0001092400E1092410E20913E0130913F01B5
:10C9B000821793074CF010920D0E10920C0E80E02F
:10C9C0000E9456630E946B152091080E3091090E4B
:10C9D0008091300E9091310E821793074CF0109297
:10C9E0000D0E10920C0E80E00E9496630E946B1553
:10C9F0002091060E3091070E8091400190914101E7
:10CA00002817390744F010920B0E10920A0E0E945C
:10CA1000D6630E946B15FF91EF91BF91AF919F91EB
:10CA20008F917F916F915F914F913F912F910F90D7
:10CA30000FBE0F901F901895CF93DF93FC01148ABF
:10CA4000178A84E892E0938B828B13AA16AA92AB82
:10CA500081ABDF01A05BBF4F1C9213961C92DF01DC
:10CA6000A25BBF4F8D939C93DF01A359BF4F1C92D4
:10CA700013961C92DF01A559BF4F8D939C93DF0144
:10CA8000A857BF4F29E111962C93119714961C9229
:10CA9000DF01A357BF4F57961C92DF01A355BF4F2D
:10CAA0001C9213961C92DF01A555BF4F8D939C934A
:10CAB000DF01A853BF4F1D921D921D921C92139728
:10CAC000DF01A053BF4F1D921D921D921C92139720
:10CAD000118212821082EF01C453DF4F1882198233
:10CAE0001A821B82DF01AC52BF4F81E08C93118A06
:10CAF000108A0E94882C68577C4E8F4F9F4F688306
:10CB000079838A839B83DF91CF910895DB01FC01B8
:10CB100020E03EE24C91403229F0283009F4319374
:10CB20004C9141932F5F11962B30A1F710820895FD
:10CB30002F923F924F925F926F927F928F929F922D
:10CB4000AF92BF92CF92DF92EF92FF920F931F931B
:10CB5000CF93DF93CDB7DEB7C158D1090FB6F894A4
:10CB6000DEBF0FBECDBF8C017B01212C4A0182E0CC
:10CB7000880E911C6801E5EDCE0ED11C5801F6ED32
:10CB8000AF0EB11C8EE3482E512C4C0E5D1E82E080
:10CB9000480E511CEBE9F1E13490F3C09C85292F3C
:10CBA0002871203109F007C1F6018081813009F434
:10CBB00002C1823009F0EFC0FEC061EB72E0CE012D
:10CBC000855A9F4F0E949677B701CE01855A9F4F95
:10CBD0000E949677BE016B587F4FCE01855A9F4FBA
:10CBE0000E94967761EB72E0CE01855A9F4F0E94BA
:10CBF000967721961FAE219724961FAE249784E83E
:10CC000092E09FAF8EAF21E0AE014B585F4FB40171
:10CC1000C2010E947B36811139C0F60180818111E9
:10CC200035C0832DEBE9F1E108C09091C00095FF7C
:10CC3000FCCF8093C600319684918111F6CFA3EB8F
:10CC4000B2E006C09091C00095FFFCCF8093C60073
:10CC50008D918111F7CF8091C00085FFFCCF8AE0D4
:10CC60008093C600DE01AB58BF4F06C09091C00054
:10CC700095FFFCCF8093C6008D918111F7CF8091F5
:10CC8000C00085FFFCCF8AE08093C6008BE1FE01E7
:10CC9000E05CFF4FDE01939601900D928A95E1F7DB
:10CCA00084E892E09AA389A3AE014F5D5F4FBE0175
:10CCB000655A7F4FC8010E949865CE0181960E94F7
:10CCC0000F2CCE01CE960E940F2C5BC0853E09F43E
:10CCD00058C08E3209F455C08F3509F452C093FD07
:10CCE00050C081E0203109F080E0F8018787811190
:10CCF00008C08985873409F044C08A858E3709F4D5
:10CD000040C03801F3E06F0E711CBE016F5F7F4FB2
:10CD1000C3010E948665F601808181111EC0D70182
:10CD200006C09091C00095FFFCCF8093C6008D9106
:10CD30008111F7CFD30106C09091C00095FFFCCFC1
:10CD40008093C6008D918111F7CF8091C00085FF3F
:10CD5000FCCF8AE08093C60014C0813039F4F5011D
:10CD6000808191810196918380830BC0823049F448
:10CD7000222D30E0F5018081918128173907F1F0EB
:10CD80002394BE016F5F7F4FC4010E94E9321816E1
:10CD90000CF404CF13C0BE016F5F7F4FCE018B58E0
:10CDA0009F4F0E9486656C961FAE6C97F70180813D
:10CDB00081110ACF02CF8981811188CFCF57DF4FF0
:10CDC0000FB6F894DEBF0FBECDBFDF91CF911F919C
:10CDD0000F91FF90EF90DF90CF90BF90AF909F901A
:10CDE0008F907F906F905F904F903F902F9008951D
:10CDF000EF92FF920F931F93CF93DF93CDB7DEB7E0
:10CE00006D970FB6F894DEBF0FBECDBF8C01FC014D
:10CE1000EB52FF4F10827C0184E1E80EF11C40E0F0
:10CE200050E0BA01C7010E945C338BE1F701DE01DB
:10CE3000139601900D928A95E1F784E892E09A8327
:10CE40008983AE014F5F5F4F6DE972E0C8010E94B8
:10CE50009865CE0101960E940F2C6D960FB6F8943E
:10CE6000DEBF0FBECDBFDF91CF911F910F91FF901D
:10CE7000EF900895EF92FF920F931F93CF93DF935C
:10CE8000EC011A828F89882321F0CE0144960E94FA
:10CE900043347E0188E8E80EF11C4FE160E0C701F1
:10CEA0000E949A6E81111FC0EBE9F1E107C09091D9
:10CEB000C00095FFFCCF8093C6003196849181110C
:10CEC000F6CFE1EAF1E107C09091C00095FFFCCFF9
:10CED0008093C600319684918111F6CF8091C00075
:10CEE00085FFFCCF76C08E0103571F4F41E0B7018D
:10CEF000C8010E94783C811126C040E0B701C801FA
:10CF00000E94783C81111FC0EEEAF1E107C09091C8
:10CF1000C00095FFFCCF8093C600319684918111AB
:10CF2000F6CFE5EBF1E107C09091C00095FFFCCF93
:10CF30008093C600319684918111F6CF8091C00014
:10CF400085FFFCCF46C0B801CE0144960E94563101
:10CF500081111FC0EEEAF1E107C09091C00095FF7A
:10CF6000FCCF8093C600319684918111F6CFE8EC16
:10CF7000F1E107C09091C00095FFFCCF8093C600FF
:10CF8000319684918111F6CF8091C00085FFFCCF4E
:10CF900020C081E08A83EBE9F1E107C09091C000F5
:10CFA00095FFFCCF8093C600319684918111F6CF16
:10CFB000E8EDF1E107C09091C00095FFFCCF8093B0
:10CFC000C600319684918111F6CF8091C00085FF13
:10CFD000FCCF8AE08093C6008BE1FE017496DE01EF
:10CFE000D39601900D928A95E1F7CE01429698ABC7
:10CFF0008FA7DF91CF911F910F91FF90EF90089530
:10D00000FC01118212820895FC012281222311F079
:10D0100021E021830895FC012181211111820895CD
:10D020002F923F924F925F926F927F928F929F9238
:10D03000AF92BF92CF92DF92EF92FF920F931F9326
:10D04000CF93DF93CDB7DEB7AA970FB6F894DEBFC4
:10D050000FBECDBF7C016B01342EFC018281882381
:10D0600009F4B4C14701FDEA8F0E911CC4010E946E
:10D070004334F70111821B821E8284E892E09A8376
:10D080008983C701429690AB87A7F60180818F32D2
:10D0900009F08CC06FE270E0C6010E94A1778C019C
:10D0A0000F5F1F4F9AE0292E44244394512C4C0EBD
:10D0B0005D1E77C06FE270E0C8010E94A1775C013D
:10D0C000009709F47BC00817190708F077C03C01E6
:10D0D000601A710AA301B801CE014E960E94C17771
:10D0E000EEE1F0E0EC0FFD1FE60DF71D10828E0162
:10D0F000025E1F4FF80106C09091C00095FFFCCF63
:10D100008093C60081918111F7CF8091C00085FF87
:10D11000FCCF2092C600F70167A570A961157105C3
:10D1200019F06E5F7F4F02C060E070E021E0AE0159
:10D13000425E5F4FCE0103960E947B3681112BC069
:10D14000E3EEF1E107C09091C00095FFFCCF809322
:10D15000C600319684918111F6CF06C09091C0002F
:10D1600095FFFCCF8093C600F80181918F0181115A
:10D17000F5CFE7EFF1E107C09091C00095FFFCCF3C
:10D180008093C600319684918111F6CF8091C000C2
:10D1900085FFFCCF14C1F70150AA47A685010F5F98
:10D1A0001F4F0115110509F085CF05C0C701C196B4
:10D1B000F70190AB87A7BC2CAD2C02C0B02EA12EDE
:10D1C000F70167A570A9332009F49FC061157105A7
:10D1D00019F06E5F7F4F02C060E070E021E04B2DE0
:10D1E0005A2DC4010E947B36882309F463C0F701DD
:10D1F000E853FF4FD701A355BF4F51960D911D9195
:10D200002D913C9154970083118322833383E9EF5E
:10D21000F1E107C09091C00095FFFCCF8093C6005C
:10D22000319684918111F6CFEB2DFA2D06C09091A5
:10D23000C00095FFFCCF8093C60081918111F7CF8C
:10D24000E6E0F2E107C09091C00095FFFCCF80932B
:10D25000C600319684918111F6CFF701E853FF4F54
:10D2600040815181628173812AE030E08DEC95E04C
:10D270000E94272F8091C00085FFFCCF8AE0809319
:10D28000C600F701E053FF4F108211821282138211
:10D29000EDE0F2E107C09091C00095FFFCCF8093D4
:10D2A000C600319684918111F6CF8091C00085FF30
:10D2B000FCCF85C0EBE1F2E107C09091C00095FF83
:10D2C000FCCF8093C600319684918111F6CFEB2D6F
:10D2D000FA2D06C09091C00095FFFCCF8093C60048
:10D2E00081918111F7CFEFE2F2E107C09091C00088
:10D2F00095FFFCCF8093C600319684918111F6CFC3
:10D300008091C00085FFFCCF5AC06115710519F0EE
:10D310006E5F7F4F02C060E070E026E54B2D5A2D16
:10D32000C4010E947B3681112BC0E1E3F2E107C00A
:10D330009091C00095FFFCCF8093C60031968491F8
:10D340008111F6CFEB2DFA2D06C09091C00095FF0C
:10D35000FCCF8093C60081918111F7CFE5E4F2E123
:10D3600007C09091C00095FFFCCF8093C600319616
:10D3700084918111F6CF8091C00085FFFCCF1FC042
:10D3800081E0F7018083E7E4F2E107C09091C000FB
:10D3900095FFFCCF8093C600319684918111F6CF22
:10D3A000F60106C09091C00095FFFCCF8093C600A7
:10D3B00081918111F7CF8091C00085FFFCCF8AE079
:10D3C0008093C600CE0101960E940F2CAA960FB63C
:10D3D000F894DEBF0FBECDBFDF91CF911F910F91AB
:10D3E000FF90EF90DF90CF90BF90AF909F908F9085
:10D3F0007F906F905F904F903F902F9008955F9235
:10D400006F927F928F929F92AF92BF92CF92DF9254
:10D41000EF92FF920F931F93CF93DF93CDB7DEB7B9
:10D42000AA970FB6F894DEBF0FBECDBF8C016B017B
:10D43000FC018281882309F408C1C80183559F4FEC
:10D440000E944334F80111821B821E8284E892E01C
:10D450009A838983C801429690AB87A7F6018081A1
:10D460008F3209F08EC06FE270E0C6010E94A17792
:10D4700001967C014AE0542E66246394712C6C0E54
:10D480007D1E7AC06FE270E0C7010E94A1775C0147
:10D49000009709F47CC0E816F90608F078C04C0142
:10D4A0008E189F08A401B701CE014E960E94C17745
:10D4B000EEE1F0E0EC0FFD1FE80DF91D10823EE1FA
:10D4C000E32EF12CEC0EFD1EF70106C09091C0007A
:10D4D00095FFFCCF8093C60081918111F7CF809199
:10D4E000C00085FFFCCF5092C600F80167A570A967
:10D4F0006115710519F06E5F7F4F02C060E070E04A
:10D5000021E0AE01425E5F4FCE0103960E947B3662
:10D5100081112BC0E9E5F2E107C09091C00095FFB1
:10D52000FCCF8093C600319684918111F6CF06C05E
:10D530009091C00095FFFCCF8093C600F7018191C8
:10D540007F018111F5CFEDE6F2E107C09091C000B7
:10D5500095FFFCCF8093C600319684918111F6CF60
:10D560008091C00085FFFCCF69C0F80170AA67A652
:10D570007501FFEFEF1AFF0AE114F10409F082CF01
:10D5800005C0C801C196F80190AB87A77601F801E4
:10D5900087A590A9009711F0029602C080E090E064
:10D5A000B7010E943837882301F1EFE6F2E107C0A6
:10D5B0009091C00095FFFCCF8093C6003196849176
:10D5C0008111F6CFF70106C09091C00095FFFCCF06
:10D5D0008093C60081918111F7CFF801E053FF4F8E
:10D5E00010821182128213822CC0EDE7F2E107C093
:10D5F0009091C00095FFFCCF8093C6003196849136
:10D600008111F6CFF70106C09091C00095FFFCCFC5
:10D610008093C60081918111F7CFE5E9F2E107C05F
:10D620009091C00095FFFCCF8093C6003196849105
:10D630008111F6CF8091C00085FFFCCF8AE08093F6
:10D64000C600CE0101960E940F2CAA960FB6F89440
:10D65000DEBF0FBECDBFDF91CF911F910F91FF9025
:10D66000EF90DF90CF90BF90AF909F908F907F9082
:10D670006F905F900895CF93DF93EC018A818823A8
:10D68000C1F1E7E9F2E107C09091C00095FFFCCF3E
:10D690008093C600319684918111F6CFFE01E0534C
:10D6A000FF4F40815181628173812AE030E08DEC2F
:10D6B00095E00E94272FE9EAF2E107C09091C000AF
:10D6C00095FFFCCF8093C600319684918111F6CFEF
:10D6D000C853DF4F488159816A817B812AE030E05D
:10D6E0008DEC95E00E94272F8091C00085FFFCCF34
:10D6F00011C0EBEAF2E107C09091C00095FFFCCFAA
:10D700008093C600319684918111F6CF8091C0003C
:10D7100085FFFCCF8AE08093C600DF91CF9108950A
:10D72000CF92DF92EF92FF920F931F93CF93DF93ED
:10D730007C01EB01EC2FFD2FDF010D900020E9F7BC
:10D740008D01015011090E1B1F0BF701E355FF4F0F
:10D7500010826EE470E0CE010E94A1776C01009708
:10D7600029F4F8013197EC0FFD1F0DC060E270E065
:10D770000E94A177EC0121966AE270E0C6010E9446
:10D78000A177FC0131978DE081838AE08283138247
:10D79000BE01C70185559F4F0E94FC38F701E35534
:10D7A000FF4F8081882309F1EEEAF1E107C09091F3
:10D7B000C00095FFFCCF8093C60031968491811103
:10D7C000F6CFEBEBF2E107C09091C00095FFFCCFE4
:10D7D0008093C600319684918111F6CF8091C0006C
:10D7E00085FFFCCF8AE08093C600DF91CF911F9127
:10D7F0000F91FF90EF90DF90CF9008953F924F925E
:10D800005F926F927F928F929F92AF92BF92CF92D0
:10D81000DF92EF92FF920F931F93CF93DF93CDB7D9
:10D82000DEB7CC55D1090FB6F894DEBF0FBECDBF21
:10D830008C01662349F0F801EC52FF4F1082F80189
:10D840008281811118C030C0FC01EC52FF4F8081F1
:10D85000882309F4AEC0F801E453FF4FC080D180A3
:10D86000E280F3800E94882CC616D706E806F906E7
:10D8700008F49FC0E0CFF80181898F9380898F934E
:10D8800086EC92E09F938F937E01FFE3EF0EF11CF5
:10D89000FF92EF920E94EA770F900F900F900F90F7
:10D8A0000F900F90670110C0C8010E943A67F801FD
:10D8B00082818111E0CF7DC0F701808190E00E94DC
:10D8C0006077F70181937F01F60101900020E9F76D
:10D8D0003197EC19FD09C7018C199D098E179F0717
:10D8E0005CF33801F4E16F0E711C40E050E0BA01C6
:10D8F000C3010E945C33312CEE24E394F12CEC0E36
:10D90000FD1E5E018FE3A80EB11C7FEC472E72E076
:10D91000572E4E01E1E28E0E911C37C0F601808138
:10D9200090E00E946077F60181936F01F70101900A
:10D930000020E9F73197EE19FF09C6018E199F09FA
:10D940008E179F075CF38A858E37F9F045E050E02B
:10D95000B501C7010E94B3770097B9F4BF92AF92A7
:10D960005F924F929F928F920E94EA77C4010E9429
:10D970009B0D86ED92E00E949B0D0F900F900F90F3
:10D980000F900F900F9033243394B701C3010E947E
:10D99000E932181614F46701C9CF311004C08FEFB3
:10D9A0009FEFF80104C0F801808991890196918B5D
:10D9B000808BC45ADF4F0FB6F894DEBF0FBECDBFC9
:10D9C000DF91CF911F910F91FF90EF90DF90CF905B
:10D9D000BF90AF909F908F907F906F905F904F908F
:10D9E0003F9008950F931F93CF93DF938C01EC0129
:10D9F000C355DF4FCE010E94F733CE010E9443345E
:10DA0000F8011082DF91CF911F910F910895CF936C
:10DA1000DF93EC010E94DE590E94535A19828AED6D
:10DA200092E00E949B0D8091320D8823A1F110920B
:10DA3000320D6091E802E62FF0E0EE0FFF1FE45F89
:10DA4000F14F808191810E94635B2091210130918F
:10DA5000220140912301509124010E94B7721816AF
:10DA6000D4F46091E802C62FD0E080E090E00E94FC
:10DA7000935AFE01EE0FFF1FE45FF14F9183808305
:10DA8000FE01EE0FFF1FEE0FFF1FEE5FF14F108242
:10DA9000118212821382DF91CF910895EF92FF924B
:10DAA0000F931F93CF93DF937C01EB018A01060F45
:10DAB000171F09C06991D701ED91FC910190F08188
:10DAC000E02DC7010995C017D107A1F7DF91CF91CC
:10DAD0001F910F91FF90EF9008958FEF8EBD0DB4C1
:10DAE00007FEFDCF8EB508958EBD0DB407FEFDCFA8
:10DAF000089561E0FC0180810C94CC2DFC014281F1
:10DB0000242F30E03595279520652CBD40FD03C0BE
:10DB100021E0463009F420E02DBD60E0FC01808169
:10DB20000C94CC2DCF92DF92EF92FF920F931F9324
:10DB3000CF93DF93EC018B017A010E94882C6B015B
:10DB400009C00E94882C6C197D096D32714010F05B
:10DB500081E108C00E946D6D8B838F3F91F38E3FF2
:10DB600019F08FE0898328C0E114F104E1F081E02D
:10DB7000E81AF1088FEF8EBDF8012FEF06C00DB443
:10DB800007FEFDCF8EB581932EBDCF01801B910B7B
:10DB90008E159F05A0F30DB407FEFDCF8EB5F801DD
:10DBA000EE0DFF1D80830E946D6D0E946D6DCE0194
:10DBB0000E94796D81E004C0CE010E94796D80E001
:10DBC000DF91CF911F910F91FF90EF90DF90CF9059
:10DBD00008950F931F93CF93DF938B010E94882C9E
:10DBE000EB0107C00E94882C6C1B7D0B601771072E
:10DBF00030F40E946D6D8F3FA9F781E001C080E095
:10DC0000DF91CF911F910F910895CF92DF92FF92F4
:10DC10000F931F93CF93DF9300D000D0CDB7DEB723
:10DC20008C01F62E29833A834B835C830E947E6DA0
:10DC30006CE271E0C8010E94E96D8F2D80640E9442
:10DC4000746D68E1C62ED12C5C814B813A812981AB
:10DC5000DA01C9010C2C04C0B695A7959795879554
:10DC60000A94D2F729833A834B835C830E94746DB4
:10DC700068E0C61AD10829813A814B815C8188EF1E
:10DC8000C8168FEFD80621F7FF2029F098E0F91683
:10DC900021F08FEF03C085E901C087E80E94746D11
:10DCA000ECE0FE1202C00E946D6DF12C0E946D6DC1
:10DCB000F801838387FF05C0FFEFFF1611F0F3948F
:10DCC000F5CF0F900F900F900F90DF91CF911F9194
:10DCD0000F91FF90DF90CF9008950F931F93CF93F4
:10DCE000DF93EC0189018C81833039F0B9E0440F76
:10DCF000551F661F771FBA95D1F79A01AB0161E1F5
:10DD0000CE010E94056E81110AC040E052E0B801C8
:10DD1000CE01DF91CF911F910F910C94926D84E011
:10DD20008983CE010E94796D80E0DF91CF911F91B0
:10DD30000F910895BF92CF92DF92EF92FF920F93CF
:10DD40001F93CF93DF93EC01B62E1C821982488378
:10DD50000E94882C8B0161E088810E94B02DCE0149
:10DD60000E94796D60E086E00E94B02D61E085E060
:10DD70000E94B02D61E087E00E94B02D61E084E058
:10DD80000E94B02D61E084E00E94CC2D85E08A8362
:10DD900082E58CBD1DBC2AE0F22E8FEF0E94746DCF
:10DDA000FA94D9F709C00E94882C601B710B613D61
:10DDB000774010F081E058C020E030E0A90160E039
:10DDC000CE010E94056EF82E8B8381E0F812EBCF16
:10DDD0002AEA31E040E050E068E0CE010E94056EA2
:10DDE00082FF02C0FC820DC094E0F92E0E946D6D8E
:10DDF0008B83FA94D9F78A3A11F082E035C082E039
:10DE00008C838C81823031F4C12CD12CE12C80E4C4
:10DE1000F82E0DC0C12CD12C760109C00E94882C8F
:10DE2000601B710B613D774010F08AE01DC020E05F
:10DE300030E0A90167E3CE010E94056EA7019601BB
:10DE400069E2CE010E94056E8B838111E7CF8C8140
:10DE50008230C9F420E030E0A9016AE3CE010E94DB
:10DE6000056E882319F088E0898319C00E946D6DC2
:10DE7000807C803C11F483E08C830E946D6D0E9455
:10DE80006D6D0E946D6DCE010E94796D86E08B15DF
:10DE900018F488E1898306C0BA8281E004C0CE010B
:10DEA0000E94796D80E0DF91CF911F910F91FF90DB
:10DEB000EF90DF90CF90BF900895CF93DF93EC0168
:10DEC0006EBD20E030E00DB407FEFDCFFA01E20F99
:10DED000F31F80818EBD0DB407FEFDCF81818EBD05
:10DEE0002E5F3F4F211582E0380769F70DB407FE1A
:10DEF000FDCF8FEF0E94746D8FEF0E94746D0E94B2
:10DF00006D6D8B838F71853039F083E18983CE010C
:10DF10000E94796D80E001C081E0DF91CF9108958A
:10DF20000F931F93CF93DF93EC0189018C81833092
:10DF300039F0E9E0440F551F661F771FEA95D1F7C6
:10DF40009A01AB0168E1CE010E94056E882311F0B1
:10DF500086E029C0A8016EEFCE010E945D6F882384
:10DF6000B9F068E572E0CE010E94E96D811102C04E
:10DF700087E119C020E030E0A9016DE0CE010E94E8
:10DF8000056E81110FC00E946D6D81110BC005C01F
:10DF9000CE010E94796D80E008C0CE010E94796DAB
:10DFA00081E003C086E18983F3CFDF91CF911F9198
:10DFB0000F9108955058BB27AA270ED076C23FD2A2
:10DFC00030F044D220F031F49F3F11F41EF40FC220
:10DFD0000EF4E095E7FBDCC1E92F89D280F3BA1794
:10DFE000620773078407950718F071F49EF5B8C2AD
:10DFF0000EF4E0950B2EBA2FA02D0B01B901900164
:10E000000C01CA01A0011124FF27591B99F0593FA7
:10E0100050F4503E68F11A16F040A22F232F342FEF
:10E020004427585FF3CF469537952795A795F0403D
:10E030005395C9F77EF41F16BA0B620B730B840B52
:10E04000BAF09150A1F0FF0FBB1F661F771F881F0A
:10E05000C2F70EC0BA0F621F731F841F48F4879562
:10E0600077956795B795F7959E3F08F0B3CF939551
:10E07000880F08F09927EE0F979587950895DFD1BF
:10E0800058F080E891E009F49EEFE0D128F040E8F4
:10E0900051E059F45EEF09C0AAC162C2E92FE078ED
:10E0A00026D268F3092E052AC1F326173707480739
:10E0B000590738F00E2E07F8E02569F0E025E064F6
:10E0C0000AC0EF6307F8009407FADB01B9019D016C
:10E0D000DC01CA01AD01EF935DD0E7D10AD05F91B9
:10E0E000552331F02BED3FE049E450FD49EC63CF7F
:10E0F0000895DF93DD27B92FBF7740E85FE3161659
:10E10000170648075B0710F4D92F96D29F938F9379
:10E110007F936F93A9D3ECE7F0E06CD1C6D12F9138
:10E120003F914F915F9101D3DD2349F09058A2EACE
:10E130002AED3FE049EC5FE3D0785D274DDFDF91CA
:10E14000B4C1F7D180F09F3740F491110EF409C2A9
:10E1500060E070E080E89FE3089526F01B16611DE3
:10E16000711D811D1BC135C1EFD008F481E00895F8
:10E1700075D1E395ABC10CD098C168D140F05FD1A7
:10E1800030F021F45F3F19F003C15111EAC12FC1F2
:10E19000AED198F39923C9F35523B1F3951B550BD1
:10E1A000BB27AA2762177307840738F09F5F5F4F6A
:10E1B000220F331F441FAA1FA9F333D00E2E3AF0AB
:10E1C000E0E830D091505040E695001CCAF729D0C5
:10E1D000FE2F27D0660F771F881FBB1F2617370714
:10E1E0004807AB07B0E809F0BB0B802DBF01FF2744
:10E1F00093585F4F2AF09E3F510568F0C9C0B1C1E6
:10E200005F3FECF3983EDCF3869577956795B7957D
:10E21000F7959F5FC9F7880F911D9695879597F998
:10E220000895E1E0660F771F881FBB1F6217730711
:10E230008407BA0720F0621B730B840BBA0BEE1F26
:10E2400088F7E095089504D06894B1118AC10895C3
:10E2500056D188F09F5790F0B92F9927B751A0F069
:10E26000D1F0660F771F881F991F1AF0BA95C9F76A
:10E2700012C0B13081F074D1B1E0089571C1672F3F
:10E28000782F8827B85F39F0B93FCCF3869577951A
:10E290006795B395D9F73EF4909580957095619503
:10E2A0007F4F8F4F9F4F0895E89409C097FB3EF42E
:10E2B00090958095709561957F4F8F4F9F4F9923D3
:10E2C000A9F0F92F96E9BB279395F6958795779551
:10E2D0006795B795F111F8CFFAF4BB0F11F460FF11
:10E2E0001BC06F5F7F4F8F4F9F4F16C0882311F069
:10E2F00096E911C0772321F09EE8872F762F05C07D
:10E30000662371F096E8862F70E060E02AF09A9517
:10E31000660F771F881FDAF7880F9695879597F90C
:10E32000089507D180F09F3740F491110EF019C184
:10E3300060E070E080E89FEB089526F41B16611DF5
:10E34000711D811D2BC045C0990F0008550FAA0BE8
:10E35000E0E8FEEF16161706E807F907C0F01216F8
:10E360001306E407F50798F0621B730B840B950BFB
:10E3700039F40A2661F0232B242B252B21F4089550
:10E380000A2609F4A140A6958FEF811D811D0895ED
:10E3900097F99F6780E870E060E00895882371F442
:10E3A000772321F09850872B762F07C0662311F42E
:10E3B00099270DC09051862B70E060E02AF09A9565
:10E3C000660F771F881FDAF7880F9695879597F95C
:10E3D00008959F3F31F0915020F487957795679588
:10E3E000B795880F911D9695879597F908959FEF9A
:10E3F00080EC0895DF93CF931F930F93FF92EF92DA
:10E40000DF927B018C01689405C0DA2EEF018DD17B
:10E41000FE01E894A5912591359145915591AEF372
:10E42000EF01DADDFE019701A801DA9479F7DF90B8
:10E43000EF90FF900F911F91CF91DF9108950024ED
:10E440000A941616170618060906089500240A9459
:10E4500012161306140605060895C9CF50D0E8F326
:10E46000E894E0E0BB279F57F0F02AED3FE049EC4D
:10E4700006C0EE0FBB0F661F771F881F28F0B23A49
:10E4800062077307840728F0B25A620B730B840B80
:10E49000E3959A9572F7803830F49A95BB0F661F12
:10E4A000771F881FD2F7904896CF092E0394000C4F
:10E4B00011F4882352F0BB0F40F4BF2B11F460FF1E
:10E4C00004C06F5F7F4F8F4F9F4F0895EF93E0FF22
:10E4D00006C0A2EA2AED3FE049EC5FEB7DDDE5DF17
:10E4E0000F90039401FC9058E9EAF0E0C7C157FD92
:10E4F0009058440F551F59F05F3F71F04795880FB2
:10E5000097FB991F61F09F3F79F087950895121648
:10E5100013061406551FF2CF4695F1DF08C01616F4
:10E5200017061806991FF1CF8695710561050894A5
:10E530000895E5DFA0F0BEE7B91788F4BB279F3840
:10E5400060F41616B11D672F782F8827985FF7CFD4
:10E55000869577956795B11D93959639C8F308957B
:10E56000E894BB2766277727CB0197F90895ECDE5F
:10E5700008F48FEF089563DF19F068DF09F037CFF3
:10E5800007CFB901CA0125CF9F775F77B0DF98F336
:10E590009923B9F35523B9F3FF27951758F4E52FBD
:10E5A000E91BED3070F75E3B10F0F1E41CC09034D5
:10E5B000E0F40AC0E92FE51BED3028F79E3B10F090
:10E5C000F1E411C0503488F4F9EA88232AF09A95CE
:10E5D000660F771F881FDAF744232AF05A95220F17
:10E5E000331F441FDAF79F1B5F1BFF931F930F938B
:10E5F000FF92EF9279018A01BB27AB2F9B01AC01FF
:10E6000096D09701A801BF937B018C01AA27BA2F4E
:10E61000B901CA018CD0AF919701A801EF90FF908A
:10E620000F911F91D9DC41DFE1D04F9140FF089558
:10E63000552747FD509509C09B01AC0160E070E093
:10E6400080E89FE398CDA4CEC4CE59DFE8F39923A8
:10E65000D9F3940F511DBBF39150504094F059F0F1
:10E66000882332F0660F771F881F91505040C1F702
:10E670009E3F510544F7880F911D9695879597F910
:10E6800008955F3FACF0983E9CF0BB278695779548
:10E690006795B79508F4B1609395C1F7BB0F58F72C
:10E6A00011F460FFE8CF6F5F7F4F8F4F9F4FE3CF35
:10E6B00058CF25DF58F19E5758F19851A0F0E9F056
:10E6C000983020F5092E9927660F771F881F991F0C
:10E6D0000A94D1F712C0062E672F782F8827985FEB
:10E6E00011F4000C07C0993FB4F3869577956795B0
:10E6F0009395D9F7611D711D811D3EF4909580950C
:10E70000709561957F4F8F4F9F4F0895689429CFE3
:10E7100027CF0BD0CACE93DE28F098DE18F09523D1
:10E7200009F036CE64CE11241CCFE1DEA0F3959F14
:10E73000D1F3950F50E0551F629FF001729FBB27E8
:10E74000F00DB11D639FAA27F00DB11DAA1F649F94
:10E750006627B00DA11D661F829F2227B00DA11D47
:10E76000621F739FB00DA11D621F839FA00D611DCD
:10E77000221F749F3327A00D611D231F849F600DEE
:10E78000211D822F762F6A2F11249F5750408AF027
:10E79000E1F088234AF0EE0FFF1FBB1F661F771FB3
:10E7A000881F91505040A9F79E3F510570F0F0CD61
:10E7B000D8CE5F3FECF3983EDCF38695779567956E
:10E7C000B795F795E7959F5FC1F7FE2B880F911DD1
:10E7D0009695879597F908959F9340DE0F9007FCD3
:10E7E000EE5F74CE11F40EF402CEF3CD88DED0F3DA
:10E7F0009923D9F3CEF39F57550B87FF38D00024C8
:10E80000A0E640EA900180585695979528F4805CE0
:10E81000660F771F881F20F026173707480730F448
:10E82000621B730B840B202931294A2BA695179460
:10E830000794202531254A2758F7660F771F881F30
:10E8400020F026173707480730F4620B730B840B50
:10E85000200D311D411DA09581F7B901842F9158DC
:10E86000880F9695879508959B01AC0152CF9150E2
:10E870005040660F771F881FD2F708959F938F939C
:10E880007F936F93FF93EF939B01AC0142DFEF9176
:10E89000FF91B0DD2F913F914F915F913ACF0E9450
:10E8A000C474A59F900DB49F900DA49F800D911DE1
:10E8B00011240895B7FF0C944F740E944F74821B6B
:10E8C000930B0895DB018F939F930E944F74BF9128
:10E8D000AF91A29F800D911DA39F900DB29F900DAF
:10E8E0001124089597FB072E16F4009407D077FDA6
:10E8F00009D00E94D07407FC05D03EF49095819514
:10E900009F4F0895709561957F4F0895A1E21A2E4B
:10E91000AA1BBB1BFD010DC0AA1FBB1FEE1FFF1FC3
:10E92000A217B307E407F50720F0A21BB30BE40B13
:10E93000F50B661F771F881F991F1A9469F760955A
:10E940007095809590959B01AC01BD01CF01089514
:10E95000052E97FB16F4009407D057FD0DD00E94AA
:10E96000867407FC09D07EF490958095709561952A
:10E970007F4F8F4F9F4F089550954095309521952B
:10E980003F4F4F4F5F4F0895A29FB001B39FC0010B
:10E99000A39F01D0B29F700D811D1124911D089578
:10E9A000AA1BBB1B51E107C0AA1FBB1FA617B707B5
:10E9B00010F0A61BB70B881F991F5A95A9F78095D1
:10E9C0009095BC01CD010895EE0FFF1F0590F491C5
:10E9D000E02D0994A0E0B0E0E0EFF4E70C94AA7A0F
:10E9E0008B016115710519F0FB01808391837C0116
:10E9F000F701C1907F01EF018C2D90E00E945877C4
:10EA0000892BB1F7FDE2CF1204C0C990DD24D39465
:10EA100005C02BE2C21201C0C990D12C7E0141E099
:10EA2000E41AF10843E050E06BE373E1C7010E9490
:10EA30006877892BE9F47E0182E0E80EF11C45E05D
:10EA400050E06EE373E1C7010E946877892B21F4DF
:10EA50007E01E7E0EE0EF11C0115110519F0F80139
:10EA6000F182E08210E0D0E0C0E8D110FBC0FFC02E
:10EA700043E050E063E473E1C7010E946877892BAB
:10EA800049F40115110509F4EFC02296F801D1836C
:10EA9000C083EAC060E070E0CB01E12CF12CEC2DEA
:10EAA000E053EA3048F5FD2DF2602D2D2870D2FE9E
:10EAB00006C0211127C02FEFE21AF20A23C0222339
:10EAC00019F041E0E41AF108A5E0B0E09B01AC01C7
:10EAD0000E944F74660F771F881F991F6E0F711D5C
:10EAE000811D911D6839E9E97E078E07E9E19E07DE
:10EAF00048F0FD2DF66006C0EE3F39F4D3FC3DC072
:10EB0000FD2DF860C990DF2ECACFE53311F0E53155
:10EB1000A1F5A881AD3219F4F0E1DF2A06C0AB32CD
:10EB200021F0219621E030E004C0A981229622E064
:10EB300030E0A053AA3018F0C21BD30B1EC0FE0158
:10EB400020E030E020384CE034075CF4A901440FA9
:10EB5000551F440F551F240F351F220F331F2A0F37
:10EB6000311DA191A053EF01AA3060F3D4FE03C080
:10EB7000319521953109E20EF31ED1FE07C0011532
:10EB8000110521F02197F801D183C0830E945471AF
:10EB90002D2D2370233029F0162FD72FC82F092FA2
:10EBA00007C0DC01CB01B058182FD92FCA2F0B2F6B
:10EBB00020E030E0A901612F7D2F8C2F902F0E9443
:10EBC000B470882309F454C0F7FE08C0F194E194AE
:10EBD000F10832E7C32E33E1D32E04C02AE5C22E5A
:10EBE00023E1D22E4601F8E18F1A910890E2A92E76
:10EBF000B12C15C0F6014591559165917491242F62
:10EC0000352F462F572F612F7D2F8C2F902F0E944D
:10EC10008973162FD72FC82F092FEA18FB08EA147B
:10EC2000FB0444F724E0C21AD108B594A794C81491
:10EC3000D904A9F7612F7D2F8C2F902F282F220F19
:10EC4000292F221F2F3F39F020E030E0A9010E9438
:10EC5000B47081110DC082E290E09093500E8093C9
:10EC60004F0E06C00FEF04C010E0D0E0C0EC0FE77D
:10EC7000612F7D2F8C2F902FCDB7DEB7ECE00C9459
:10EC8000C67AA0E0B0E0E7E4F6E70C94A67A2B01A0
:10EC90008A016115710519F0FB01808391830115CB
:10ECA000110539F09801225031092332310508F05D
:10ECB000E6C07C01F701C1917F013F018C2F90E0FC
:10ECC0000E945877892BB1F7CD3229F4F701C19111
:10ECD0003F01D1E006C0CB3219F4F701C1913F01E9
:10ECE000D0E00115110509F4D8C00031110581F4F7
:10ECF000D0C0F3018081883719F0883509F0C3C08E
:10ED0000F301C181F2E06F0E711CD26000E110E0EE
:10ED100008301105D9F024F402301105F9F407C0C8
:10ED20000A30110551F000311105C1F425C0C12C84
:10ED3000D12CE12C30E4F32E24C00AE010E02CECBE
:10ED4000C22EDC2CEC2C2CE0F22E1BC008E010E0D4
:10ED5000C12CD12CE12C90E1F92E13C0980144274D
:10ED600037FD4095542F60E070E080E090E80E940D
:10ED7000867469017A0105C0C12CD12CE12C88E090
:10ED8000F82E40E060E070E0CB014801AA2497FC37
:10ED9000A094BA2CEC2FE053EA3060F02C2F2154D1
:10EDA0002A3110F4E75006C02C2F21562A3128F5BD
:10EDB000EC2FE7552E2F30E020173107F4F447FDF4
:10EDC00018C0C616D706E806F90680F09B01AC010C
:10EDD000C501B4010E9462746E0F711D811D911DE9
:10EDE00061307105810520E8920710F04FEF01C0F6
:10EDF00041E0F301C1913F01CDCF4114510491F0A5
:10EE0000442339F0F1E06F1A7108F20171826082D7
:10EE100009C0D1FF1BC0F2E06F1A7108F2017182C4
:10EE2000608214C047FF12C0D0FF05C060E070E0F0
:10EE300080E090E804C06FEF7FEF8FEF9FE722E262
:10EE400030E03093500E20934F0E16C0D0FF08C014
:10EE500090958095709561957F4F8F4F9F4F0CC017
:10EE600097FF0AC082E290E09093500E80934F0E7D
:10EE70006FEF7FEF8FEF9FE76B017C0112C0C12C1A
:10EE8000D12C76010EC0C0E30115110509F45ECF47
:10EE90003FCFC03309F03CCF2CCFC03309F04DCF6A
:10EEA00028CFB601C701CDB7DEB7E0E10C94C27A36
:10EEB0009111A7C2803219F089508550D0F708957A
:10EEC0009111089581548A5108F4805E855A0895FD
:10EED000FB01DC014150504088F08D9181341CF0E1
:10EEE0008B350CF4805E659161341CF06B350CF44D
:10EEF000605E861B611171F3990B0895881BFCCF2E
:10EF0000FB01DC0104C08D910190801921F4415076
:10EF10005040C8F7881B990B0895FB01DC0102C023
:10EF200001900D9241505040D8F70895FB01DC014B
:10EF30000D900020E9F7119701900D920020E1F764
:10EF40000895FC018191861721F08823D9F799272C
:10EF500008953197CF010895FB01DC0101900D92D6
:10EF60000020E1F70895FB01DC014150504030F0F2
:10EF70008D910190801919F40020B9F7881B990B25
:10EF80000895FB01DC014150504048F001900D9282
:10EF90000020C9F701C01D9241505040E0F708958C
:10EFA000FB0151915523A9F0BF01DC014D9145179B
:10EFB0004111E1F759F4CD010190002049F04D9144
:10EFC00040154111C9F3FB014111EFCF81E090E001
:10EFD00001970895A0E1B0E0E0EFF7E70C94B27A72
:10EFE0000F89188D86E08C831A8309838FEF9FE742
:10EFF0009E838D83AE01455E5F4F588B4F87698D31
:10F000007A8DCE0101960E940E78EF81F885E00F8F
:10F01000F11F10826096E4E00C94CE7AACE0B0E090
:10F02000E4E1F8E70C94A47A7C016B018A01FC010D
:10F0300017821682838181FFC7C188248394912C13
:10F040008C0E9D1EF7019381F60193FD859193FF30
:10F0500081916F01882309F4B3C1853239F493FD9E
:10F06000859193FF81916F01853229F4B70190E07A
:10F070000E941A7AE7CF712C312C20E02032A8F4BC
:10F080008B3261F028F4803251F0833271F40BC07E
:10F090008D3239F0803349F4216028C02260246029
:10F0A00025C0286023C0206121C027FD27C0382F3C
:10F0B00030533A3078F426FF06C0FAE07F9E300DD8
:10F0C0001124732E13C08AE0389E300D1124332E84
:10F0D00020620CC08E3221F426FD72C1206406C06D
:10F0E0008C3611F4206802C0883641F4F60193FD95
:10F0F000859193FF81916F018111C0CF982F955415
:10F10000933018F09052933028F40C5F1F4FFFE3B8
:10F11000F9830DC0833631F0833771F0833509F000
:10F120005EC023C0F801808189830E5F1F4F662473
:10F130006394712C540115C02801F2E04F0E511C4C
:10F14000F801A080B18026FF03C0672D70E002C0E7
:10F150006FEF7FEFC5012C870E940F7A3C0182017F
:10F160002C856FE7262E222218C02801F2E04F0ED0
:10F17000511CF801A080B18026FF03C0672D70E00C
:10F1800002C06FEF7FEFC5012C870E94047A3C011B
:10F190002C8550E8252E222A820123FC1CC006C0A3
:10F1A000B70180E290E00E941A7A3A94832D90E0B1
:10F1B00068167906A8F30FC0F50127FC859127FE94
:10F1C00081915F01B70190E00E941A7A31103A9460
:10F1D000F1E06F1A71086114710471F7EEC08436A2
:10F1E00011F0893641F5F80127FF07C06081718170
:10F1F000828193810C5F1F4F08C0608171818827D5
:10F2000077FD8095982F0E5F1F4F4FE6642E622288
:10F2100097FF09C090958095709561957F4F8F4FAE
:10F220009F4FF0E86F2A2AE030E0A4010E94467A5E
:10F23000A82EA81844C0853731F43FEEB32EB22271
:10F240002AE030E024C099EFB92EB2228F36B9F00F
:10F2500020F4883509F0B4C00DC0803721F088371C
:10F2600009F0AEC002C020E1B22AB4FE0BC084E0B7
:10F27000B82A08C024FF09C0E6E0BE2A06C028E07C
:10F2800030E005C020E130E002C020E132E0F801CA
:10F29000B7FE07C060817181828193810C5F1F4F2F
:10F2A00006C06081718180E090E00E5F1F4FA40175
:10F2B0000E94467AA82EA8188FE7682E6B2066FE5B
:10F2C0000BC0362D3E7FA71450F464FE0AC062FCCA
:10F2D00008C0362D3E7E05C0BA2C362D03C0BA2C90
:10F2E00001C0B72C34FF0DC0FE01EA0DF11D808175
:10F2F000803311F4397E09C032FF06C0B394B39451
:10F3000004C0832F867809F0B39433FD14C030FF16
:10F310000FC07A2CB31460F4730C7B18B32C08C0A4
:10F32000B70180E290E03C870E941A7AB3943C8552
:10F33000B314B0F304C0B31410F43B1801C0312C63
:10F3400034FF12C0B70180E390E03C870E941A7A34
:10F350003C8532FF1EC031FF03C088E590E002C04B
:10F3600088E790E0B7010CC0832F867891F031FDDB
:10F3700002C080E201C08BE237FD8DE2B70190E070
:10F380000E941A7A06C0B70180E390E00E941A7AC0
:10F390007A94A714C0F3AA94F401EA0DF11DB70101
:10F3A000808190E00E941A7AA110F5CF06C0B701C3
:10F3B00080E290E00E941A7A3A943110F8CF42CE5F
:10F3C000F7012681378102C02FEF3FEFC9012C964C
:10F3D000E2E10C94C07AF999FECF92BD81BDF89A12
:10F3E000992780B50895262FF999FECF1FBA92BDAF
:10F3F00081BD20BD0FB6F894FA9AF99A0FBE019616
:10F400000895992788270895FC0105906150704060
:10F410000110D8F7809590958E0F9F1F0895FC01DD
:10F420006150704001900110D8F7809590958E0F33
:10F430009F1F08950F931F93CF93DF938C01EB01D0
:10F440008B8181FD03C00FEF1FEF1AC082FF0DC03B
:10F450002E813F818C819D812817390764F4E881D2
:10F46000F9810193F983E88306C0E885F985802F47
:10F470000995892B41F78E819F8101969F838E8309
:10F48000C801DF91CF911F910F910895FA01AA272A
:10F49000283051F1203181F1E8946F936E7F6E5FD7
:10F4A0007F4F8F4F9F4FAF4FB1E03ED0B4E03CD085
:10F4B000670F781F891F9A1FA11D680F791F8A1F68
:10F4C000911DA11D6A0F711D811D911DA11D20D0CF
:10F4D00009F468943F912AE0269F11243019305D89
:10F4E0003193DEF6CF010895462F4770405D41937A
:10F4F000B3E00FD0C9F7F6CF462F4F70405D4A33C7
:10F5000018F0495D31FD4052419302D0A9F7EACF8E
:10F51000B4E0A6959795879577956795BA95C9F7BD
:10F5200000976105710508959B01AC010A2E0694B0
:10F530005795479537952795BA95C9F7620F731F69
:10F54000841F951FA01D08952F923F924F925F92A6
:10F550006F927F928F929F92AF92BF92CF92DF92E3
:10F56000EF92FF920F931F93CF93DF93CDB7DEB748
:10F57000CA1BDB0B0FB6F894DEBF0FBECDBF0994DC
:10F580002A88398848885F846E847D848C849B8433
:10F59000AA84B984C884DF80EE80FD800C811B8141
:10F5A000AA81B981CE0FD11D0FB6F894DEBF0FBE70
:10F5B000CDBFED01089513E1C8E7D3E104C0FE011A
:10F5C0000E94E6742296CA37D107C9F7F894FFCF94
:10F5D0006400640000803B4500803B4500007043B0
:10F5E000000000000080BB440160EA0000CDCCCCEC
:10F5F0003D0000524300007A430101010101000077
:10F60000803FE7849145AECF1A3D00004041FF3F67
:10F61000FF3F0171DBB64271DBB64200007A450064
:10F62000C05A440000FA430000FA430000A0400022
:10F63000003442E8030000E803000032000000FA52
:10F640000000004D313130002569206D696E2C209D
:10F65000256920736563005573696E67204465668C
:10F6600061756C742073657474696E67733A0048D1
:10F6700020004C20004D31303420496E76616C6999
:10F680006420657874727564657220004D31303580
:10F6900020496E76616C6964206578747275646562
:10F6A0007220004D31303920496E76616C696420DA
:10F6B000657874727564657220003F006F6B00207E
:10F6C000703A0020693A0020643A0020633A0054FE
:10F6D00000496E76616C6964206578747275646542
:10F6E000720041637469766520457874727564654B
:10F6F000723A20004D32390058595A450000010035
:10F700000F0015000E001200FFFF160017000E007C
:10F710001300FFFF030002001A001400FFFFFFFFA9
:10F72000FFFF0A00FFFF010000000E000D000700B0
:10F73000FFFFFFFF060000000000000000000000C7
:10F7400000000000000000000000000000002E008B
:10F75000000000000839FC384E6D5374657072610A
:10F76000746520746F2068696768203A20005049EA
:10F7700044204175746F74756E6520737461727482
:10F78000002F0043616E6E6F74206F70656E207382
:10F790007562646972006175746F25692E67004D2A
:10F7A0003233202573004D3234004D383420582038
:06F7B00059205A2045001B
:00000001FF
